:020000040000FA
:1000000000020400000000004C8900004C89000040
:100010004C8900004C8900004C8900004C8900008C
:100020004C8900004C8900004C8900004C8900007C
:100030004C8900004C8900004C8900004C8900006C
:100040004C8900004C8900004C8900004C8900005C
:100050004C8900003C5B0000625B00004C890000A2
:100060004C8900004C8900004C8900004C8900003C
:100070004C8900004C8900004C8900004C8900002C
:100080004C8900004C8900004C8900004C8900001C
:100090004C8900004C8900004C8900004C8900000C
:1000A0004C8900004C8900004C8900004C890000FC
:1000B0004C8900004C8900004C8900004C890000EC
:1000C0004C8900004C8900004C8900004C890000DC
:1000D0004C8900004C8900004C8900004C890000CC
:1000E0004C8900004C8900004C8900004C890000BC
:1000F0004C8900004C8900004C8900004C890000AC
:100100004C8900004C8900004C8900004C8900009B
:100110004C8900004C8900004C8900004C8900008B
:100120004C8900004C8900004C8900004C8900007B
:100130004C8900004C8900004C8900004C8900006B
:100140004C8900004C8900004C8900004C8900005B
:100150004C8900004C8900004C8900004C8900004B
:100160004C8900004C8900004C8900004C8900003B
:100170004C8900004C8900004C8900004C8900002B
:100180004C8900004C8900004C8900004C8900001B
:100190004C8900004C8900004C8900004C8900000B
:1001A0004C8900004C8900004C8900004C890000FB
:1001B0004C8900004C8900004C8900004C890000EB
:1001C0004C8900004C8900004C8900004C890000DB
:1001D0004C8900004C8900004C8900004C890000CB
:1001E0004C8900004C8900004C8900004C890000BB
:1001F0004C8900004C8900004C8900004C890000AB
:10020000FFFFFF00FFFFFF004C8900004C8900004A
:100210004C8900004C8900004C8900004C8900008A
:100220004C8900004C8900004C8900004C8900007A
:100230004C8900004C8900004C8900004C8900006A
:100240004C8900004C8900004C8900004C8900005A
:100250004C8900003C5B0000625B00004C890000A0
:100260004C8900004C8900004C8900004C8900003A
:100270004C8900004C8900004C8900004C8900002A
:100280004C8900004C8900004C8900004C8900001A
:100290004C8900004C8900004C8900004C8900000A
:1002A0004C8900004C8900004C8900004C890000FA
:1002B0004C8900004C8900004C8900004C890000EA
:1002C0004C8900004C8900004C8900004C890000DA
:1002D0004C8900004C8900004C8900004C890000CA
:1002E0004C8900004C8900004C8900004C890000BA
:1002F0004C8900004C8900004C8900004C890000AA
:100300004C8900004C8900004C8900004C89000099
:100310004C8900004C8900004C8900004C89000089
:100320004C8900004C8900004C8900004C89000079
:100330004C8900004C8900004C8900004C89000069
:100340004C8900004C8900004C8900004C89000059
:100350004C8900004C8900004C8900004C89000049
:100360004C8900004C8900004C8900004C89000039
:100370004C8900004C8900004C8900004C89000029
:100380004C8900004C8900004C8900004C89000019
:100390004C8900004C8900004C8900004C89000009
:1003A0004C8900004C8900004C8900004C890000F9
:1003B0004C8900004C8900004C8900004C890000E9
:1003C0004C8900004C8900004C8900004C890000D9
:1003D0004C8900004C8900004C8900004C890000C9
:1003E0004C8900004C8900004C8900004C890000B9
:1003F0004C8900004C8900004C8900004C890000A9
:10040000AF032200007F22000001880000000000EE
:100410000C000700A02F2800010020001100070099
:10042000000020000000E000020032000000020096
:10043000000000007A870200000000000040DA009F
:100440000000FE004440A900E02020000000E00081
:100450000300320000002000A00188004440A800F2
:100460000000060091018800800078000000EB0089
:1004700015003700E280400032A0B4009101BA00BC
:10048000E280400032A0B4009102BA00E280400055
:1004900032A0B4000002EB00472BDE00F507B200EB
:1004A000602CE10004003A000059EB008301E900F0
:1004B000FDFF3E00040037006128E100010032002A
:1004C0000082EB00040007001101BA000200E00006
:1004D000E8FF3A00000006003159BA008301E90044
:1004E0000C0032002159BA008301E90008003200F3
:1004F0000400E00003003A00E280400032A0B400B3
:10050000F5FF370011D9BA008301E900FAFF3A007C
:100510008100E800E180400032A0B4000000060045
:1005200000000000000000000000000000000000CB
:1005300000000000000000000000000000000000BB
:1005400000000000000000000000000000000000AB
:10055000000000000000000000000000000000009B
:10056000000000000000000000000000000000008B
:10057000000000000000000000000000000000007B
:10058000000000000000000000000000000000006B
:10059000000000000000000000000000000000005B
:1005A000000000000000000000000000000000004B
:1005B000000000000000000000000000000000003B
:1005C000000000000000000000000000000000002B
:1005D000000000000000000000000000000000001B
:1005E000000000000000000000000000000000000B
:1005F00000000000000000000000000000000000FB
:1006000000000000000000000000000000000000EA
:1006100000000000000000000000000000000000DA
:1006200000000000000000000000000000000000CA
:1006300000000000000000000000000000000000BA
:1006400000000000000000000000000000000000AA
:10065000000000000000000000000000000000009A
:10066000000000000000000000000000000000008A
:10067000000000000000000000000000000000007A
:10068000000000000000000000000000000000006A
:10069000000000000000000000000000000000005A
:1006A000000000000000000000000000000000004A
:1006B000000000000000000000000000000000003A
:1006C0000000000000000000889FBE008A9FBE005E
:1006D000010578000100E0000400350008003C003E
:1006E0000000E0002000320005003700600010002C
:1006F000E080180002003B0001F02C001A003700D7
:100700000004BE006011B8006B0920000982CF0010
:10071000020039000882CF000441B0006942520053
:100720000E00320008003B0082817100610164000C
:100730008904D1000884D3008B05E8000442E80056
:10074000F9FF3A00050037000804440089844C0092
:100750008B05E9000442E900FBFF3A002C01070089
:100760000AF0A70001F0A0004F05BE004F04BE0034
:1007700000000600F4FF2F004B013700140020009A
:1007800049013700889FBE008A9FBE008C1F7800F9
:10079000600107006701330003866C006450E100CC
:1007A0002E0032006420E100330032006150E1008D
:1007B0002F0032006120E1003100320085855500B4
:1007C000EB07B000090020000804200005003700F6
:1007D0000804440089844C000A00310006034300E9
:1007E00087834B000001530081815B00F8FF3300D9
:1007F0000203BE000800A0000804440089844C00E5
:10080000F6FF3900C639DD008301730001003200B4
:10081000130020008904D1000884D3000998A300A4
:10082000050032000800A7000300A0008904D100E1
:100830000884D3008B05E8008904D1000884D30024
:100840000001EB000281D200F100070001F0A100DD
:100850000CF0A70001F0A0003F0137006420E10088
:10086000410132000801BE000200BE00F7FF370060
:100870006120E1003C0132006000B800F3FF370066
:100880000000200001F82700F0FF370003F0A2006D
:10089000889FBE008A9FBE008C1F78001D01070044
:1008A000240133006450E1004F0032006420E10075
:1008B0005200320003826C0007003B000905D000A3
:1008C0000306D000820F54000C065D0002003900C0
:1008D0000200320089017800030678008582550005
:1008E00004003D000003FD008103FD008502EA00D5
:1008F0008B854200840F720002003B0060001000F4
:10090000E08018006011B8000005EB007A28E100D3
:100910000A00390006007800C75DDD00F707B20065
:10092000878075002D003700828171000A017800F0
:10093000610560008180D1000080D3008502E9005C
:10094000F9FF3B00060440008784480002003B009A
:1009500060041400E0841C000988A3000700320032
:100960008A81710082817100610164008904D10073
:100970000884D3008B05E800170037000978A3002E
:1009800013003A000B00E000130034008B05E9006F
:100990000804440089844C000A4474000978A300C8
:1009A0000D003A000B00E000070034008B05E90061
:1009B0000804440089844C0001003A000B00200028
:1009C0000978A300F7FF32000001EB0002003700B6
:1009D000828171000A0178008D0007000CF0A700E9
:1009E00001F0A000DC0037006420E10002003A00C2
:1009F000838F6C00DC0033000801BE000200BE00E3
:100A0000D5003700889FBE008A9FBE008C1F7800EB
:100A1000C0000700C700330003866C006450E1008B
:100A2000240032006420E100270032006150E10020
:100A3000220032006120E100210032008B8542005B
:100A4000EB07B1000134B800003AB80008044200D6
:100A500089844A00013AB8000030B800888040001C
:100A600009014A0004003300000040008180480072
:100A7000020149008B05E900C909DD00830170000E
:100A80000100320013002000C814DE004814DD000D
:100A90004709DE001200B200C808DE0008847000BA
:100AA0005B00070001F0A1000CF0A70001F0A0001E
:100AB000A90037006120E100AB0032000801BE0050
:100AC0000200BE00F7FF37006150E100FCFF3A0072
:100AD000A50037000001BE00A60007000470A700B3
:100AE00003F0A10003F8A30013003A006509B10068
:100AF00010003200090035006928E10002003500CD
:100B0000010028000000050000004000818048002E
:100B10008502E900FCFF3A0000000600F88F420061
:100B2000050035008100D1000080D3008502E80077
:100B3000FCFF3A00000006008000EB00000005000A
:100B40006022B800060220000000D0008180D200A0
:100B50000482D2008582D2000000A000020252006E
:100B600083825A00030031000202420083824A005D
:100B70000000A1000603E900F3FF3A0000000600B0
:100B8000EFFF07000400BE00000006000001BE00E9
:100B9000780007000470A70003F0A1006509B10008
:100BA000160032000D0035006828E100060035000F
:100BB000F0FF2F00F1FF27000300E00013003B00CF
:100BC000010028000000050000004000818048006E
:100BD0008502E900FCFF3A0008003700F88F420068
:100BE00002003C008000EB00000005008100D10005
:100BF0000080D3008502E800FCFF3A000300E0001B
:100C000002003B0060001000E080180000000600B9
:100C100081002000618055000B003D000B0020008A
:100C200061FE2F000100E1001D003400828171008F
:100C3000610164008904D1000884D3000000E80049
:100C4000FAFF3A00710020006100640003007000A8
:100C5000020060000900320061044400E0844C009E
:100C60000988A500050032008B05E8006808E1004E
:100C700002003A008904D1000884D300F20F20005A
:100C80000258E10005003D00C75DDD00F907B20034
:100C90008980750008007800000006000BF8270026
:100CA0008B00780000000500889FBE008A9FBE0070
:100CB000841F7800170007004F00780011003300F0
:100CC000F0FF2F00838F6C0006003B0004056500D9
:100CD0000A00A7000800370009F0A6001000200055
:100CE00008003700820F5400838F5C000300390036
:100CF0001000200001003E000000200009F0A700C5
:100D00000000EA004F05BE004F04BE000000E000F6
:100D1000000006000004BE00160007000003BE002D
:100D20000405BE000200BE0012000700844F7500DB
:100D3000000006000200BE006450E100050036001D
:100D40006420E100020036000968A30001003A00B7
:100D50000800BE000160A0004F0678004F05BE00ED
:100D60004F04BE0000000600F0FF2F00F1FF270037
:100D7000F9FF3700C70ADE00F107B200F50FB20035
:100D800008003200E1CF4200020032000170A000F2
:100D900024000500810F70000100320004080500E6
:100DA00044000500810F700002003A0014000500A5
:100DB0008502E9000000400081C04800FCFF3B00C4
:100DC0000170A000240005003E2000000008000083
:100DD00020080000001B00005B440000001B000016
:100DE0005B000000440000001B5B000043000000AB
:100DF0001B5B0000324B00000D00000043000000B0
:100E0000001B00005B32000044000000576100003E
:100E1000726E0000696E0000673A0000206E0000EC
:100E20006F200000766F00006C74000061670000A6
:100E3000652000006F6E00002056000070750000F5
:100E40006C6C00007570000020700000696E00007E
:100E5000002000003D200000005600005245000028
:100E600047200000746F00006F2000006C6F0000CE
:100E7000772C0000206900007320000074680000D7
:100E800065720000652000006120000073680000AA
:100E90006F720000743F0000002E0000203C000034
:100EA000003E0000002E0000200000000D0A00009F
:100EB00028000000293E00002000000042750000CC
:100EC000732000005069000072610000746500002A
:100ED000207600003300000046690000726D0000BB
:100EE000776100007265000020760000352E00005A
:100EF0003920000028720000353200003929000036
:100F0000200000002028000032340000464A000083
:100F1000363400004741000030300000322000002D
:100F20000041000033000000423400000042000095
:100F30003500000042380000005500004E4B000014
:100F40000029000000490000090000004F090000CE
:100F500000480000090000004C09000000450000A6
:100F60006E7400006572000020720000617700005E
:100F700020760000616C00007565000020660000AE
:100F80006F72000020420000524700000000000085
:100F90004C45000054000000494600000054000089
:100FA000484500004E000000454C0000534500003D
:100FB000004700004F5400004F000000474F000062
:100FC00053550000420000005245000054550000F7
:100FD000524E000000520000454D0000005000003D
:100FE000524900004E540000004900004E500000DD
:100FF00055540000004600004F520000005400000D
:101000004F0000004E450000585400000052000000
:1010100045410000440000004441000054410000EC
:1010200000530000544100005254000052000000E0
:10103000535400004152000054000000535400007B
:101040004F50000052000000535400004F50000069
:1010500000530000454E00004400000052450000CF
:10106000434500004956000045000000434C000085
:101070004B000000444100005400000042490000C1
:10108000545200004541000044000000414400006B
:10109000430000004155000058500000494E000038
:1010A000005000005355000000500000554C000057
:1010B0004C55000050000000444500004C41000029
:1010C0005900000041550000580000004652000041
:1010D0004551000000440000555400005900000034
:1010E0004D410000435200004F000000454E0000FB
:1010F0004400000000520000554E0000004C00006B
:1011000049530000540000004558000049540000B5
:10111000004400004542000055470000004E00001A
:101120004557000000000000306200000030000061
:10113000303000002C000000303000000030000093
:1011400031320000333400003536000037380000FB
:101150003941000042430000444500004630000091
:101160007800000000290000002000005700000067
:10117000205200000049000032430000310000000E
:101180000808000008080000080000000000000037
:10119000204800007A0000000000000042420000E9
:1011A000494F00003100000052410000573100005B
:1011B00000000000314100004C530000000000001E
:1011C0004F43000044310000000000000000000018
:1011D00000000000290000000000000000000000E6
:1011E000000000002800FA000000EB00600F9800EB
:1011F0000000EB00805788000000EB00705788006B
:1012000070578000200798000000EB00100798003E
:101210000000EB00000F78000000EB00A040880009
:101220000000EB00905788000000EB00400798009A
:101230000000EB00000F9800140037000000EB00E6
:10124000600798000B0037000E089000EE00900039
:101250004500DD008100400040AF2000808040005C
:101260000040EB00804878006E0090000000E8002D
:10127000600798006E009000FF0F5000F2FF3400EE
:101280000E0890000000E800000F98000E08900083
:10129000E40F5000E9FF34000000EB00A05C880080
:1012A000A1408000E00220000088B9006102200017
:1012B00080804000008320000080400088560200AB
:1012C00000000000D140800000202000008060006D
:1012D0000000E0000400320071002000C05920002E
:1012E0009A84020000000000406E28008856020028
:1012F0000000000032043700A05C80000000E00025
:1013000063003200A05C80000000E900A05C88005F
:101310000000EB00600798001E0037007257800045
:10132000A05C8000EE0090004500DD0081004000E0
:1013300040AF20000080400090407800E09E2000F8
:101340000000410001487800A05C8000EE009000A1
:101350004500DD008100400040AF200000804000DB
:1013600010407800E45A020000000000705780002E
:101370000000E800705788006E0090000000E80050
:101380006007980071578000F00F20000080600017
:1013900070578800A05C8000EE0090004500DD00E2
:1013A0008100400040AF20000080400010407800E5
:1013B0000004E000D9FF3A000000EB00A05C8800C8
:1013C00033003700A09C200010407800644060008B
:1013D0000004E0002E003200A1408000E002200066
:1013E0000088B900FA00400000832000008040001F
:1013F00010007800000001000000E000240032002E
:10140000A1408000E00220000088B90061022000B5
:101410008080400000832000008040008856020049
:1014200000000000406E2800885602000000000006
:101430008157800070578000808F50001400320068
:1014400080578000600798000D003700EE00900084
:10145000E09E20000080400010407800E45A020026
:1014600000000000EE009000F00F200000806000FF
:10147000600798006E0090000000E8006007980088
:10148000EE00900070578000808F5000EFFF3A0010
:10149000C65A0200000000000004E000C9FF32004C
:1014A00022C2BF00624060000004E000050032007C
:1014B00010118000D1FF2F00010060001011880082
:1014C000BF033700D25A020000000000604F9800AE
:1014D0006E4890000080FB006101B900021798007F
:1014E00013179800F0072000010020000E11900053
:1014F0009E119000800F5100818F59003C033E00E7
:101500000E1090009E109000006001002D03370027
:10151000E20237003E01370035033700D8003700BC
:10152000F9023700530137003103370077003700E5
:101530002F0337000F0337002D0337002C0337002C
:101540000C033700FE013700290337005A0137002A
:10155000270337002603370025033700240337000D
:10156000230337002203370021033700200337000D
:101570001F0337001E033700020137001C0337002A
:101580001B0337001A03370019033700180337000D
:10159000170337001603370015033700140337000D
:1015A000130337001203370011033700100337000D
:1015B0000F0337000E0337000D0337000C0337000D
:1015C0000B0337000A03370009033700080337000D
:1015D000070337000603370005033700040337000D
:1015E000030337000203370001033700000337000D
:1015F000FF023700FE023700FD023700FC02370011
:10160000FB023700FA023700F9023700F802370010
:10161000F7023700F6023700F5023700F402370010
:10162000F3023700F2023700F1023700F002370010
:10163000EF023700EE023700ED023700EC02370010
:10164000EB023700EA023700E9023700E802370010
:10165000E7023700E6023700E5023700E402370010
:10166000E3023700E2023700E1023700E002370010
:10167000DF023700DE023700DD023700DC02370010
:10168000DB023700DA023700D9023700D802370010
:10169000D7023700D6023700D5023700D402370010
:1016A000D3023700D2023700D1023700D002370010
:1016B000CF023700CE023700CD023700CC02370010
:1016C000CB023700CA023700C9023700C802370010
:1016D000C7023700C6023700C5023700C402370010
:1016E000C3023700C2023700C1023700C002370010
:1016F000BF023700BE023700BD023700BC02370010
:10170000BB023700BA0237005D0037008157800006
:101710002E009000810F500055003200715780005C
:101720002E009000810F500010003A00705780008A
:101730008000E900F00F20000080600070578800F2
:1017400071578000E09E2000808040000040EB0048
:10175000804878007157800021079800706E28003B
:101760008856020000000000150337000000EB005F
:10177000000F98002E0090008000E900F00F20007C
:101780000080600020079800B06E28008856020094
:10179000000000002E019000620798002100370031
:1017A0006E0190006E0090008000E800E09E200036
:1017B0000080400090407800E09E20000000410042
:1017C00001487800EE009000E09E2000008040007C
:1017D000104078000004E00007003200EE009000A6
:1017E000E09E20000080400010407800E45A020093
:1017F000000000000300370000C2B300E45A0200FA
:10180000000000000E0890000000E800000F9800A3
:101810006E0090008000E800F00F20000080600063
:1018200060079800EE00900070578000808F500095
:10183000DBFF3A00705780008000E900F00F2000C5
:101840000080600070578800F06E28008856020003
:10185000000000000E089000205902000000000067
:10186000206F28008856020000000000D4023700D4
:1018700070C0B300E45A020000000000D00237003C
:10188000715780002E009000810F50003900320007
:101890000000EB00000F9800AE0190006307980075
:1018A000210037006E0190006E0090008000E8007B
:1018B000E09E20000080400090407800E09E2000E4
:1018C0000000410001487800EE009000E09E2000FA
:1018D00000804000104078000004E0000700320063
:1018E000EE009000E09E2000008040001040780054
:1018F000E45A0200000000000300370000C2B300F9
:10190000E45A0200000000000E0890000000E80009
:10191000000F98006E0090008000E800F00F20009B
:101920000080600060079800EE0090007057800013
:10193000808F5000DBFF3A00705780008000E90084
:10194000F00F20000080600070578800F06E2800C3
:1019500088560200000000000E0890002059020086
:1019600000000000206F28008856020000000000E0
:101970009302370070C0B300E45A02000000000078
:101980008F023700D25A020000000000604F98001A
:10199000EE489000B0C5B30080CF500088023A00F6
:1019A000D25A020000000000604F98006E4890007C
:1019B0000080FB00700F980020042000FE089000BB
:1019C000808F5000DE003200200420007E0990004D
:1019D000800F510005003C0010042000FE0990001B
:1019E000808F51003400320075023700300420002F
:1019F000FE089000808F50001E003200400420003E
:101A00007E099000800F5100010032006C02370007
:101A10004E009000E40F500005003400E47702000F
:101A2000000000000000EB0040079800640237004F
:101A3000815780002E009000810F50000900320075
:101A40002E0090008000E900F00F20000080600070
:101A500020079800B06E28008856020000000000A1
:101A60005702370070C0B300E45A020000000000C3
:101A700053023700715780002E009000810F5000F4
:101A8000090032002E0090008000E800F00F2000D6
:101A90000080600020079800406F280088560200F0
:101AA000000000004602370070C0B300E45A020094
:101AB00000000000420237000000EB00000F780039
:101AC000805780000000E90080007800F00F2000BF
:101AD00000806000600798008D003700EE009000E5
:101AE000E09E200000804000104078000004E000EC
:101AF00082003A006E0090008000E900F00F2000A4
:101B000080806000E09E200000804000104078004F
:101B10000004E000790032001E0FE8001E00900073
:101B20009E0F1000750036001E0090000000E800B7
:101B3000100798008157800070578000808F5000F8
:101B4000140032000A00370071578000E09E200028
:101B5000808040000040EB00804878007057800093
:101B60008000E900F00F20000080600070578800BE
:101B70007157800080578000808F5000F2FF3A003C
:101B800071578000E09E2000808040000040EB0004
:101B9000804878006E0090008000E900F00F20007F
:101BA00000806000000F9800110037008E08900040
:101BB000E09E200000804000104078000004E0001B
:101BC00006003A000E0890008000E800F00F2000A8
:101BD0000080600050079800090037000E08900050
:101BE0008000E900F00F200000806000000F9800E6
:101BF0008E08900070578000808F5000EBFF3A00F5
:101C0000806F28008856020000000000A14080007C
:101C1000E00220000088B9006102200080804000BE
:101C20000083200000804000885602000000000071
:101C3000D140800000202000008060000000E00013
:101C40000400320071002000C05920009A84020074
:101C500000000000406E28008856020000000000CE
:101C6000DE019000030F9800180037008E089000E6
:101C7000E09E20000080400010407800E45A0200FE
:101C800000000000725780008E089000E09E200047
:101C90000080400090407800E09E2000000041005D
:101CA00001487800705780008000E800F00F2000A5
:101CB00000806000705788000E0890008000E800E7
:101CC000F00F200000806000000F98008E08900048
:101CD0006E009000808F5000E4FF3A007157800042
:101CE000E09E2000808040000040EB0080487800AB
:101CF0007057800020079800090037006E009000A0
:101D00008000E900F00F200000806000600798006C
:101D1000EE00900070578000808F50006FFF3A00F7
:101D2000EE00900070578000808F5000A4013A00B0
:101D300070C0B300E45A020000000000A0013700A8
:101D40000000EB00000F7800805780000000E900E1
:101D500080007800F00F200000806000600798008D
:101D60008E003700EE009000E09E200000804000D2
:101D7000104078000004E00083003A006E009000FC
:101D80008000E900F00F200080806000E09E2000CD
:101D900000804000104078000004E0007A0032002B
:101DA0001E0FE8001E0090000000E9009E0F50008A
:101DB00075003A001E0090000000E900100798002E
:101DC0008157800070578000808F500014003200CF
:101DD0000A00370071578000E09E2000808040009C
:101DE0000040EB0080487800705780008000E900D8
:101DF000F00F20000080600070578800715780004D
:101E000080578000808F5000F2FF3A0071578000A9
:101E1000E09E2000808040000040EB008048780079
:101E20006E0090008000E900F00F2000008060004C
:101E3000000F9800110037008E089000E09E2000EF
:101E400000804000104078000004E00006003A00E6
:101E50000E0890008000E800F00F20000080600075
:101E600050079800090037000E0890008000E90034
:101E7000F00F200000806000000F98008E08900096
:101E800070578000808F5000EBFF3A00806F280071
:101E90008856020000000000A1408000E0022000FF
:101EA0000088B9006102200080804000008320008B
:101EB000008040008856020000000000D1408000F1
:101EC00000202000008060000000E00004003200DC
:101ED00071002000C05920009A8402000000000018
:101EE000406E28008856020000000000DE009000CE
:101EF000010F9800180037008E089000E09E200027
:101F00000080400010407800E45A02000000000009
:101F1000725780008E089000E09E200000804000F4
:101F200090407800E09E20000000410001487800C9
:101F3000705780008000E800F00F200000806000F3
:101F4000705788000E0890008000E800F00F200015
:101F500000806000000F98008E0890006E009000D6
:101F6000808F5000E4FF3A0071578000E09E20000F
:101F7000808040000040EB0080487800725780006D
:101F800022079800090037006E0090008000E900E9
:101F9000F00F20000080600060079800EE009000C5
:101FA00070578000808F50006EFF3A00EE00900066
:101FB00070578000808F500001013A001E00900091
:101FC000E10F500031003A00806F2800885602006F
:101FD00000000000A1408000E00220000088B9005D
:101FE00061022000808040000083200000804000CB
:101FF0008856020000000000D14080000020200030
:10200000008060000000E000040032007100200049
:10201000C05920009A84020000000000406E280091
:1020200088560200000000000A0037007157800047
:10203000E09E2000808040000040EB008048780057
:10204000705780008000E900F00F200000806000E1
:10205000705788007157800080578000808F500033
:10206000F2FF3A0071578000E09E2000808040001F
:102070000040EB00804878007357800023079800E9
:102080000000EB0010079800CD00370070C0B300CF
:10209000E45A020000000000C900370081578000A8
:1020A0002E009000810F50001300320081578000F5
:1020B0002E0090000100500080007800F00F2000FA
:1020C00000806000000F9800F06E28008856020023
:1020D000000000000E0890002059020000000000DF
:1020E000206F280088560200000000008057800002
:1020F00020079800B200370070C0B300E45A020015
:1021000000000000AE003700715780002E009000E4
:10211000810F500013003200715780002E00900094
:102120000080500080007800F00F200000806000E8
:10213000000F9800F06E2800885602000000000092
:102140000E0890002059020000000000E06F2800F7
:102150008856020000000000715780002107980097
:102160009700370070C0B300E45A0200000000007E
:102170009300370010002000600F98000000EB0073
:102180001007980071578000E09E2000808040007A
:102190000040EB0080487800705780008000E80025
:1021A000F00F200000806000705788007257800098
:1021B0002207980000702800B456020000000000BA
:1021C0007F0037004E0090000000E80040079800B4
:1021D0004E009000F40F500079003A006E5C02004F
:1021E000000000000000EB0040079800740037007A
:1021F000705780008000E800F00F200080806000B1
:1022000080578000808F50006A0032006E48900036
:10221000FF4F500067003600EE489000E0C7B30063
:1022200080CF500063003E00715780002E00900068
:10223000808F500015003A006E489000E45A02006A
:1022400000000000715780006E499000E09E200061
:102250000080400002487800705780008000E8004D
:10226000F00F2000008060007057880071578000D8
:10227000E09E2000808040000040EB008048780015
:1022800073578000230798004D0037007157800076
:102290002E0090000080500080007800F00F200099
:1022A00000806000000F9800F06E28008856020041
:1022B000000000000E0890002059020000000000FD
:1022C000E06F280088560200000000007057800070
:1022D000600798001D0037006E0090000001E800C4
:1022E000EE009000E09E20000080400090407800CA
:1022F000E09E20000000410001487800EE009000C0
:10230000E09E200000804000104078000004E000C3
:1023100009003200EE009000E09E200000804000A6
:1023200010407800E45A02000000000010702800FD
:1023300088560200000000006E0090008000E90056
:10234000F00F200000806000600798006E01900090
:102350002E0090008000E900F00F20000080600057
:10236000800F5100DCFF3A006E489000E45A0200F2
:1023700000000000AE0090006E499000E09E20003A
:1023800000804000024878002E0090008000E800A5
:10239000F00F200000806000200798007057800038
:1023A0008000E800F00F2000008060007057880077
:1023B0000300370070C0B300E45A020000000000C0
:1023C0006E0890000000E000CBFB320070578000E8
:1023D000400F980080578000300F98000000EB00FD
:1023E000600F98000000EB00500F98000000EB0019
:1023F00090578800D14080000020200000806000BD
:102400000000E000110532007835020000000000F5
:1024100051002000305A20002485020000000000F6
:1024200010002000500F98000805370081578000E9
:10243000E09E20000080400010407800604F98002F
:102440006E4890000080FB006101B90022179800DF
:1024500033179800E0072000010020002E119000A3
:10246000BE119000800F5100818F5900CB043E00B7
:102470002E109000BE10900000600100C9043700CB
:10248000C6043700C5043700C4043700C30437004E
:10249000C2043700C1043700C0043700BF0437004E
:1024A000BE043700BF043700BC043700BB0437004C
:1024B000BC043700B9043700B8043700B70437004C
:1024C000B6043700B5043700B4043700B30437004E
:1024D000B2043700B1043700B0043700AF0437004E
:1024E000AE043700AD043700AC043700AB0437004E
:1024F000AA043700A9043700A8043700A90437004C
:1025000086043700C60237002B013700340137003C
:10251000DD013700CB013700A00437009F023700F0
:102520009E0437009D0437009E0437009D04370049
:10253000320437004B043700160437003F033700DE
:102540003E0337003D0337003C0337003B033700B1
:102550003A033700390337003803370037033700B1
:10256000360337008D0437008C043700E60137004E
:10257000C9003700890437003F00370046013700A3
:10258000380137008504370065003700AA0137009D
:102590008204370081043700800437007F0437004D
:1025A0007E0437007D0437007C0437006700370065
:1025B0007A04370079043700780437008F00370039
:1025C0007604370075043700C40137007304370000
:1025D0007204370071043700450137006F0437007B
:1025E0006E0437006D043700F0023700F603370041
:1025F000000337002A0437000D0437006704370052
:102600000B013700270037003A0037007C01370004
:1026100062043700290037002B0037005F043700C1
:10262000180037005D0437005C04370054003700A1
:102630001A003700590437001C0037005D003700CE
:102640005604370079033700A001370053043700E0
:102650005204370017003700570137004F04370086
:102660004E0437004D043700D9023700A50037006B
:10267000E9023700C30037003A850200000000007D
:1026800048043700B7070700A04080000000E000C2
:102690004404320037080700420437006C06070084
:1026A000400437006E0907003E0437004809070060
:1026B0003C043700BC0807003A043700A46302005A
:1026C0000000000037043700A04080000000E00058
:1026D00005003A00D1012000305D20002485020071
:1026E000000000002F0437000C6202000000000010
:1026F0002C043700A09C2000104078000000A100AE
:102700000010A100A19C20008048780061012000F9
:10271000805A2000248502000000000021043700B8
:10272000A09C2000104078000000A0000010A10034
:10273000A19C20008048780051012000E05B20002F
:10274000248502000000000016043700A09C200031
:10275000104078000030A000A19C20008048780044
:10276000C1012000B07E20009A8402000000000019
:1027700000702800B4560200000000000904370071
:10278000A09C2000104078000030A100A19C2000F7
:1027900080487800B1012000007D20009A8402006A
:1027A0000000000000702800B45602000000000085
:1027B000FC033700A04080000000E00005003A0064
:1027C000D1012000305D20002485020000000000BF
:1027D000F4033700CB62A900C962A90051012000AF
:1027E000005F20009A8402000000000000702800B2
:1027F000B456020000000000EA033700A040800049
:102800000000E00005003A00D1012000305D20000A
:102810002485020000000000E2033700A09C200095
:1028200010407800704060000004E00004003A00AE
:102830002102200050E82000248502000000000052
:10284000C962A800CB62A9004101200050602000AD
:102850009A8402000000000000702800B4560200B4
:102860000000000021E3A800B0C0B300F280020025
:102870000000000080007800F0042000808F5000ED
:1028800003003E0060702800B45602000000000003
:1028900021E3A900C3033700805780008000E800CF
:1028A000F00F20000080600080578800D8050700E6
:1028B000F0030700600798006E0090008259020044
:1028C00000000000907228008856020000000000FE
:1028D0006E00900020590200000000009072280055
:1028E00088560200000000006E009000E8560200CA
:1028F0000000000000702800B45602000000000034
:10290000A8033700805780008000E800F00F200007
:102910000080600080578800BD050700D5030700D0
:10292000600798006E0090000080FB00B2820200F9
:1029300000000000600798006E00900082590200BD
:10294000000000009072280088560200000000007D
:102950006E009000205902000000000090722800D4
:1029600088560200000000006E009000E856020049
:102970000000000000702800B456020000000000B3
:1029800088033700A04080000000E00005003A0006
:1029900011C0B30010C0B300C87D020000000000E9
:1029A00080033700A10120009061200024850200EF
:1029B000000000007B03370051002000306320003E
:1029C000248502000000000023C2BF0061406000B7
:1029D0000004E000FCFF32000000FE00710337003D
:1029E000CA850200000000000000E0006D03320014
:1029F000A100200080632000248502000000000068
:102A0000400620005082020000000000A880020062
:102A10000000000023C2BF00614060000004E0002D
:102A2000FCFF320081BF2A00014001005D03370036
:102A3000350507000000E800000F9800020037008D
:102A4000E2640200000000000E0890000000E900AF
:102A5000000F98000E0890000000E000F8FF3A0018
:102A600050033700280507000000E800000F980019
:102A700002003700C0640200000000000E08900051
:102A80000000E900000F98000E0890000000E00030
:102A9000F8FF3A00430337001B0507000000E80079
:102AA000000F98000B003700610120002064200017
:102AB0009A8402000000000004650200000000008B
:102AC000725602000000000000702800B456020098
:102AD000000000000E0890000000E900000F9800C0
:102AE0000E0890000000E000EFFF3A002D033700D1
:102AF000A04080000000E00005003A00D101200065
:102B0000305D20002485020000000000250337000E
:102B1000C002A900C202A80021E3A80020002000F2
:102B20005082020000000000A0C0B300F28002004A
:102B30000000000080007800001B2000808F500003
:102B40000F00360090C0B300F280020000000000C9
:102B500080007800702B2000808F50000800360025
:102B600011012000806520009A840200000000000E
:102B700000702800B4560200000000000C0037006E
:102B8000C002A900C202A900D0722800B4560200F7
:102B90000000000021012000906620009A840200BD
:102BA0000000000000702800B45602000000000081
:102BB00021E3A900FB023700A04080000000E000F4
:102BC00005003A00D1012000305D2000248502007C
:102BD00000000000F3023700C002A900C202A900F1
:102BE00021012000906620009A840200000000006D
:102BF00000702800B456020000000000E90237000F
:102C0000F1002000A03920009A840200000000009A
:102C10000C8102000000000011002000903A20000A
:102C20009A8402000000000000702800B4560200E0
:102C300000000000DB0237001E81020000000000DF
:102C4000D8023700B0040700000F98006100200090
:102C5000706820009A840200000000000E089000B6
:102C6000C25802000000000021002000D0682000AF
:102C700024850200000000000E0890007C82020003
:102C800000000000C70237009F040700000F9800F3
:102C900061002000706820009A840200000000009B
:102CA0000E089000C2580200000000002100200021
:102CB00090EC200024850200000000000E08900027
:102CC0005082020000000000B6023700D0408000B1
:102CD0000090A000D0408800B2023700A0408000E1
:102CE0000000E00005003A00D1012000305D200026
:102CF0002485020000000000AA02370038650200A7
:102D000000000000A7023700100020009057880044
:102D100010002000600798001000370081578000E5
:102D20006E00900080804000F00F200080806000E6
:102D3000E09E20000080400090407800E0C3B30097
:102D400080CF500002003A000000EB00905788004E
:102D50006E0090000000E800600798008157800036
:102D60006E00900080804000F00F200080806000A6
:102D7000E09E200000804000104078000004E00049
:102D8000E6FF3A00EE00900020022000808F500005
:102D900002003400100020009057880090578000F7
:102DA0000000E0007F023A00805780008000E800C9
:102DB000F00F20000080600080578800AD020700FF
:102DC0006007980081578000F00F2000808060002D
:102DD000E09E20000080400090407800D0C3B30007
:102DE00080CF500040003A006E0090000000E000EC
:102DF0003A0034006E009000E50F500037003C00B0
:102E0000805780008000E800F00F20000080600004
:102E1000805788006E0090000000E900600798006D
:102E20000000EB00000F98000B0037006E009000D0
:102E30008E0890004500DD008100400040AF20007A
:102E4000808040000040EB00804878000E08900031
:102E50000000E800000F98000E089000FF0F5000DF
:102E6000F2FF34000000EB00000F98001300370061
:102E7000EE0190000E0A900081578000E09E200035
:102E800000804000104178004518DD0084004000BB
:102E900040AF200000804000024878000E089000FB
:102EA0000000E800000F9800805780008000E800D4
:102EB000F00F20000080600080578800815780005C
:102EC000E09E20000080400090407800E0C3B30006
:102ED00080CF5000E6FF3A00320237001000200099
:102EE000905788002F0237006E0090000000E0002D
:102EF0001B003A000000EB00000F980014003700A0
:102F00000E0890000040E800205902000000000078
:102F1000D074280088560200000000000E089000BF
:102F20004500DD008000780040AF200000804000B8
:102F3000885602000000000010752800B4560200F8
:102F4000000000000E0890000000E800000F98004C
:102F50000E089000E40F5000E9FF34001102370022
:102F60006E0090000000E000090034006E00900048
:102F7000E50F500006003C0000702800B456020027
:102F800000000000EE009000A15C88000502370000
:102F90001000200090578800020237008057800000
:102FA0008000E800F00F200000806000805788005B
:102FB00030020700200F9800150407008157800099
:102FC000F00F200080806000E09E20000080400024
:102FD0009040780090C2B30080CF50000D003A00BE
:102FE000A1408000E00220000088B900FC00400001
:102FF0000083200000804000900078002E089000A0
:103000000100010000702800B4560200000000001A
:10301000E40137001000200090578800E1013700DC
:1030200010002000905788001000200060079800D2
:1030300010003700815780006E00900080804000B3
:10304000F00F200080806000E09E200000804000A3
:103050009040780020C2B30080CF500002003A00B8
:103060000000EB00905788006E0090000000E80020
:1030700060079800815780006E00900080804000BB
:10308000F00F200080806000E09E20000080400063
:10309000104078000004E000E6FF3A0090578000FE
:1030A0000000E000BF013A0071002000F06820003D
:1030B0009A8402000000000020C2B300E45A02001B
:1030C000000000002200370081578000F00F200030
:1030D000008060008057880081578000E09E2000BB
:1030E0000080400010407800E45A02000000000018
:1030F00081578000E09E2000008040001040780052
:103100000000FB00200F9800A09C200010407800D9
:10311000684060000004E000040032002E089000C7
:10312000B282020000000000200F9800A140800041
:10313000E00220000088B900E80040000083200081
:1031400000804000900078002E08900001000100EF
:10315000805780000000E800805788008157800079
:10316000F00F200080806000E09E20000080400082
:103170009040780020C2B30080CF5000D2FF3A00C8
:1031800080578000F10F2000010060008057880008
:1031900020C2B300E45A02000000000000702800C2
:1031A000B4560200000000007E013700A1408000FC
:1031B000E00220000088B900800078000083200031
:1031C0000080400010007800000001007501370009
:1031D000A1408000E00220000088B9008080E80063
:1031E00000832000008040001000780000000100F3
:1031F0006C013700A1408000E00220000088B90087
:10320000E4004000008320000080400010007800AF
:103210000000010063013700A1408000E0022000AF
:103220000088B900E60040000083200000804000D4
:1032300010007800000001005A01370071002000E2
:10324000F06820009A840200000000008901070055
:10325000200F9800805780000000E9008057880008
:1032600081578000F00F20000080600080578800A8
:10327000250307000000E800000F98004503070041
:10328000300798003E0090000000E0005D00320032
:103290003E00900080407800909B2000014878001C
:1032A0003E009000E80F500006003400A09C200073
:1032B000104078000050A000A19C200080487800B9
:1032C00050003700A09C2000104078000050A10062
:1032D000A19C2000804878004A0037002E0890000A
:1032E000AA81020000000000A09C2000104078008D
:1032F0000042B2000004E00004003A00909B20006D
:1033000010407800E84F500009003A00A09C2000CF
:10331000104078000042B2000004E0000B003200D0
:10332000909B200010407800F04F500007003200C2
:10333000B0C3B300E45A020000000000909B2000DC
:10334000104078002059020000000000A09C2000DE
:1033500010407800684060000004E0000400320083
:103360002E089000B282020000000000200F98009A
:10337000A1408000E00220000088B900E800400081
:103380000083200000804000900078002E0890000C
:1033900001000100100F980000C2B300E45A0200BF
:1033A00000000000A09C2000104078000044B20003
:1033B0000004E0001300320061002000606920007A
:1033C0009A84020000000000A09C200010407800B9
:1033D000684060000004E000040032001E08900015
:1033E000B282020000000000100F98001E0890003A
:1033F000AA8102000000000000C2B300E45A0200EB
:10340000000000000E0890000000E900000F980086
:103410000E0890000000E000B0FF3A0000702800A5
:10342000B456020000000000DE00370061002000FA
:10343000606920009A84020000000000B2020700C8
:103440000000E800000F9800D20207003007980043
:103450003E0090000000E000440032003E0090007A
:1034600080407800909B2000014878003E0090004A
:10347000E80F500006003400A09C200010407800A7
:103480000050A000A19C2000804878003700370041
:10349000A09C2000104078000050A100A19C2000BA
:1034A0008048780031003700A1408000E002200011
:1034B0000088B900EA00400000832000008040003E
:1034C0001000780000000100100F9800A09C200060
:1034D00010407800684060000004E0000400320002
:1034E0001E089000B282020000000000100F980039
:1034F0001E089000AA81020000000000A09C20008D
:10350000104078000042B2000004E00004003A00DD
:10351000909B200010407800E84F500009003A00CE
:10352000A09C2000104078000042B2000004E0009F
:103530000B003200909B200010407800F04F5000AC
:1035400007003200B0C3B300E45A020000000000DC
:10355000909B2000104078002059020000000000DD
:1035600000C2B300E45A0200000000000E08900000
:103570000000E900000F98000E0890000000E00035
:10358000C9FF3A0000702800B45602000000000095
:103590008400370081002000C069200024850200DB
:1035A00000000000A1408000E00220000088B90077
:1035B000EC004000008320000080400010007800F4
:1035C000000001007700370081002000406A2000E1
:1035D0002485020000000000A1408000E0022000DD
:1035E0000088B900EE004000008320000080400009
:1035F00010007800000001006A003700E1002000A0
:10360000C06A20002485020000000000A140800064
:10361000E00220000088B900F00040000083200094
:103620000080400010007800000001005D003700BD
:10363000E1002000A06B20002485020000000000B3
:10364000A1408000E00220000088B900F2004000A4
:10365000008320000080400010007800000001007E
:1036600050003700C1002000B06720009A8402009B
:1036700000000000A1408000E00220000088B900A6
:10368000F40040000083200000804000100078001B
:1036900000000100725602000000000041003700E7
:1036A00019020700000F9800D1002000806D200053
:1036B0009A840200000000000E089000AA81020017
:1036C000000000000E0890000000E800000F9800C5
:1036D00008003700A1408000E00220000088B90007
:1036E000F6004000008320000080400010007800B9
:1036F000000001000E0890000000E900000F980093
:103700000E0890000000E000F2FF3A000070280070
:10371000B45602000000000022003700FA01070042
:103720000000E800000F9800A1002000506E20006B
:103730009A840200000000000D003700A1408000C4
:10374000E00220000088B900F8004000008320005B
:103750000080400010007800000001007256020056
:103760000000000000C2B300E45A020000000000A4
:103770000E0890000000E900000F98000E0890006D
:103780000000E000EDFF3A0001012000806C200005
:103790002485020000000000020037001000200015
:1037A00090578800805780008000E800F00F2000CC
:1037B0000080600080578800905780000000E00083
:1037C0001C00320051012000F06E20009A8402009B
:1037D00000000000BE08900080578000808F5000DD
:1037E0000700310080578000804078003E0890003C
:1037F00000C0500020590200000000000600370001
:1038000080578000804078003E08900000C0500043
:1038100020590200000000000000EB0090578800D3
:1038200010002000500F980000702800B4560200CD
:10383000000000008157800070578000808F50008A
:1038400002003A0010002000500F98005E0890001F
:103850000000E000F5FA32004E0890008057880022
:103860004E089000705788000000EB00600F980031
:103870008BF637000600FA000000EB0010079800F6
:103880000000EB00000F7800815780001E009000C0
:1038900080804000F00F200080806000E09E2000CB
:1038A000008040009040780000C3B30080CF5000FB
:1038B00043003400815780001E009000808040004B
:1038C000F00F200080806000E09E2000008040001B
:1038D0009040780090C3B30080CF500038003C0087
:1038E000815780001E00900080804000F00F200073
:1038F00080806000E09E2000008040001040780042
:103900008000FB0000FD2F00008F40001E00900093
:103910000000E80010079800120037001E00780031
:103920006A00B900000F7800815780001E009000E7
:1039300080804000F00F200080806000E09E20002A
:1039400000804000104078000000FB009E00400016
:1039500000FD2F00008F40001E0090000000E800D6
:1039600010079800815780001E0090008080400062
:10397000F00F200080806000E09E2000008040006A
:1039800090407800F0C2B30080CF50005101340065
:10399000815780001E00900080804000F00F2000C2
:1039A00080806000E09E2000008040009040780011
:1039B00090C3B30080CF5000D8FF340045013700DA
:1039C000815780001E00900080804000F00F200092
:1039D00080806000E09E20000080400090407800E1
:1039E00000C3B30080CF500035013A001E009000A4
:1039F0000000E80010079800815780001E0090002A
:103A000080804000F00F200080806000E09E200059
:103A1000008040009040780020C6B30080CF500066
:103A20000B003200815780001E0090008080400013
:103A3000F00F200080806000E09E200000804000A9
:103A40009040780020C4B30080CF50002D003A0091
:103A50001E0090000000E8001007980012003700D8
:103A60001E00780000004000000F780081578000A1
:103A70001E00900080804000F00F200080806000D9
:103A8000E09E200000804000104078000000FB0015
:103A90009E00400000FD2F00008F40001E0090009F
:103AA0000000E80010079800815780001E00900079
:103AB00080804000F00F200080806000E09E2000A9
:103AC000008040009040780010C3B30080CF5000C9
:103AD000E3FF3200815780001E009000808040008C
:103AE000F00F200080806000E09E200000804000F9
:103AF0009040780000C3B30080CF5000D8FF320060
:103B0000F4003700815780001E0090008080400044
:103B1000F00F200080806000E09E200000804000C8
:103B20009040780080C7B30080CF50000B00320077
:103B3000815780001E00900080804000F00F200020
:103B400080806000E09E200000804000904078006F
:103B500080C5B30080CF50008E003A001E00900058
:103B60000000E80010079800470037001E007800AA
:103B70004400DD00000F7800815780001E00900097
:103B800080804000F00F200080806000E09E2000D8
:103B90000080400090407800F0C2B30080CF500019
:103BA00018003400815780001E0090008080400083
:103BB000F00F200080806000E09E20000080400028
:103BC0009040780090C3B30080CF50000D003C00BF
:103BD000815780001E00900080804000F00F200080
:103BE00080806000E09E200000804000104078004F
:103BF0000000FB009E00400000FD2F00008F4000F1
:103C00001E003700815780001E0090008080400019
:103C1000F00F200000816000815780001E0090009E
:103C200080804000F00F200080806000E09E200037
:103C3000008040009040780000C2B30080C0700057
:103C4000E09E20000000410001487800815780007C
:103C50001E00900080804000F00F200080806000F7
:103C6000E09E200000804000104078000000FB0033
:103C70009E00400090FA2F00008F40001E00900030
:103C80000000E80010079800815780001E00900097
:103C900080804000F00F200080806000E09E2000C7
:103CA0000080400090407800F0C2B30080CF500008
:103CB0000B003400815780001E009000808040007F
:103CC000F00F200080806000E09E20000080400017
:103CD0009040780090C3B30080CF5000A3FF340021
:103CE000815780001E00900080804000F00F20006F
:103CF00080806000E09E20000080400090407800BE
:103D000000C4B30080CF50000B0034008157800006
:103D10001E00900080804000F00F20008080600036
:103D2000E09E2000008040009040780060C4B30016
:103D300080CF50008DFF3400815780001E0090001E
:103D400080804000F00F200080806000E09E200016
:103D5000008040009040780000C6B30080CF500043
:103D60005C003400815780001E009000808040007D
:103D7000F00F200080806000E09E20000080400066
:103D80009040780060C6B30080CF500077FF3400C9
:103D900050003700815780001E0090008080400056
:103DA000F00F200080806000E09E20000080400036
:103DB00090407800F0C2B30080CF5000450034003E
:103DC000815780001E00900080804000F00F20008E
:103DD00080806000E09E20000080400090407800DD
:103DE00090C3B30080CF50003A003C008157800060
:103DF0001E00900080804000F00F20008080600056
:103E0000E09E200000804000104078008000FB0011
:103E100000FD2F00008F4000120037001E007800C8
:103E20006A00B900000F7800815780001E009000E2
:103E300080804000F00F200080806000E09E200025
:103E400000804000104078000000FB009E00400011
:103E500000FD2F00008F40001E0090000000E800D1
:103E600010079800815780001E009000808040005D
:103E7000F00F200080806000E09E20000080400065
:103E800090407800F0C2B30080CF500011003400A1
:103E9000815780001E00900080804000F00F2000BD
:103EA00080806000E09E200000804000904078000C
:103EB00090C3B30080CF5000D8FF34000500370016
:103EC00010002000905788000000EB0020079800A9
:103ED0000A003700815780001E00900000804000DB
:103EE0008057880081578000F00F2000008060001C
:103EF000805788001E007800200798002E00900050
:103F00000080FA00000006000400FA0080578000DC
:103F10008000E800F00F200080806000E09E20001C
:103F20000080400090407800A0C3B30080CF5000D4
:103F300013003A00805780000080E8008057880016
:103F400081578000F00F20000080600080578800BB
:103F500048FE0700000F7800805780000000E9004D
:103F60008057880081578000F00F2000008060009B
:103F7000805788001E007800100798000200370064
:103F800010002000100798001E0090000080FA002A
:103F9000000006000400FA00805780008000E8005E
:103FA000F00F200080806000E09E20000080400034
:103FB00090407800B0C3B30080CF50000F003A00AB
:103FC000805780008080E800F00F200000806000B3
:103FD0008057880027FE0700000F78008057800078
:103FE0008000E900F00F200000806000805788000A
:103FF0001E00780010079800020037000000EB0058
:10400000100798001E0090000080FA0000000600D3
:104010000000FA0005003700805780008000E800AB
:10402000F00F2000008060008057880081578000DA
:10403000E09E2000008040009040780000C2B30065
:1040400080CF5000F4FF32000080FA00000006002C
:104050000400FA000000EB00000F78008057800099
:104060008000E800F00F200000806000805788008A
:10407000E7FF0700FFFD0700000F78001E00E000CB
:104080004D003A000000EB001007980013003700C5
:104090001E0090000040E8002059020000000000CF
:1040A0003075280088560200000000009E00900035
:1040B000E00220000088B9006102200080804000FA
:1040C0000083200000804000B45602000000000081
:1040D0001E0090000000E800100798001E009000ED
:1040E000E50F5000EAFF340071012000407020000D
:1040F00024850200000000000000EB0090578800BB
:104100001300200062002000110020001000200099
:1041100055000700000FE900E0FF2F009E0F100080
:10412000030032000080EB009E0F100005003A00F3
:10413000E1002000B0712000248502000000000092
:1041400042003700A1408000E00220000088B90052
:104150000102200080804000008320000080400099
:104160001000780000000100A8800200000000009C
:104170001E007800A0408800A1408000E0022000DE
:104180000088B900FE00400000832000008040004D
:1041900010007800000001001E00E0000100320065
:1041A000C222A80051002000305A200024850200BD
:1041B00000000000250037001E0FE900500020001D
:1041C0009E0F10001D003C00A1408000E002200076
:1041D0000088B90001022000808040000083200098
:1041E000008040001000780000000100A88002005C
:1041F000000000001E007800A0408800A140800060
:10420000E00220000088B900FE004000008320008A
:104210000080400010007800000001001E00E00057
:1042200001003200C222A80051002000305A2000B4
:104230002485020000000000040037005101200026
:10424000907220002485020000000000705780005A
:104250008000E900F00F2000008060008057880097
:104260000080FA00000006001E00FA00100F9800FF
:10427000210F9800320F9800430F98000000EB00C8
:10428000400798000000EB00200798000000EB00BA
:10429000100798000000EB00000F78006075280000
:1042A00088560200000000001E08900020590200FD
:1042B00000000000A07528008856020000000000E1
:1042C00067003700D25A020000000000204F98001B
:1042D0002E4890000000FB00600F98006E089000D0
:1042E000ED0F500029003200EE089000ED8F5000D5
:1042F00007003C006E099000E80F51000D003200ED
:104300006E089000EA0F50002000320035003700A0
:10431000D0022000EE089000808F50001E00320076
:10432000800720006E099000800F510027003200A6
:104330002C0037004E0090000000E0000700320023
:104340004E0090000000E90040079800706E2800C1
:104350008856020000000000410037001E00E00007
:10436000060032000000EB00000F7800706E28009D
:1043700088560200000000003900370070C0B3000A
:10438000E45A020000000000350037001000200051
:1043900020079800320037004E0090000000E00037
:1043A00006003A00D0C2B300E45A02000000000048
:1043B00010002000000F78002900370070C0B30003
:1043C000E45A020000000000250037004E0890006B
:1043D0000000E000030032000080EB00500F980066
:1043E0005D003700AE489000F0C2B30080CF5000AF
:1043F00018003400AE48900090C3B30080CF500046
:1044000014003C004E009000E30F50000600340002
:1044100070C0B300E45A0200000000004000200019
:10442000400798000E0037002E489000E45A020022
:1044300000000000CE0090006B0047002E49900065
:10444000827078004E0090000000E800400798005D
:104450000300370070C0B300E45A020000000000FF
:104460002E0090000000E00096FF3200007028004F
:10447000B4560200000000004E0090000000E00072
:1044800003003A001E089000500F980032003700D9
:104490000000EB00100798004E0090000000E900BB
:1044A00040079800CE0090003107980011003700B7
:1044B0001E0090006A00B90010079800BE0090002E
:1044C0004E009000808050006B00470061407800F3
:1044D0008000FB001E0090008080400000FD2F0047
:1044E00000804000100798004E0090000000E90096
:1044F000400798004E0090000000E000ECFF3D00F7
:104500009E0090002E089000808F50000D00350016
:104510009E0090003E089000808F500009003C00F3
:104520001E00E000040032001E0090000000EA00BF
:10453000500F9800080037001E019000520F98009D
:1045400005003700B1012000E0EA200024850200C8
:104550000000000049FF37005E0890000080FA006C
:10456000000006000400FA00E075280088560200EA
:1045700000000000A081200010407800E45A0200F2
:104580000000000000702800B45602000000000087
:10459000C07628008856020000000000B0C5B300B5
:1045A000E45A0200000000000000EB00000F780059
:1045B0000F0037001E00E0000300320000C2B3000D
:1045C000E45A0200000000009E007800E002200093
:1045D0000088B90061022000808040000083200034
:1045E0000080400088560200000000001E0FE80016
:1045F000500020009E0F1000EEFF3600D0C5B30023
:10460000E45A020000000000D10020007080200069
:104610009A84020000000000A1BF2A000000EB0005
:104620003E5C020000000000000F78001E007800D1
:104630004800DE002059020000000000E0C2B30084
:10464000E45A0200000000001E0078002059020019
:104650000000000000702800B456020000000000B6
:1046600061002000007620009A8402000000000013
:10467000B0408000DA590200000000007100200004
:1046800070EA20009A84020000000000C040800010
:10469000DA59020000000000207828008856020045
:1046A00000000000C1408000110798002004230092
:1046B0009E009000808F50001600320020042300DE
:1046C0009E009000808F500005003E0030002300C7
:1046D0009E009000808F50000A00320019003700C1
:1046E000300423009E009000808F50000D003200A7
:1046F000600423009E009000808F50000D00320067
:1047000010003700107928008856020000000000D1
:104710000F00370040792800885602000000000092
:104720000B00370070792800885602000000000056
:1047300007003700A079280088560200000000001A
:1047400003003700D07928008856020000000000DE
:10475000107A2800B456020000000000E101200099
:104760006076200024850200000000000080FA002E
:10477000000006000000FA005100200020922000F6
:104780009A84020000000000C1BF2A000000EB0074
:104790003E5C020000000000DA5902000000000048
:1047A00061002000709220009A8402000000000046
:1047B000E1BF2A000000EB003E5C020000000000A8
:1047C000DA5902000000000000702800B456020010
:1047D00000000000C1002000407820002485020075
:1047E0000000000070000700C2C2BF00614060000E
:1047F0000004E00005003200110120008065200067
:104800009A8402000000000004003700210120000B
:10481000906620009A84020000000000C0C2B3002D
:10482000E45A02000000000000C2B300E45A020093
:1048300000000000CBC2BF00684060000004E00040
:104840000500320041012000506020009A840200DF
:10485000000000000400370051012000005F20002C
:104860009A84020000000000C0C2B300E45A0200B3
:104870000000000000C2B300E45A02000000000083
:10488000A09C200010407800704060000004E00010
:10489000050032002102200000792000248502005A
:1048A0000000000004003700E1012000207B200010
:1048B0002485020000000000A09C20001040780029
:1048C000684060000004E00005003A00B1012000EB
:1048D000007D20009A8402000000000004003700E0
:1048E000C1012000B07E20009A8402000000000078
:1048F000C0C2B300E45A02000000000000C2B300CE
:10490000E45A020000000000B1012000C020210094
:104910009A84020000000000909B20001040780064
:10492000205902000000000000702800B456020068
:1049300000000000A09C2000104078006340600050
:10494000E14F500005003A0051012000E05B2000DB
:1049500024850200000000000400370061012000EF
:10496000805A20002485020000000000A140800041
:10497000E00220000088B900410220008080400051
:10498000008320000080400010007800000001003B
:10499000C1002000407820002485020000000000B3
:1049A0000080FA00000006000000FA00A1002000CC
:1049B000A005210024850200000000006104200001
:1049C000200B21002485020000000000A10120002E
:1049D000400621009A84020000000000A1408000EF
:1049E000E00220000088B900210220008080400001
:1049F00000832000008040001000780000000100CB
:104A0000A1002000E00721009A84020000000000BD
:104A10000040200050000700001020004E0007005A
:104A2000002020004C000700000420004A0007007E
:104A3000000820004800070000702800B45602005B
:104A40000000000041002000800F21009A84020035
:104A50000000000021E3A800A0C0B300F280020023
:104A600000000000245A0200000000001100200095
:104A7000903A20009A8402000000000090C0B30029
:104A8000E45A02000000000090C0B300F28002006F
:104A900000000000245A0200000000001100200065
:104AA000903A20009A8402000000000090C0B300F9
:104AB000E45A020000000000C0C0B300F28002000F
:104AC00000000000245A0200000000001100200035
:104AD000903A20009A8402000000000090C0B300C9
:104AE000E45A020000000000B0C0B300F2800200EF
:104AF00000000000245A0200000000001100200005
:104B0000903A20009A8402000000000090C0B30098
:104B1000E45A02000000000021E3A9000040200048
:104B20001C000700001020001A00070000202000D1
:104B300018000700000420001600070000082000ED
:104B40001400070000702800B456020000000000A6
:104B50000080FA00000006000200FA00000F780052
:104B6000401680001E0060000000E00004003200DB
:104B7000307A280088560200000000000300370049
:104B8000607A280088560200000000000080FA00C9
:104B9000000006000200FA00000F780050168000A6
:104BA0001E0060000000E00004003200907A28003F
:104BB000885602000000000003003700C07A280079
:104BC00088560200000000000080FA000000060085
:104BD0000200FA00805780008000E800F00F2000FB
:104BE000008060008057880009FD070021FB070056
:104BF000000F78001E00E000060034004000200096
:104C00009E0F100003003C001E00E9009040880049
:104C10000D0037000000EB009057880021022000B3
:104C20004081200024850200000000008001EB008C
:104C30004200200011002000100020008AFD070023
:104C40000000E900904088002101200060832000DE
:104C500024850200000000000080FA000000060029
:104C60000200FA00805780008000E800F00F20006A
:104C70000080600080578800E5FC0700FDFA07000F
:104C8000104798001E4090000004E0000900320028
:104C90001E409000EA4F500006003E001E4090006B
:104CA0000040E90080407800008120000148780041
:104CB0000F0037000000EB0090578800D10820005B
:104CC0003087200024850200000000008001EB00F6
:104CD000A2002000110020009000200062FD0700CB
:104CE0000040E90080407800008120000148780001
:104CF0000081200010407800E94F500010003A0079
:104D0000C3FC0700DBFA0700004F78001E04E00038
:104D10000B003A000000EB0090578800F07A280062
:104D2000B4560200000000008001EB00F2FF2700F3
:104D30008000EB00200220004BFD0700004F7800B0
:104D400041012000009020002485020000000000A6
:104D500011012000B01F2100248502000000000086
:104D600023C2BF00614060000004E000FCFF32008D
:104D70000081200010407800E94F500003003A0005
:104D80001E407800025B0200000000007C810200EF
:104D90000000000000003700C65A020000000000BA
:104DA0000004E000FCFF3200D25A020000000000C4
:104DB0008040780000C2B30080CF50000100320074
:104DC000F5FF37000080FA00000006000000FA003E
:104DD0005161800020C32000008040009040780096
:104DE00030C8B30080CF50000E003A005061800000
:104DF0000000E80050618800030037005061800027
:104E00000000E800506188005161800020C320004C
:104E1000008040009040780000CEB30080CF50006A
:104E2000F6FF36000080FA00000006000A00FA00D3
:104E3000300798000000EB0020079800AE009000BB
:104E400020C32000008040009040780000CEB300D6
:104E500080CF500003003E000080EB004007980028
:104E600023003700AE00900020C3200000804000E7
:104E7000104078008080FB0000F22F00008040008E
:104E8000100798002E0090008000E80020C320004A
:104E900000804000104078000080FB004801DD00E9
:104EA0002E0090008080E80020C320000080400099
:104EB000104078000080FB00000F41009E00780049
:104EC0003E009000808F500003003A002E009000BA
:104ED00040079800060037009E0090002E009000CA
:104EE000008040006300400020079800D3FF370097
:104EF0004E0090000080FA00000006000600FA0054
:104F0000881F78000000EB00000F780051618000DE
:104F100020C32000008040009040780080C2B30091
:104F200080CF500010003A00506180000000E8007F
:104F30005061880030010700000F78005161800047
:104F400020C32000008040009040780090C2B30051
:104F500080CF5000BD003A00506180000000E800A2
:104F600050618800B90037005161800020C32000E3
:104F7000008040009040780000C4B30080CF500013
:104F8000160036005161800020C3200000804000E0
:104F900090407800A0C5B30080CF50000F003E00C5
:104FA0005261800020C320000000410010407800C2
:104FB0008080FB00F0FB2F0000804000800040005C
:104FC000A0BC20000080400010007800200798005E
:104FD0000200E800506188009E00370051618000A7
:104FE00020C32000008040009040780000C8B3003B
:104FF00080CF5000870036005161800020C3200020
:1050000000804000104078000080FB0010079800EE
:105010000100E80050618800700920009E009000A7
:10502000808F50004A003200700920009E009000DE
:10503000808F50000D003C00400920009E00900031
:10504000808F50001F003200600920009E009000F9
:10505000808F500034003200300920009E00900004
:10506000808F50002100320059003700A009200035
:105070009E009000808F50003F003200A009200069
:105080009E009000808F500005003C0080092000A9
:105090009E009000808F5000460032004C00370088
:1050A000B00920009E009000808F50003700320031
:1050B000D00920009E009000808F50001600320022
:1050C00043003700A1408000E00220000088B900C2
:1050D000EA004000008320000080400010007800BB
:1050E00000000100000F780058003700A140800048
:1050F000E00220000088B900E800400000832000A2
:1051000000804000100478008C00070008000100B7
:10511000000F78004D003700046502000000000019
:10512000000F780049003700A1408000E002200015
:105130000088B900F4004000008320000080400097
:105140001000780000000100000F78003F003700D9
:10515000A1408000E00220000088B900F800400073
:105160000083200000804000100078000000010053
:10517000000F780035003700C2C2BF0061406000F8
:105180000080FB00000F780030003700CBC2BF006A
:105190000080FB004300DE00614060000081FB00F6
:1051A000020078000080EA008180EA00000F7800A9
:1051B0002600370021E3A800C0C0B300F28002003F
:1051C00000000000000F780021E3A9001F00370055
:1051D0000000EB00000F78001C0037001E00780074
:1051E0006A00B900000F78005161800020C32000E0
:1051F00000804000104078000080FB009E004000CE
:1052000000FD2F00008F4000506180000000E8008A
:10521000506188005161800020C320000080400060
:1052200090407800F0C2B30080CF500007003600F5
:105230005161800020C32000008040009040780031
:1052400090C3B30080CF5000E4FF36001E0078000A
:10525000200798002E0090004F0478000080FA008C
:10526000000006000600FA0024FF0700000F780087
:10527000000037005161800020C320000080400002
:1052800090407800A0C2B30080CF50000A003200E6
:105290005161800020C320000080400090407800D1
:1052A000F0C2B30080CF5000030032001E0078002F
:1052B000200798001E0037005161800020C32000A5
:1052C00000804000104078000080FB00100798002C
:1052D0000100E80050618800A00220009E009000BC
:1052E000808F500005003200F00220009E009000E8
:1052F000808F500007003200DEFF3700FFFE0700FE
:10530000800078001E0078000180B900000F78004E
:10531000D8FF3700F9FE0700000178001E00780072
:10532000110009000200D800000F7800D1FF3700FB
:105330002E0090000080FA00000006000600FA002F
:10534000C8FF0700000F780000003700516180009F
:1053500020C320000080400090407800D0C2B300FD
:1053600080CF50000A0032005161800020C320002D
:105370000080400090407800B0C2B30080CF500061
:10538000030032001E007800200798001700370045
:105390005161800020C32000008040001040780050
:1053A0000080FB00100798000100E80050618800B1
:1053B000B00220009E009000808F50000800320054
:1053C000D00220009E009000808F5000010032002B
:1053D000DEFF3700A3FF07001E0F1000DBFF3700C2
:1053E000A0FF07001E0F4000D8FF37002E009000DE
:1053F0000080FA00000006000C00FA0052618000F4
:1054000020C3200000004100104078008080FB0095
:10541000F0FB2F000080400080004000A0BC200076
:105420000080400090007800210798000200E8000A
:10543000506188000000EB00000F78000B0037007F
:105440009E0178005261800020C3200000004100CE
:105450001040780080407800660047008171780035
:105460000200E800506188001E0FE80051618000D2
:1054700020C32000008040009040780000C4B300AA
:1054800080CF5000070036005161800020C320000B
:105490000080400090407800A0C5B30080CF50004D
:1054A0000E0036005161800020C3200000804000C3
:1054B00090407800F0C2B30080CF5000E0FF36008B
:1054C0005161800020C3200000804000904078009F
:1054D00090C3B30080CF5000D9FF3E0097FF070074
:1054E0001007980066004700104078000000FB009D
:1054F00050079800C0032000DE009000808F50000D
:1055000032003200C0032000DE009000808F500087
:1055100005003C0010022000DE009000808F50004B
:10552000410032004E003700D0032000DE00900022
:10553000808F500005003200E0032000DE00900064
:10554000808F50000A003200450037000000EB0059
:1055500040079800AE0090001E009000808F500021
:1055600041003A0011002000410798003E0037003A
:105570006600470090409000D0C3B30080CF500039
:1055800009003A000000EB0040079800AE009000D0
:105590001E009000808F5000330035001100200065
:1055A00041079800300037000000EB0040079800EA
:1055B000AE0090001E009000808F50002A00340042
:1055C00011002000410798002700370066004700BF
:1055D00090409000D0C3B30080CF500009003A0043
:1055E0000000EB0040079800AE0090001E00900005
:1055F000808F50001C003C001100200041079800E3
:10560000190037000000EB0040079800AE00900042
:105610001E009000808F500013003D0011002000FC
:105620004107980010003700660047009040900046
:10563000D0C3B30080CF500009003A000000EB0057
:1056400040079800AE0090001E009000808F500030
:1056500005003200110020004107980002003700C9
:105660000000EB00400798004E0090000080FA0018
:10567000000006001C00FA00881F78000000EB0004
:10568000506188000000EB00300798000000EB003C
:10569000200798000000EB00100798000000EB00C6
:1056A000606188000000EB00706188000000EB0082
:1056B000806188000000EB0050079800D040800017
:1056C0000080A000D04088000000EB004007980058
:1056D000090037004E00900080004000A0BC200070
:1056E000808040000000EB00800878004E009000B1
:1056F0000000E800400798004E009000F90F5000AD
:10570000F4FF3400340437001E0090000000E00075
:1057100021003A005161800020C320000080400039
:1057200090407800F0CDB30080CF500003003E00E1
:1057300020002000300798002A04370051618000C3
:1057400020C3200000804000104078008080FB00D3
:1057500000F22F0000804000600798005061800038
:105760008000E80020C32000008040001040780046
:105770000080FB004801DD00506180008080E8006F
:1057800020C3200000804000104078000080FB0013
:1057900000007100500798000000EB00100798000F
:1057A00050618000E300400020C3200000804000E2
:1057B000104078000080FB006101B90000F82F0064
:1057C000F1FF2F000201400083814800420F980042
:1057D000530F980010022000010020004E09900095
:1057E000DE099000800F5100818F5900EE033E00CA
:1057F0004E089000DE089000006001002100370094
:1058000035003700E8033700E70337007100370041
:1058100081003700A3003700B7003700BE00370013
:105820003B01370088013700DF033700EE01370006
:105830003502370099023700AF0237009F02370068
:10584000CB023700BB023700D8023700D60337003F
:10585000780337005C033700D3033700D2033700E7
:1058600000033700F00237009F033700AD03370015
:10587000DE0237001203370032033700B50337006A
:10588000C6033700100020002007980050618000F8
:105890006600400050618800506180008080E9000F
:1058A00020C3200000804000104078008080FB0072
:1058B000F0FB2F0000844000A0FE070000017800EC
:1058C00088004400A0BC200000804000020878004E
:1058D0003EFD0700B60337001000200020079800A7
:1058E000506180006400400050618800C2FE0700E3
:1058F0000000E0001C00320051618000310F980070
:1059000020C320003E099000000041009040780034
:105910008041EB004357980020C8B30080CF50006F
:1059200002003A0010C0B30040579800BE08900033
:105930000100E800506188004E5190000204E00030
:105940009B03320010002000100798005061800077
:10595000630050005061880095033700506180005B
:105960000000E800506188005161800020C32000E1
:10597000008040009040780030C8B30080CF5000D5
:10598000070032005161800020C3200000804000E9
:105990009040780000CEB30080CF5000EFFF36007B
:1059A0005161800020C320000080400090407800BA
:1059B00030C8B30080CF50007D033A0010002000B3
:1059C00010079800506180000080E9005061880055
:1059D00077033700100020002007980050618000F6
:1059E000640040005061880054FE07000FFD07006E
:1059F000000F78008081EB009E8F110003003200C1
:105A00001E007800506188006903370060002000A4
:105A10003007980066033700100020002007980028
:105A20005061800064004000506188007061800017
:105A3000E90F500018003C00726180005161800045
:105A40006E009000008040008001E900820041006B
:105A5000E0BF2000008040000308780070618000F3
:105A60000000E8007061880034FE0700EFFC0700CA
:105A7000000F78008080EB009E8F10000300320042
:105A80001E01780052618800490337006000200041
:105A90003007980046033700700020003007980058
:105AA00043033700407E28008856020000000000B3
:105AB0001000200020079800706180000000E000C6
:105AC0000A003200706180000000E9007061880007
:105AD0007061800080004000E0BF20000080400036
:105AE00010007800506188003103370080002000EA
:105AF000300798002E033700100020002007980080
:105B0000516180006E009000008040006300400002
:105B100050618800260337001000200020079800FD
:105B200050618000640040005061880057003700D9
:105B30005161800020C32000008040009040780028
:105B400020C2B30080CF50001F003A005061800097
:105B50000000E8005061880010003700D04080004D
:105B60000080A100D04088005161800020C3200047
:105B70000080400010407800004178000100E800FB
:105B80005061880002407800E45A020000000000E2
:105B9000D04080000080A000D0408800516180008B
:105BA00020C32000008040009040780020C2B30055
:105BB00080CF5000E9FF3A00506180000000E8000B
:105BC00050618800310037005161800020C32000FF
:105BD000008040009040780000C4B30080CF5000A7
:105BE000070036005161800020C320000080400083
:105BF00090407800A0C5B30080CF50000D00360063
:105C00005161800020C320000080400010407800D7
:105C10000004E00013003D005161800020C320001B
:105C20000080400090407800F0CDB30080CF50005D
:105C30000C003E00C1FD0700000F7800D04080003E
:105C40000080A100D04088001E007800C2580200E9
:105C500000000000D04080000080A000D0408800FC
:105C60000A0037005161800020C3200000804000FE
:105C700090407800B0C3B30080CF500003003A00DA
:105C8000506180000000E800506188005161800090
:105C900020C320000080400090407800F0CDB30089
:105CA00080CF500007003E005161800020C32000DB
:105CB000008040009040780030C8B30080CF500092
:105CC0009BFF3A00506180008000E90020C3200063
:105CD0000080400090407800B0C3B30080CF5000F7
:105CE00009003200D04080000080A100D040880030
:105CF000A0872800B456020000000000D0408000B9
:105D00000080A000D040880030FC0700A8023700C7
:105D10001000200020079800D04080000080A100E3
:105D2000D0408800506180006400400050618800CD
:105D30005161800020C32000008040009040780026
:105D400020C2B30080CF500018003A00506180009C
:105D50000000E800506188000A00370051618000AF
:105D600020C32000008040001040780000417800EF
:105D70000100E8005061880002407800E45A020007
:105D8000000000005161800020C32000008040001E
:105D90009040780020C2B30080CF5000EFFF3A005F
:105DA000506180000000E80050618800516180006F
:105DB00020C320000080400090407800C0C2B300A3
:105DC00080CF500004003A00506180000000E800DD
:105DD0005061880002003700300020003007980032
:105DE0005161800020C320000080400010407800F6
:105DF0008080FB00F0FB2F00008440008001EB005E
:105E0000F2FF27008000EB000000EB0034210200CD
:105E1000000000000001780088004400A0BC2000C1
:105E20000080400002087800506180000000E80017
:105E300050618800E5FB0700D04080000080A00092
:105E4000D04088005A023700100020002007980038
:105E500050618000640040005061880060618000F3
:105E6000E30F500004003C00606180000000E80087
:105E70006061880002003700400020003007980071
:105E8000626180005361800020C3200000804100D7
:105E9000104078008080FB0000FC2F000082400052
:105EA0006610B9008080E80020C12000008040001A
:105EB000040878000300E800506188005161800008
:105EC00020C320000080400090407800D0C3B30081
:105ED00080CF500011003A00506180000000E800BF
:105EE00050618800606180006600B9008080E80031
:105EF00020C1200000804000100078000004E9006C
:105F00000EFD07000001780088004400A0BC2000BE
:105F100000804000020878000200370030002000B6
:105F20003007980053618000130F980020C32000B1
:105F30009E08900000804000904078000041EB00F7
:105F400002579800B0C8B30080CF500002003A005A
:105F500013C0B300035798009E0890000100E800AA
:105F6000506188000E5190000204E00009003200E8
:105F700068618000F1FC0700000178006640B9000C
:105F8000E400400020C120000080400002087800AA
:105F90000200370030002000300798005161800077
:105FA00020C320000080400090407800F0CDB30076
:105FB00080CF500008003600606180005261800090
:105FC0006600B9008000780020C1200000804000F9
:105FD00002087800020037003000200030079800E7
:105FE0007AFB0700F201370010002000200798001C
:105FF0005061800064004000506188005261800060
:1060000020C3200000004100104078008080FB0089
:1060100000FC2F00008F40000200E8005061880063
:1060200050002000300798000000EB004007980067
:106030002F0037004E0090006600B9008080E80015
:1060400020C1200000804000100078009E0F50000A
:1060500024003A001E00E90080004000A0BC20009F
:1060600000804000100178004E0090006600B900EA
:10607000E400400020C120000080400010007800B3
:10608000800F510012003D009E00E9000181400098
:10609000A0BC200000004100100078000001E800D2
:1060A00081804000A0BC20000080400002087800F1
:1060B0004E0090006600B9008000780020C12000EA
:1060C0000080400010007800506188000300370015
:1060D000606180000000E900606188000000EB0062
:1060E000300798004E0090000000E800400798003C
:1060F000616180004E009000810F5000CDFF3400A0
:1061000032FB0700AA01370010002000200798008A
:106110005061800064004000506188008061800010
:106120000000E00027003A000000EB004007980064
:106130000A003700CE00900020C3200000804000FD
:10614000104078008080FB004E009000808040006E
:1061500030F22F0000804000400798004E00900071
:10616000E300400020C32000008040009040780001
:10617000E0C8B30080CF500006003200CE0090008F
:1061800020C3200000804000104078000004E000A0
:10619000E8FF3A00CE00900020C3200000804000BD
:1061A000104078000004E000040032004E0090002F
:1061B00064004000806188000200370090002000E9
:1061C0003007980053618000030F780080618000E1
:1061D000506188009E00780020C3200000804000AD
:1061E000104078008080FB00F0FB2F00008440000E
:1061F00042FB07000001780088004400A0BC20009A
:1062000000804000020878005061800080618800B2
:106210001E00E800506188008161800020C32000DA
:106220000080400090407800C0C2B30080CF500092
:1062300003003A00806180000000E800806188006F
:106240008161800020C320000080400090407800E1
:1062500000CEB30080CF50000E0036008061800079
:10626000E300400020C32000008040009040780000
:10627000E0C8B30080CF5000030032000000EB0004
:106280008061880003003700806180006400400066
:1062900080618800CDFA070045013700100020001A
:1062A00020079800516180006E009000008040003F
:1062B00063004000506188003D013700100020005D
:1062C0002007980050618000640040005061880001
:1062D000A1408000E00220000088B9008000780022
:1062E00000832000008040001000780000000100C2
:1062F000B6FA07002E013700100020002007980092
:10630000506180006400400050618800A14080001E
:10631000E00220000088B9008080E80000832000AF
:10632000008040001000780000000100A7FA07007C
:106330001F013700100020002007980050618000E6
:106340006400400050618800A1408000E00220000D
:106350000088B900E4004000008320000080400075
:10636000100078000000010098FA070010013700C3
:106370001000200020079800506180006400400059
:1063800050618800A1408000E00220000088B90030
:10639000E6004000008320000080400010007800EC
:1063A0000000010089FA07000101370010002000F9
:1063B0002007980050618000640040005061880010
:1063C000A1408000E00220000088B900E800400001
:1063D000008320000080400010047800D7FB0700F5
:1063E0000800010079FA0700F100370010002000D2
:1063F00020079800506180006400400050618800D0
:10640000CEFB07000000E00003003200C064020081
:106410000000000002003700E264020000000000FB
:106420006AFA0700E20037001000200020079800F9
:10643000506180006400400050618800BFFB07008D
:106440000000E00003003200C002A900C202A80060
:1064500002003700C002A900C202A9005BFA0700CF
:10646000D300370010002000200798005061800002
:106470006400400050618800B0FB07000000E000AD
:1064800007003200A09C2000104078000000A0000F
:106490000010A100A19C2000804878000600370071
:1064A000A09C2000104078000000A0000010A10077
:1064B000A19C20008048780044FA0700BC00370007
:1064C0001000200020079800506180006400400008
:1064D0005061880099FB0700504F8800504F8000A2
:1064E0000000E00002003D000000EB00504F88007B
:1064F000514F800000FA2000808F500002003400CD
:1065000000FA2000504F8800604F8000E10F5000DB
:1065100002003C0020002000604F8800614F800096
:1065200030062000808F500002003400300620002A
:10653000604F88006A6102000000000023FA070033
:106540009B00370010002000200798005061800059
:10655000640040005061880078FB0700604F8800AD
:10656000504F80000000E00002003D000000EB0002
:10657000504F8800514F800000FA2000808F50005B
:106580000200340000FA2000504F8800604F800065
:10659000E10F500002003C0020002000604F880006
:1065A000614F800030062000808F500002003400D0
:1065B00030062000604F88006A6102000000000081
:1065C00002FA07007A003700100020002007980028
:1065D00050618000640040005061880057FB070054
:1065E0000000E00009003200A1408000E00220002D
:1065F0000088B900F00040000083200000804000C7
:10660000100078000000010008003700A140800061
:10661000E00220000088B900F20040000083200062
:10662000008040001000780000000100E7F907003A
:106630005F003700100020002007980050618000A4
:1066400064004000506188003CFB07007007980020
:106650007E009000E10F500010003200FE0090001C
:10666000E28F5000160032007E0190000200E00030
:10667000010032001A003700A1408000E002200033
:106680000088B900EE004000008320000080400038
:10669000100078000000010011003700A1408000C8
:1066A000E00220000088B900EC00400000832000D8
:1066B0000080400010007800000001000800370052
:1066C000A1408000E00220000088B900F6004000F0
:1066D00000832000008040001000780000000100CE
:1066E000BAF9070032003700100020002007980098
:1066F0005061800064004000506188000FFB07007B
:106700000000E00003003200C962A800CB62A900CB
:1067100002003700CB62A900C962A900ABF90700EB
:1067200023003700100020002007980050618000EF
:10673000640040005061880000FB0700000F7800F3
:106740001E00780050820200000000009FF9070040
:1067500017003700100020002007980050618000CB
:106760006400400050618800F4FA0700000F7800D0
:10677000A1408000E00220000088B900FC00400039
:106780000083200000804000900078001E00780008
:10679000010001008DF907000500370010002000FE
:1067A00030079800020037003000200030079800C2
:1067B0002E0090000000E00005003A0051618000CA
:1067C0006E0090000080400063004000506188002F
:1067D0000000EB00200798003E0090000000E00061
:1067E000C9FB3200D04080000080A100D04088006A
:1067F0003E009000E10F50001800320061002000C0
:10680000A03A20009A840200000000003E009000A0
:10681000C25802000000000081002000003B200060
:106820009A840200000000005E009000C25802003E
:1068300000000000B1002000803B20009A8402008C
:106840000000000050618000C258020000000000FB
:10685000A0872800B4560200000000004F04780012
:106860000080FA00000006000200FA00000F780025
:1068700000C2B300E45A0200000000001E007800CD
:10688000885602000000000000C2B300E45A020073
:10689000000000000080FA00000006000400FA007A
:1068A0000000EB00506188003F003700516180001C
:1068B00020C32000008040009040780021479800CD
:1068C0002E4090000004E000040035002E409000AF
:1068D000E45A02000000000030003700AE40900093
:1068E00000CEB30080CF50001C003600A0872800E7
:1068F000B456020000000000506180008000E800F3
:1069000020C3200000804000104078000080FB0081
:106910004801DD00506180008080E80020C3200035
:1069200000804000104078000080FB000000410023
:10693000000F7800506180000080E80050618800FE
:106940001E007800C25802000000000000C2B30020
:10695000E45A0200000000001000370000C2B3003B
:10696000E45A0200000000002E4090008080FB00EE
:1069700000F82F0000804000800040002097200099
:1069800000804000100078008856020000000000DF
:1069900000C2B300E45A0200000000005061800011
:1069A0000000E800506188005161800020C3200091
:1069B00000804000104078000004E000BBFF3A0077
:1069C000A0872800B456020000000000506180003B
:1069D0000000E900C2580200000000007100200021
:1069E000303C200024850200000000000080FA00F6
:1069F000000006000600FA0010079800805780008B
:106A0000000F7800150037001E009000104178003C
:106A100081578000E09E20000080400010407800F8
:106A2000804F5100050032001E007800805788001A
:106A30000000EB00200798000E0037008057800010
:106A40008000E800F00F2000008060008057880080
:106A50001E0090000000E800100798001E00900043
:106A6000104078000004E000E7FF3A00100020002A
:106A7000200798002E0090000080FA000000060019
:106A80000400FA000000EB00000F7800100037004F
:106A90001E00780080004000209720000080400009
:106AA00010007800D3FF07000000E000070032006C
:106AB0001E0078008040780000C8B30000C040008D
:106AC0000080FB0010079800060037001E0FE8004A
:106AD000100220009E0F1000EDFF34000000EB00BC
:106AE000100798001E0090000080FA0000000600C9
:106AF0003600FA0080578000000F98001F00370012
:106B00008E089000E09E20000080400090407800B9
:106B100000C6B30080CF5000110034008E089000F2
:106B2000E09E20000080400090407800A0C7B300A5
:106B300080CF50000A003C000E0990008E089000A3
:106B4000E09E20000080400090407800F0CDB3002F
:106B500080C06000E09E20000000410001487800F5
:106B60000E0890000000E800000F98008E089000CA
:106B7000F00F200000806000000F98008E08900049
:106B800070578000808F5000DDFF3A000000EB005E
:106B9000000F980081578000E09E20000080400098
:106BA00090407800F0C2B30080CF50002D01340037
:106BB00081578000E09E20000080400090407800D7
:106BC00090C3B30080CF500026013C000000EB00D2
:106BD000000F9800070037000E099000F2004700F0
:106BE0000040EB0000F178000E0890000000E80083
:106BF000000F98008E08900020022000808F500027
:106C0000F5FF34003A1C0200000000006007980005
:106C10006E0090004880DE008040780072004700DF
:106C2000114098006E0090008040780000C0EB009A
:106C300080C0600072004700214098006E00900004
:106C40007AF80700500798005E009000E10F4000BE
:106C50002B003200DE00900020C3200000804000A6
:106C6000104078008080FB0030F22F000080400050
:106C7000300798005E009000000F98000D0037006C
:106C80000E0990008E0890003E0090008080400029
:106C900020C32000008040009040780020C32000E6
:106CA00000004100014878000E0890000000E80054
:106CB000000F9800014020003E00900080805000AE
:106CC0000E089000808F5000EDFF3C000800370058
:106CD0008E08900020C32000808040000040EB0020
:106CE000804878000E0890000000E800000F98002F
:106CF0008E089000F03F2000808F5000F4FF340099
:106D000030002000000F98000000EB0020079800E2
:106D10000820020000000000430037002E00900011
:106D20000000E00002003A0008200200000000001D
:106D30002E0090000000E00004003A0050FF070021
:106D40000080FB0060079800020037000000EB00A5
:106D5000600798006E009000825902000000000059
:106D60006E0090000000E0000C0032000E09900060
:106D70006E0090008040780072004700017178003A
:106D8000EE00900070082000808F50001A003A003A
:106D9000100020002007980017003700815780005E
:106DA000E09E2000008040009040780020C2B300A8
:106DB00080CF500003003A002E0090000000A20097
:106DC000200798000E09900081578000E09E200067
:106DD000008040001040780080407800720047003A
:106DE00001717800805780008000E800F00F2000DB
:106DF00000806000805788000E0890000000E800C6
:106E0000000F98008E08900030022000808F500004
:106E10000500340091002000A03C200024850200E1
:106E200000000000D40037008157800070578000B8
:106E3000808F5000B9FF3A000E089000E30F500019
:106E4000CD0032000E089000E40F5000CA0032005E
:106E50000E08900080407800C0CDB30000C0400014
:106E60008040780072004700014878000000EB0085
:106E7000000F98000000EB00400798000000EB00B6
:106E800050079800460037008E08900020C320006D
:106E9000008040009040780000CEB30080CF5000CA
:106EA0002E0036008E08900020C320000080400095
:106EB000104078008080FB0000F22F00008040002E
:106EC000300798000E0890008000E80020C32000E2
:106ED00000804000104078000080FB004801DD0089
:106EE0000E0890008080E80020C320000080400051
:106EF000104078000080FB0000004100100798005F
:106F000072004700104090000080FB00C800DD00C8
:106F100072004700204090000080FB00008040008D
:106F2000000F78001E0090009E0F500005003100F9
:106F30008E0890003E0090000080400063004000FA
:106F400050079800BE0090000E089000008040009E
:106F500063004000000F9800020037000E08900008
:106F6000400798000E0890008000E80020C3200031
:106F700000804000104078000080FB004801DD00E8
:106F80000E0890008080E80020C3200000804000B0
:106F9000104078000080FB0000004100600798006E
:106FA0004E0090000000E000B7FF32007200470082
:106FB000104078008080FB0030F22F0000804000FD
:106FC000600798004E009000000F98000D003700F9
:106FD0008E0890006E009000008140008E089000A6
:106FE00020C32000008040009040780020C3200093
:106FF00000004100014878000E0890000000E90000
:10700000000F98008E0890005E009000808F500066
:10701000EFFF3D000000EB00000F98000C00370070
:10702000DE0090000E089000008140008E08900065
:1070300072004700E140780020C3200000004100BA
:10704000014878000E0890000000E800000F98004A
:107050008E0890006E009000808F5000F0FF350089
:1070600045003700B087280062FE07000000E000FE
:10707000050032007FF90700A0872800B4560200FF
:10708000000000003C003700F087280059FE070090
:107090000000E0000200320000FE0700360037006A
:1070A0004088280053FE07000000E0000400320082
:1070B000D04080000090A100D04088002E00370012
:1070C000908828004BFE07000000E00020003200FE
:1070D0000000EB00000F9800180037000000EB00E4
:1070E000700798000F0037008E0890007E00900017
:1070F0008080400020C320000080400010407800C5
:107100000080FB00825902000000000000C2B300B2
:10711000E45A0200000000007E0090000000E80039
:10712000700798007E009000EF0F5000EEFF3400D3
:107130000E08900070004000000F98008E0890002C
:10714000F03F2000808F5000E4FF34000A00370039
:10715000F088280027FE07000000E000020032004F
:107160000700070004003700C1002000303D200068
:1071700024850200000000000080FA0000000600E4
:107180000200FA000000EB00000F78000600370054
:107190009E00780020C32000808040000040EB006B
:1071A000804878001E0FE800F03F20009E0F10007E
:1071B000F7FF340011CEB30020C32000014878004F
:1071C00080C0EB0030C320000148780080C0EB0095
:1071D00040C320000148780011CAB30050C320000A
:1071E000014878000080FA0000000600575249006C
:1071F00054452000424954003A2020002A6E650080
:1072000078742000636C6F00636B2000285E290097
:10721000207769006C6C200075736500207468002D
:107220006973200076616C00756531005749520022
:10723000452072006F757400696E65007320280028
:10724000432920003230300030204D00696368004F
:1072500061656C0020506500617263006520470025
:107260004E55200047504C004E6F2000646576005C
:10727000696365002C2074007279200028414C005D
:1072800041524D00292053004541520043482000FF
:107290006D616300726F2000666972007374410053
:1072A0004444520045535300204D410043524F0087
:1072B000202030002E4D610063726F00206D65004C
:1072C0006E754D00616372006F2020002020200049
:1072D00031574900524520006164640072657300B3
:1072E000730D0A00202020002A3157004952450022
:1072F00020524F004D2043004F4D4D00414E440061
:10730000204D410043524F00733A0D000A203500D2
:10731000312E52004541440020524F004D2028009C
:1073200030783300332920002A666F007220730002
:10733000696E67006C6520006465760069636500AE
:1073400020627500730D0A00203835002E4D410073
:107350005443480020524F004D202800307835001B
:10736000352920002A666F006C6C6F007765640019
:107370002062790020363400626974002061640064
:107380006472650073730D000A20320030342E00E1
:10739000534B4900502052004F4D200028307800B8
:1073A00043432900202A66006F6C6C006F776500EC
:1073B00064206200792063006F6D6D00616E64006F
:1073C0000D0A2000323336002E414C0041524D0050
:1073D00020534500415243004820280030784500A2
:1073E00043290D000A20320034302E00534541005D
:1073F0005243480020524F004D202800307846006C
:10740000302941004C4152004D205300454152006B
:107410004348200028307800454329005345410067
:107420005243480020283000784630002944650047
:10743000766963006520490044732000617265002D
:107440002061760061696C0061626C0065206200F9
:1074500079204D00414352004F2C20007365650098
:1074600020283000292E52004541440020524F0070
:107470004D2028003078330033293A00204D410058
:107480005443480020524F004D20280030783500EA
:10749000352953004B49500020524F004D20280001
:1074A00030784300432955006E6B6E006F776E0095
:1074B000206D610063726F002C20740072792000CF
:1074C0003F206F007220280030292000666F720074
:1074D000206865006C7042005553200052455300EF
:1074E00045542000576172006E696E00673A2000B3
:1074F0002A5368006F727400206F7200206E6F0054
:10750000207075006C6C2D00757020002A4E6F0085
:107510002064650076696300652064006574650019
:1075200063746500642044005331380053323000E6
:10753000204869006768200050726500732044008D
:107540006967200054686500726D4400533138004B
:1075500042323000205072006F6720005265730085
:107560002044690067205400686572006D44530030
:107570003138320032204500636F6E0020446900CC
:1075800067205400686572006D4453003234300047
:1075900034204500636F6E0072616D0020746900D5
:1075A0006D65200043686900704453003234330035
:1075B000312031004B204500455052004F4D5500C1
:1075C0006E6B6E006F776E002064650076696300F5
:1075D000655057004D20640069736100626C65005E
:1075E00064314B00487A2D00342C300030304B0091
:1075F000487A200050574D0046726500717565004D
:107600006E63790020696E00204B48007A2050009C
:107610007265730063616C00653A500052323A0043
:10762000447574007920630079636C0065206900FB
:107630006E202500205057004D20610063746900C2
:107640007665450052524F00523A200050574D0087
:107650002061630074697600652C20006720740047
:107660006F20640069736100626C650041555800C9
:107670002046720065717500656E6300793A2000DE
:107680004155580020494E00505554002F4849009C
:107690002D5A41005558200048494700484155009F
:1076A00058204C004F5756004F4C54004D45540045
:1076B000455220004D4F440045564F004C54410068
:1076C0004745200050524F0042453A0020564500A1
:1076D00072726F007228290020406C00696E65008C
:1076E0003A20400070676D007370610063653A0076
:1076F00020627900746573002E546F006F206C0057
:107700006F6E6700215379006E7461007820650008
:1077100072726F00724E6F002045450050524F004C
:107720004D457200617369006E6764006F6E65009D
:1077300053617600696E670020746F0020736C00DF
:107740006F742000496E7600616C690064207300DC
:107750006C6F74004C6F610064696E006720660096
:10776000726F6D0020736C006F74200045525200E0
:107770004F523A0020636F006D6D61006E6420000F
:1077800068617300206E6F002065660066656300A7
:10779000742068006572650041434B004E41430010
:1077A0004B493200432053005441520054204200C0
:1077B000495449003243200053544F0050204200A6
:1077C00049544900324320006D6F6400653A0D0052
:1077D0000A2031002E2053006F667400776172001A
:1077E000650D0A0020322E00204861007264770087
:1077F00061726500536574002073700065656400F4
:107800003A0D0A0020312E00207E35004B487A00C8
:107810000D0A2000322E20007E3530004B487A00C1
:107820000D0A2000332E20007E313000304B4800FE
:107830007A0D0A0020342E00207E340030304B00B8
:10784000487A570041524E00494E47003A204800BE
:107850004152440057415200452049003243200024
:107860006973200062726F006B656E00206F6E009E
:1078700020746800697320005049430021202800CB
:10788000524556002041330029536500742073008F
:1078900070656500643A0D000A2031002E20310029
:1078A00030304B00487A0D000A2032002E20340080
:1078B00030304B00487A0D000A2033002E20310072
:1078C0004D487A004932430020286D006F64200043
:1078D00073706400293D2800202030002E4D610087
:1078E00063726F00206D65006E750D000A20310017
:1078F0002E37620069742000616464007265730051
:10790000732073006561720063680D000A20320005
:107910002E493200432073006E696600666572006E
:107920005365610072636800696E67002049320028
:1079300043206100646472006573730020737000FB
:10794000616365002E2046006F756E006420640040
:107950006576690063657300206174003A536E00B8
:107960006966660065722800424153004943290058
:1079700052656100647961002F412F00402063004F
:107980006F6E7400726F6C007320410055582000B8
:1079900070696E00612F41002F402000636F6E0000
:1079A00074726F006C7320004353200070696E0086
:1079B000436F6D006D616E0064206E006F74200077
:1079C00075736500642069006E2074006869730037
:1079D000206D6F0064655000756C6C002D75700033
:1079E0002072650073697300746F720073204F001A
:1079F00046465000756C6C002D7570002072650055
:107A000073697300746F720073204F004E536500EA
:107A10006C662D0074657300742069006E20480048
:107A2000695A20006D6F640065206F006E6C7900EC
:107A300052455300455442004F4F54004C4F4100B3
:107A4000444552004155580020494E0050555400BD
:107A50002F4849002D5A2C002052450041443A003D
:107A600020506F00776572002073750070706C0095
:107A700069657300204F4E00506F770065722000DB
:107A800073757000706C6900657320004F46460086
:107A9000444154004120530054415400453A2000D1
:107AA00044454C0041592000757357005249540019
:107AB000453A200052454100443A2000434C4F00D3
:107AC000434B2C00203143004C4F43004B2C2000F3
:107AD00030444100544120004F555400505554004B
:107AE0002C2031004441540041204F005554500097
:107AF00055542C00203020002A7069006E20690047
:107B000073206E006F77200048695A00434C4F0085
:107B1000434B2000544943004B533A002052450048
:107B200041442000424954003A205300796E7400C9
:107B300061782000657272006F722000617420000D
:107B400063686100722078002E20650078697400F7
:107B50002877690074686F0075742000636861009D
:107B60006E676500296E6F00206D6F0064652000F0
:107B7000636861006E6765004E6F6E00657869002E
:107B8000737465006E74200070726F00746F630010
:107B90006F6C2100782E200065786900740D0A0052
:107BA000496E7600616C690064206300686F69004B
:107BB00063652C00207472007920610067616900A0
:107BC0006E444500564944003A68740074703A00A7
:107BD0002F2F6400616E670065726F00757370000F
:107BE000726F74006F747900706573002E636F009C
:107BF0006D2A2D002D2D2D002D2D2D002D2D2D002C
:107C00002A4F7000656E200064726100696E20006A
:107C10006F7574007075740073202800483D48002B
:107C2000692D5A002C204C003D474E0044294E003F
:107C30006F726D00616C20006F7574007075740058
:107C400073202800483D33002E3376002C204C0052
:107C50003D474E0044294D00534220007365740097
:107C60003A204D004F535400207369006720620092
:107C7000697420006669720073744C0053422000DE
:107C8000736574003A204C00454153005420730042
:107C9000696720006269740020666900727374006D
:107CA00020426F006F746C006F6164006572200089
:107CB000762031002E20480045580D000A20320061
:107CC0002E20440045430D000A2033002E204200A0
:107CD000494E0D000A2034002E2052004157440026
:107CE000697370006C61790020666F00726D6100CD
:107CF00074207300657456006F6C740061676500D2
:107D0000206D6F006E6974006F7273003A20350049
:107D1000563A2000207C2000332E3300563A2000B3
:107D2000207C2000565055004C4C5500503A200005
:107D30005365740020736500726961006C207000E7
:107D40006F72740020737000656564003A2028002B
:107D500062707300290D0A0020312E00203330009C
:107D6000300D0A0020322E002031320030300D005C
:107D70000A2033002E203200343030000D0A20005B
:107D8000342E200034383000300D0A0020352E000B
:107D90002039360030300D000A2036002E20310008
:107DA00039323000300D0A0020372E0020333800E1
:107DB000343030000D0A2000382E200035373600D0
:107DC00030300D000A2039002E20310031353200CC
:107DD00030300D000A3130002E2042005247200082
:107DE00072617700207661006C75650041646A00FD
:107DF0007573740020796F007572200074657200CD
:107E00006D696E00616C410072652000796F7500CC
:107E10002073750072653F002043460047313A00E9
:107E20002043460047323A00285C2D002F5F5C005B
:107E30002D2928005C5F2F002D295300656C6500FB
:107E4000637420006F75740070757400207479007D
:107E500070653A000D0A2000312E20004F70650039
:107E60006E206400726169006E202800483D480061
:107E7000692D5A002C204C003D474E0044290D002E
:107E80000A2032002E204E006F726D00616C2000BF
:107E900028483D00332E3300562C20004C3D47002F
:107EA0004E4429005232570020287300706420008D
:107EB00068697A00293D2800202030002E4D61009D
:107EC00063726F00206D65006E750D000A20310031
:107ED0002E4953004F37380031362D0033204100F2
:107EE00054520D000A2032002E4953004F373800FB
:107EF00031362D00332070006172730065206F00F1
:107F00006E6C790049534F002037380031362D0010
:107F1000332041005452200028524500534554005C
:107F2000206F6E0020435300290D0A005245530074
:107F30004554200048494700482C2000434C4F003E
:107F4000434B2000544943004B2C20005245530022
:107F5000455420004C4F570049534F0020373800FC
:107F600031362D003320720065706C0079202800B6
:107F7000757365007320630075727200656E74001E
:107F8000204C53004220730065747400696E6700D2
:107F9000293A200050726F00746F63006F6C3A00D2
:107FA00020736500726961006C332000776972008C
:107FB00065322000776972006552460055756E0083
:107FC0006B6E6F00776E52006561640020747900FB
:107FD00070653A0020746F0020656E006476610061
:107FE00072696100626C6500206C65006E677400E8
:107FF0006844610074612000756E690074733A0012
:10800000206E6F0020696E0064696300617469000E
:108010006F6E44006174610020756E006974200009
:108020006C656E00677468002028620069747300D4
:10803000293A200043532000454E4100424C450060
:108040004443530020444900534142004C454400FE
:1080500052335700202873007064200063736C0053
:10806000206869007A293D00282029000D0A440073
:10807000697363006F6E6E006563740020616E004B
:108080007920640065766900636573000D0A43001A
:108090006F6E6E00656374002028560070752000B6
:1080A000746F20002B355600292061006E6420007B
:1080B00028414400432074006F202B00332E3300EE
:1080C0005629430074726C00415558004D4F4400CE
:1080D00045204C0045445000554C4C005550200064
:1080E000485055004C4C5500502048005652450011
:1080F00047414400432061006E64200073757000A6
:10810000706C790035565600505533002E335600AA
:10811000414443004275730020686900676842006B
:108120007573200048692D005A2030004275730095
:10813000204869002D5A2000314D4F004445200051
:10814000616E640020565200454720004C454400B3
:1081500073207300686F75006C64200062652000F6
:108160006F6E2100466F75006E64200020657200FE
:10817000726F7200732E4D004F534900434C4B00F9
:108180004D4953004F435300204F4B0020464100C0
:10819000494C5300657420007370650065643A00B3
:1081A0000D0A2000312E200033304B00487A0D009C
:1081B0000A2032002E20310032354B00487A0D0063
:1081C0000A2033002E20320035304B00487A0D0053
:1081D0000A2034002E2031004D487A00436C6F0095
:1081E000636B2000706F6C006172690074793A00F3
:1081F0000D0A2000312E200049646C0065206C00BF
:108200006F7720002A646500666175006C740D004C
:108210000A2032002E204900646C65002068690045
:1082200067684F007574700075742000636C6F0090
:10823000636B200065646700653A0D000A20310019
:108240002E204900646C650020746F00206163007B
:1082500074697600650D0A0020322E00204163000B
:1082600074697600652074006F206900646C650095
:10827000202A640065666100756C7400496E7000A8
:108280007574200073616D00706C6500207068006B
:10829000617365003A0D0A0020312E00204D6900FF
:1082A00064646C0065202A006465660061756C007A
:1082B000740D0A0020322E0020456E0064535000D9
:1082C000492028007370640020636B0070207300E5
:1082D0006B652000736D7000206373006C20680074
:1082E000697A29003D28200020302E004D6163006E
:1082F000726F20006D656E00750D0A0020312E0032
:10830000536E690066662000435320006C6F77004F
:108310000D0A2000322E53006E696600662061004F
:108320006C6C20007472610066666900632D7000D9
:10833000202D6600202A42007974650073206400B5
:10834000726F7000706564002A464100494C450018
:10835000442C20004E4F2000444154004144610011
:108360007461200062697400732061006E642000F3
:1083700070617200697479003A0D0A0020312E0094
:1083800020382C00204E4F004E4520002A64650006
:10839000666175006C7420000D0A2000322E2000EA
:1083A000382C2000455645004E200D000A20330091
:1083B0002E2038002C204F00444420000D0A2000BD
:1083C000342E2000392C20004E4F4E0045537400AF
:1083D0006F70200062697400733A0D000A2031004A
:1083E0002E203100202A640065666100756C7400DF
:1083F0000D0A2000322E20003252650063656900AC
:1084000076652000706F6C006172690074793A00C3
:108410000D0A2000312E200049646C0065203100D7
:10842000202A640065666100756C74000D0A2000E6
:10843000322E200049646C00652030005541520006
:10844000542028007370640020627200672064006A
:1084500062702000736220007278700020686900EA
:108460007A293D0028202000302E4D0061637200E3
:108470006F206D00656E75000D0A2000312E5400CE
:1084800072616E007370610072656E00742062002C
:108490007269640067650D000A2032002E204C00CE
:1084A00069766500206D6F006E6974006F720D0053
:1084B0000A2033002E42720069646700652077004D
:1084C0006974680020666C006F772000636F6E002F
:1084D00074726F006C554100525420006272690042
:1084E000646765005265730065742000746F200036
:1084F000657869007452610077205500415254003C
:1085000020696E00707574005541520054204C0073
:10851000495645002044490053504C0041592C0015
:10852000207D2000544F200053544F00504C4900F0
:108530005645200044495300504C410059205300F7
:10854000544F500050454400574152004E494E0090
:10855000473A200070696E0073206E006F7420002F
:108560006F7065006E206400726169006E202800E3
:1085700048695A002920520045564900443A0D00E6
:108580000A496E0076616C006964200063686F00C0
:10859000696365002C2074007279200061676100B6
:1085A000696E6D0073525300204C4F00572C200011
:1085B000434F4D004D414E0044204D004F44450077
:1085C0005253200048494700482C200044415400A1
:1085D00041204D004F4445004164640072657300C2
:1085E00073206F0066205000434638003537340052
:1085F0003F546800697320006D6F6400652072004D
:108600006571750069726500732061006E206100FC
:1086100064617000746572004C43440020747900FA
:1086200070653A000D0A2000312E200048443400C5
:108630003437380030202800757369006E672000D9
:108640005043460038353700342049004F2065003C
:10865000787061006E64650072294C00434420000C
:1086600028747900702061006464720029203D0044
:108670002028200020302E004D616300726F200002
:108680006D656E00750D0A0020312E004C434400CC
:1086900020526500736574000D0A2000322E4900D7
:1086A0006E697400204C4300440D0A0020332E00F4
:1086B000436C6500617220004C4344000D0A2000A9
:1086C000342E4300757273006F722000706F730058
:1086D000697469006F6E200065783A0028342900BB
:1086E00020300D000A2036002E5772006974650094
:1086F00020746500737420006E756D0062657200F1
:1087000073206500783A28003629200038300D00A3
:108710000A2037002E5772006974650020746500C6
:108720007374200063686100726163007465720095
:1087300073206500783A280037292000383044003B
:10874000697370006C617900206C69006E6573005C
:108750003A0D0A0020312E00203120000D0A2000A1
:10876000322E20004D756C00746970006C654900F4
:108770004E495400434C450041524300555253006A
:108780004F522000534554004E6F200041434B0090
:108790002C206300686563006B20610064617000D9
:1087A00074657200434C4B00094D4F00534909005A
:1087B000435309004D4953004F5069006E737400D4
:1087C00061746500733A47004E440900332E33004C
:1087D000560935002E305600094144004309560021
:1087E00050550900415558000950090050095000E2
:1087F0000949090049092D00094F570044092D0076
:10880000092D2D000954780044092D0009527800E3
:10881000445343004C095300444109002D092D00E5
:10882000504743000950470044092D00092D3100ED
:108830002E28420052290900322E280052442900D5
:1088400009332E00284F5200290934002E285900E0
:1088500057290900352E2800474E290009362E00D9
:1088600028424C00290937002E28500055290900BC
:10887000382E28004752290009392E002857540065
:10888000290930002E2842006C6B2900474E440015
:1088900009474E004409410044430900352E300089
:1088A000560933002E335600095650005509410031
:1088B00055580900657865006375740065203A00B5
:1088C00020205400494D45004F55540020302E00C3
:1088D000204D610063726F00206D65006E750D00A4
:1088E0000A2031002E204C006976650020696E0058
:1088F00070757400206D6F006E6974006F724900AE
:108900006E70750074206D006F6E6900746F720078
:10891000202A73007461720074626900742065001B
:1089200072726F0072202A0070617200697479009F
:1089300020657200726F7200202A7300746F7000DD
:108940006269740020657200726F7200204E4F00E1
:108950004E452000554E4B004E4F57004E204500CF
:1089600052524F005220610075746F0072616E00A8
:10897000676520002B4D48007A292B006B487A0050
:108980002952610077207600616C750065206600D1
:108990006F7220004252470020284D004944490090
:1089A0003D3132003729570041524E00494E4700B1
:1089B0003A2050006F73730069626C00652062009A
:1089C0007566660065726F0076657200666C6F0092
:1089D00077416E0079206B0065792000746F20006C
:1089E00065786900745370006163650020746F00DE
:1089F00020636F006E7469006E7565004E756D00C2
:108A000062657200206F6600206269007473200046
:108A100072656100642F770072697400653A200006
:108A200043533A000D0A2000312E200043530D001D
:108A30000A2032002E202F00435320002A646500B4
:108A4000666175006C7450006F73690074696F0023
:108A50006E2069006E2064006567720065657300B2
:108A600053657200766F200061637400697665005B
:108A700047656E00657261006C090900090909000B
:108A800050726F00746F63006F6C2000696E740029
:108A900065726100637469006F6E2D002D2D2D00CD
:108AA0002D2D2D002D2D2D002D2D2D002D2D2D00AA
:108AB0002D2D2D002D2D2D002D2D2D002D2D2D009A
:108AC0002D2D2D002D2D2D002D2D2D002D2D2D008A
:108AD0002D2D2D002D2D2D002D2D2D002D2D2D007A
:108AE0002D2D2D002D2D2D002D2D2D002D2D2D006A
:108AF0002D2D2D002D2D2D002D2D2D002D2D3F0048
:108B0000095468006973200068656C0070090900E9
:108B10000928300029094C0069737400206375002E
:108B2000727265006E7420006D616300726F730075
:108B30003D582F007C580900436F6E007665720027
:108B400074732000582F720065766500727365009B
:108B5000205809000928780029094D006163720036
:108B60006F2078007E095300656C660074657300A1
:108B700074090900095B09005374610072742300D1
:108B8000095265007365740009090900095D09004F
:108B900053746F00702409004A756D0070207400D2
:108BA0006F2062006F6F74006C6F6100646572000B
:108BB00009097B0009537400617274002077690011
:108BC000746820007265610064262F002509440046
:108BD000656C610079203100207573002F6D730082
:108BE000090909007D095300746F7000612F41006D
:108BF0002F4009004155580050494E0020286C0074
:108C00006F772F0048492F00524541004429090041
:108C10000922610062632200095365006E6420002E
:108C200073747200696E67006209530065742000F6
:108C300062617500647261007465090009093100A0
:108C4000323363002F4309004155580020617300FF
:108C5000736967006E6D65006E7420002861750091
:108C6000782F43005329090009307800313233004E
:108C7000642F4400094D6500617375007265200022
:108C80004144430020286F006E6365002F434F006E
:108C90004E542E0029093000623131003009530052
:108CA000656E6400207661006C75650066094D0094
:108CB00065617300757265002066720065717500EC
:108CC000656E6300790909007209520065616400EC
:108CD000672F5300094765006E6572006174650077
:108CE000205057004D2F5300657276006F09090020
:108CF0002F0943004C4B20006869680009436F004E
:108D00006D6D61006E646800697374006F72790044
:108D1000090909005C0943004C4B20006C6F690095
:108D200009566500727369006F6E69006E666F00A8
:108D30002F7374006174750073696E00666F0900AB
:108D4000095E0900434C4B0020746900636B6C00A2
:108D50002F4C0900426974006F7264006572200034
:108D6000286D7300622F4C005342290009092D0021
:108D70000944410054206800696D0900436861009E
:108D80006E676500206D6F006465090009095F006A
:108D90000944410054206C006F6F09005365740052
:108DA000206F750074707500742074007970650010
:108DB000090909002E094400415420007265610030
:108DC00064702F0050095000756C6C0075702000A5
:108DD00072657300697374006F72730020286F00EE
:108DE00066662F004F4E2900092109004269740070
:108DF000207265006164730009536300726970003A
:108E0000742065006E6769006E65090009093A0003
:108E10000952650070656100742065002E672E00A0
:108E200020723A0031307600095368006F772000D5
:108E3000766F6C0074732F00737461007465730037
:108E400009093B000942690074732000746F200017
:108E500072656100642F7700726974006520650097
:108E60002E672E002030780035353B0032772F00FA
:108E70005709500053552000286F6600662F4F0099
:108E80004E290900093C78003E2F3C00783D200027
:108E90003E2F3C00303E090055736500726D610045
:108EA00063726F0020782F006173730069676E0032
:108EB00020782F006C697300742061006C6C0000D6
:108EC0000000FA00408D28008856020000000000D3
:108ED0000080FA00000006000000FA000040EB00ED
:108EE000606C0200000000000040EB00606C0200BB
:108EF000000000000040EB00606C02000000000079
:108F00000040EB00606C0200000000000000EB007D
:108F10009C6B0200000000000000EB009C6B020054
:108F2000000000000000EB009C6B0200000000004D
:108F30000080FA00000006000C00FA00A09C20004F
:108F4000104078000040A000A19C200080487800DC
:108F5000A09C2000104078000030A100A19C2000BF
:108F60008048780011C0B300809B20000148780041
:108F700081C0B300909B20000148780021C0B3005D
:108F8000F0BA20000148780080C0EB0020C0B30098
:108F90003C6A020000000000C922A900C902A90021
:108FA000C8E2A80010C0B300CC6C020000000000B2
:108FB000C3FF07000000370022C2BF00614060000D
:108FC0000004E000FCFF3200301180008040780097
:108FD00030BB20000148780030BB200010407800F2
:108FE0000080FB004400DE008040780020BB2000B1
:108FF0000148780020BB2000104078000080FB0072
:10900000300798003E009000E30F50001701320037
:10901000BE009000E38F50000A003C003E0190002B
:10902000E10F5100A5003200BE019000E18F510018
:10903000FB003C003E0090000000E0001200320007
:10904000E8023700BE009000E68F50009102320027
:109050003E019000E60F510004003C00BE0190006C
:10906000E48F510083023200DE0237003E009000A0
:10907000E80F50009E023200BE009000EA8F5000C0
:1090800034013200D702370030BB20001040780096
:109090000080FB006101B900420798005307980067
:1090A000D0002000010020004E019000DE01900061
:1090B000800F5100818F59007C003E004E009000CF
:1090C000DE00900000600100CA0237000C0037008B
:1090D0000D00370012003700170037001D00370061
:1090E0002300370044003700480037004C003700A9
:1090F00052003700580037005E0037006400370028
:109100006FFF0700ACFF3700CA6A020000000000D2
:1091100010C0B300E45A020000000000A6FF3700B0
:109120000A6B02000000000010C0B300E45A020005
:1091300000000000A0FF37000040EB00CC6C0200F4
:109140000000000010C0B300E45A0200000000005C
:1091500099FF370010C0B300CC6C02000000000083
:1091600010C0B300E45A02000000000092FF370074
:10917000F0BA200010407800E24F500006003A009C
:10918000F06B0200000000008040780010BB20005F
:109190000148780006003700F00F20002A6B02001B
:1091A000000000008040780010BB200001487800DB
:1091B000A09C200010407800684060000004E0009F
:1091C0000800320010BB2000104078000080FB0037
:1091D000B2820200000000008040780010BB200036
:1091E0000148780010BB200010407800E45A0200CB
:1091F0000000000070FF37003E6C0200000000001D
:10920000E45A0200000000006BFF3700DE6C020031
:1092100000000000E45A02000000000066FF370072
:1092200010C0B300826C02000000000010C0B30048
:10923000E45A0200000000005FFF37000040EB002E
:10924000BA6C02000000000010C0B300E45A020033
:109250000000000058FF370010C0B300BA6C0200D5
:109260000000000010C0B300E45A0200000000003B
:1092700051FF37000040EB00A86C02000000000026
:1092800010C0B300E45A0200000000004AFF37009B
:1092900010C0B300A86C02000000000010C0B300B2
:1092A000E45A02000000000043FF37000040EB00DA
:1092B000E45A0200000000003FFF370030BB2000EE
:1092C00090407800F0C0B30080C0600030BB200048
:1092D0000148780030BB2000104078008040E80052
:1092E00030BB20000148780010C0B300E45A0200EF
:1092F000000000008040EB0010BB20000148780017
:109300004000370022C2BF00614060000004E0005E
:10931000FCFF3200301180008040780000BB20004C
:1093200001487800A09C2000104078006840600050
:109330000004E0000800320000BB2000104078006C
:109340000080FB00B2820200000000008040780034
:1093500000BB200001487800F0BA200010407800DF
:10936000E24F500009003A0000BB20001040780096
:109370000080FB009C6B02000000000010C0B300E6
:10938000E45A0200000000001900370000BB200072
:10939000104078000080FB002A6B020000000000F3
:1093A0008040780000BB200001487800A09C20008D
:1093B00010407800684060000004E00008003200BF
:1093C00000BB2000104078000080FB00B282020049
:1093D000000000008040780000BB200001487800B9
:1093E00000BB200010407800E45A0200000000009A
:1093F00010BB2000104078008040E80010BB200027
:109400000148780010BB20009040780030BB20005D
:109410001040780080CF5000BAFF3900E6FE3700D8
:1094200030BB200090407800F0C0B30080C06000E6
:1094300030BB20000148780030BB2000104078008D
:109440008040E80030BB20000148780030BB20009D
:1094500010407800826C02000000000010C0B300D1
:10946000E45A020000000000D3FE370030BB2000A9
:1094700090407800F0C0B30080C0600030BB200096
:109480000148780030BB2000104078008040E800A0
:1094900030BB20000148780010C0B300E45A02003D
:1094A0000000000022C2BF00614060000004E00034
:1094B000FCFF3200301180008040780020BB20008B
:1094C000014878008040EB0010BB20000148780084
:1094D0001600370020BB2000104078000004E00098
:1094E00004003D0010C0B300606C020000000000EA
:1094F000030037000040EB00606C02000000000039
:1095000020BB2000104078000040400080407800E0
:1095100020BB20000148780010BB200010407800DC
:109520008040E80010BB20000148780010BB2000FC
:109530009040780030BB20001040780080CF500071
:10954000E4FF390010C0B300E45A0200000000003C
:1095500099FE370030BB2000104078000080FB00EF
:1095600020079800400A2000AE009000808F500035
:1095700015003200500A20002E019000800F51008B
:10958000C5003200000A2000AE019000808F51001B
:10959000010032003301370022C2BF006140600089
:1095A0000004E000FCFF32003011800080407800B1
:1095B000E0BA20000148780010C0B300E45A02006D
:1095C000000000007CFE3700E0BA20001040780068
:1095D0000080FB00100798001E009000E10F500073
:1095E000040032009E009000E28F50003B003200E9
:1095F000A500370022C2BF00614060000004E00007
:10960000FCFF320030118000605D8800605D8000EA
:109610006300B900605D88000000EB00505D8800C9
:109620000C00370022C2BF00614060000004E0006F
:10963000FCFF320071408000505D8000808040005F
:109640003011800080487800505D80000000E80004
:10965000505D8800515D8000605D8000808F50000B
:10966000F0FF39000000EB00505D88001300370068
:1096700071408000505D8000008040000080E80064
:109680001041780071408000505D800000804000F3
:109690000000E8009041780071408000505D80003B
:1096A000008040001040780083407800530107009C
:1096B000505D800063004000505D8800515D800077
:1096C000605D8000808F5000E9FF390010C0B3005A
:1096D000E45A02000000000037FE370022C2BF003B
:1096E000614060000004E000FCFF320030118000A7
:1096F000605D8800605D80004200DD00605D880084
:109700000000EB00505D88000C00370022C2BF0053
:10971000614060000004E000FCFF32007140800006
:10972000505D8000808040003011800080487800CB
:10973000505D80000000E800505D8800515D8000B1
:10974000605D8000808F5000F0FF39000000EB006A
:10975000505D8800440037000040EB00606C020060
:10976000000000000040EB00606C02000000000000
:109770000040EB00606C0200000000000040EB00C5
:10978000606C02000000000071408000505D8000AD
:1097900000804000104078000080FB009C6B0200BD
:1097A0000000000071408000505D8000008040009B
:1097B0000000E800104078000080FB009C6B020075
:1097C0000000000071408000505D8000008040007B
:1097D0000080E800104078000080FB009C6B0200D5
:1097E0000000000071408000505D8000008040005B
:1097F0006301400071408000505D800000804000A7
:1098000063004000104078006F406000004978001D
:109810008040EB0010BB20000148780006003700B4
:10982000ADFD070010BB2000104078008040E8002C
:1098300010BB20000148780071408000505D80001E
:1098400000804000630040009040780010BB200082
:109850001040780080CF5000F1FF3E00505D800046
:1098600064004000505D8800515D8000605D8000B4
:10987000808F5000B8FF390010C0B300E45A0200D6
:1098800000000000CCFD37000040EB00E45A02006D
:1098900000000000C8FD3700E0BA2000104078004A
:1098A0000080FB00000F78001E017800E10F5100DE
:1098B000040032009E017800E28F51004500320022
:1098C000BDFD370022C2BF00614060000004E0001F
:1098D000FCFF320030118000605D880022C2BF00B2
:1098E000614060000004E000FCFF320030118000A5
:1098F0008040780020BB2000014878000000EB0089
:10990000505D88002E00370020BB2000904078007A
:1099100000BB2000014878008040EB0010BB200015
:10992000014878001900370000BB20001040780083
:109930000080FB00610060000004E00004003200D1
:1099400010C0B300606C020000000000030037008C
:109950000040EB00606C02000000000000BB200033
:10996000104078000080FB000000D10080407800AB
:1099700000BB20000148780010BB20001040780098
:109980008040E80010BB20000148780010BB200098
:1099900010407800E34F5000E3FF3600F06B020008
:1099A00000000000F06B020000000000E45A02001A
:1099B00000000000505D80000000E800505D88005D
:1099C000515D8000605D8000808F5000CEFF3900C7
:1099D00079FD370022C2BF00614060000004E00052
:1099E000FCFF320030118000605D88000000EB0059
:1099F000505D88001600370022C0B30060B9200017
:109A0000A10B2000B7000700EA00070022C0B30046
:109A100060BB2D00A10B2000B200070022C0B300E4
:109A2000603D2D00A10B2000AE000700E100070003
:109A300022C0B30060BB2000A10B2000A9000700DA
:109A4000DC000700505D80000000E800505D8800E9
:109A5000515D8000605D8000808F5000E6FF39001E
:109A600055FD37000040EB00E45A02000000000002
:109A700051FD370030BB2000104078009088020074
:109A80000000000010C0B300E45A02000000000013
:109A900049FD370030BB20009040780030C0B30053
:109AA00080C0600030BB20000148780030BB20003F
:109AB00090407800809B200001487800809B200027
:109AC00090407800F0BA2000104078003C6A020014
:109AD0000000000010C0B300CC6C020000000000C9
:109AE00010C0B300E45A02000000000032FD37004D
:109AF000A09C2000104078000040A100A19C200004
:109B00008048780030BB2000104078000080FB00C7
:109B10004300DE000000A200610060000004E000DD
:109B200005003200A09C2000104078000040A000FA
:109B3000A19C20008048780021C0B300F0BA20002A
:109B40000148780030BB2000104078000080FB0006
:109B50004200DE00610060000004E000030032000B
:109B600031C0B300F0BA200001487800A09C20006A
:109B7000104078000030A100A19C200080487800AF
:109B800030BB2000104078000080FB000000D100B6
:109B9000610060000004E00005003200A09C20008D
:109BA000104078000030A000A19C20008048780080
:109BB000809B200090407800F0BA20001040780090
:109BC0003C6A02000000000010C0B300CC6C020030
:109BD0000000000010C0B300E45A020000000000C2
:109BE000F5FC37000040EB00E45A020000000000E2
:109BF000F1FC37000080FA00000006000600FA00C1
:109C00002047980031479800424798002E40900026
:109C10000080FB004600DE00004F78000040EB00B3
:109C200010479800220037001E409000E34F50007C
:109C30000C003A001E04E0000A00320010C0B3001D
:109C4000BA6C0200000000001E80FB00508202007F
:109C5000000000000040EB00BA6C020000000000B1
:109C6000100037002E4090000080FB006100600073
:109C70000004E0000400320010C0B300606C020079
:109C800000000000030037000040EB00606C0200A1
:109C9000000000002E4090000080FB000000D1007A
:109CA000204798001E4090000040E80010479800B0
:109CB0001E409000E34F5000DBFF36003E40900016
:109CC0000080FB009C6B0200000000004E409000F2
:109CD0000080FB009C6B0200000000000080FA0086
:109CE000000006000800FA001007980021079800FD
:109CF000624798000040EB00606C0200000000002A
:109D00000040EB00606C0200000000000040EB002F
:109D1000606C0200000000000040EB00606C02007C
:109D2000000000001E009000B2820200000000004F
:109D30009C6B0200000000001E009000AE0090002E
:109D40004809DD004800DE0000007100C808DE00A0
:109D5000B2820200000000009C6B020000000000C4
:109D60001E009000AE0090004008DE0001002000C0
:109D7000B2820200000000009C6B020000000000A4
:109D80006E4090006F406000604798000040EB001C
:109D9000004F7800020037004FFC07001E4FE8001C
:109DA0006E4090009E4F1000FBFF39000080FA00CB
:109DB000000006000000FA0010C0B300606C020052
:109DC000000000000040EB00606C0200000000009A
:109DD0000040EB00606C0200000000000040EB005F
:109DE000606C0200000000000000EB009C6B0200B1
:109DF00000000000F06B020000000000E45A0200C6
:109E000000000000F06B020000000000E45A0200B5
:109E10000000000030FC07002FFC07000080FA0063
:109E2000000006000200FA00D04E80000000E000B2
:109E30001200320000C2B300E45A02000000000029
:109E400031002000104420009A840200000000002D
:109E500000C2B300E45A020000000000C04E8000BF
:109E60000000E00003003A000040EB00606C0200DC
:109E7000000000000000EB00D04E8800C04E8000C3
:109E80000000E00003003A00F06B02000000000058
:109E9000004F780010002000D04E88001E80FB008C
:109EA0000080FA00000006000400FA00000F7800AD
:109EB000D04E80000000E0001200320000C2B3006B
:109EC000E45A02000000000031002000104420008D
:109ED0009A8402000000000000C2B300E45A0200AD
:109EE00000000000C04E80000000E00003003A00C7
:109EF0000040EB00606C0200000000000000EB007E
:109F0000D04E8800C04E80000000E00007003A00FC
:109F10001E0078009C6B0200000000003E6C0200F6
:109F2000000000000080FB00000F780000C2B300BA
:109F3000E45A0200000000001E00E00007003A00A2
:109F400031002000104420009A840200000000002C
:109F50000030200010079800060037004100200064
:109F6000404420009A8402000000000000102000FD
:109F7000100798001E0090000080FA000000060004
:109F80000000FA00D04E80000000E0000F00320018
:109F900041002000404420009A840200000000009C
:109FA000208B2800B456020000000000C04E800044
:109FB0000000E00003003A0010C0B300606C020033
:109FC000000000000000EB00D04E8800C04E800072
:109FD0000000E0000F003A00CA6A02000000000022
:109FE0000000E0000B00320091002000A0232000C0
:109FF0009A8402000000000051012000302420005B
:10A000009A84020000000000208B2800B456020051
:10A0100000000000D10020008044200024850200C0
:10A02000000000000080FA00000006000000FA00B6
:10A03000D04E80000000E0000F0032004100200000
:10A04000404420009A84020000000000208B280079
:10A05000B456020000000000C04E80000000E00086
:10A0600003003A0010C0B300606C02000000000062
:10A070000000EB00D04E8800C04E80000000E000E1
:10A0800002003A000A6B020000000000C10020003C
:10A090005045200024850200000000000080FA00E6
:10A0A000000006000000FA000101200020522000FC
:10A0B0009A840200000000000040EB0020590200DA
:10A0C0000000000000C2B300E45A020000000000DB
:10A0D000809B200010407800205902000000000002
:10A0E00000C2B300E45A020000000000308B2800D8
:10A0F000B4560200000000000080FA0000000600D4
:10A100000400FA000000EB00100798000000EB00CC
:10A11000C04E880008200200000000003A1C020027
:10A1200000000000000F78001E00E000090034006D
:10A13000400020009E0F100006003C001E0078002A
:10A140000040E90080407800809B200001487800B2
:10A15000020037000000EB00000F78001E00E00056
:10A160002D003A000000EB00905788000000EB0043
:10A17000C04E8800C04E80000000E0000F003A0092
:10A18000B103200060482000248502000000000088
:10A190008001EB0042002000110020001000200090
:10A1A00034210200000000000040E90080407800F7
:10A1B000809B20000148780022003700C1408000C9
:10A1C00030002300808F500004003E005103200027
:10A1D000104C20009A84020000000000C102200000
:10A1E000604F20009A840200000000008001EB0014
:10A1F0003200200011002000100020003421020055
:10A20000000000000040E90080407800809B2000B2
:10A21000014878000B003700C14080003000230067
:10A22000808F500004003E0051032000104C20009D
:10A230009A840200000000009AFF07000000EB0073
:10A24000D04E8800A09C2000104078000040A00064
:10A25000A19C200080487800C04E80000000E000F3
:10A2600009003A00C922A800C902A800CB02A9002F
:10A27000CB22A900809B20009040780020C0B30032
:10A280003C6A0200000000000080FA0000000600A6
:10A290000000FA000000EB00D04E8800C04E8000A5
:10A2A000E10F500001003A0007E2A9000080FA0027
:10A2B000000006000600FA00100798001E0090003B
:10A2C000200798002E009000E10F50000C00320093
:10A2D0002E009000E10F5000040039002E00900085
:10A2E000E20F500065003200730037005103200078
:10A2F000205320009A840200000000007200370002
:10A300008040EB0000302000EA6C020000000000FA
:10A31000E1022000705620002485020000000000A9
:10A32000CBC2BF00614060000004E00004003200C6
:10A33000CBC2BF00624060000004E0000C003A00A5
:10A3400091002000A02320009A8402000000000059
:10A3500051012000302420009A84020000000000F7
:10A36000208B2800B4560200000000005600370081
:10A370000000EB00000F780039003700C04E80006D
:10A380000000E00009003A00CA6A02000000000074
:10A390001E0078009C6B0200000000003E6C020072
:10A3A000000000000080FB00100798001E009000D5
:10A3B0000000E00024003A001E007800AA8102009C
:10A3C0000000000080C2B300E45A02000000000058
:10A3D0001E0078000080D100AA8102000000000069
:10A3E0001E0078000000A200610060000004E00090
:10A3F00004003200508B2800885602000000000044
:10A400000B003700C04E80000000E00005003A005D
:10A41000F06B02000000000010C0B300606C02008E
:10A4200000000000808B2800885602000000000019
:10A43000308B2800885602000000000000C2B300E4
:10A44000E45A020000000000C04E80000000E0005E
:10A4500002003A000A6B0200000000001E0FE80034
:10A46000F00F20009E0F1000C4FF3400208B280046
:10A47000B45602000000000013003700C04E8000F8
:10A48000E10F500001003A0007E2A900710020002E
:10A49000505920002485020000000000F100200037
:10A4A000C01E2100248502000000000010C0B3007F
:10A4B0000E0007000400370041022000C0202000E9
:10A4C00024850200000000000080FA000000060061
:10A4D0000000FA00B1002000C0092100248502001C
:10A4E000000000000080FA00000006000A00FA00E8
:10A4F000004F98000040EB00204798000040EB0020
:10A50000104798000040EB00004F78008C5B020081
:10A5100000000000C922A800C902A800CB02A900BF
:10A52000CB22A90062A0A80062C0A8008660A90092
:10A53000CBC2BF000080FB000000D1006140600082
:10A54000604798006E40900050479800CBC2BF0013
:10A5500061406000604798006E409000304798006E
:10A560000000370086C0BF00684060000004E000C3
:10A5700012003A0023C2BF00624060000004E00005
:10A580000E003A00D65B02000000000022C2BF00AD
:10A59000614060000004E000F2FF320030118000F2
:10A5A000004F780062A0A90062C0A9000E48900088
:10A5B0000004E00061003A00630037008660A900F3
:10A5C000CBC2BF000080FB000000D10061406000F2
:10A5D00060479800CBC2BF006140600040479800D0
:10A5E0002E4090000004E0002E0032003E4090001B
:10A5F0000004E0002B003A004E4090000004E00010
:10A60000280032001E409000E74F50000B003E0033
:10A610001E40780000404000004F78006E409000DF
:10A620000004E000010032001E04A0001E40900063
:10A630000040E800104798003B0037000E489000AB
:10A640000004E000040032001E80FB00AC59020050
:10A650000000000006003700C0C5B300A05B020088
:10A66000000000001E407800A05B02000000000017
:10A670006E4090000004E00004003200D0C2B3003D
:10A68000A05B02000000000003003700B0C2B3006E
:10A69000A05B0200000000000040EB0010479800A3
:10A6A000210037003E4090000004E0001E00320010
:10A6B0004E4090000004E0001B0032005E4090001D
:10A6C0000004E0000B0032006E4090000004E00047
:10A6D00008003A0010C0B300204798000040EB008B
:10A6E00010479800B0C5B300A05B02000000000056
:10A6F0000D0037005E4090000004E0000A003A00C0
:10A700006E4090000004E000070032000040EB00C3
:10A71000204798000040EB0010479800D0C5B300D8
:10A72000A05B0200000000006E40900050479800BF
:10A730004E409000304798008AFF3700208B280059
:10A74000B4560200000000000080FA00000006007D
:10A750000000FA00B08B28008856020000000000BC
:10A760000080FA00000006000A00FA00881F780046
:10A77000C922A800C902A800CB02A900CB22A900C7
:10A78000C8C2A900A09C2000104078000040A00092
:10A79000A19C200080487800A09C200010407800F8
:10A7A0000030A100A19C20008048780080C0EB0010
:10A7B00020C0B3003C6A020000000000E4FF070074
:10A7C0000000370022C2BF00614060000004E000CA
:10A7D000FCFF32003011800080407800609D200036
:10A7E00001487800609D2000104078000080FB0048
:10A7F0004400DE0080407800509D20000148780031
:10A80000509D2000104078000080FB004007980019
:10A810004E009000E10F5000EB0032004E0090001F
:10A82000E10F500004003C004E0090000000E000EA
:10A8300008003200240137004E009000E40F500061
:10A84000190132004E009000E60F5000070132005F
:10A850001D013700609D2000104078000080FB0043
:10A86000300798003E009000E40F500033003200A3
:10A870003E009000E40F500011003C003E009000AC
:10A88000E10F50001F0032003E009000E10F500029
:10A8900004003C003E0090000000E0000E01320089
:10A8A000C50037003E009000E20F50001700320054
:10A8B0003E009000E30F50001A003200BE00370047
:10A8C0003E009000E70F5000280032003E0090004C
:10A8D000E70F500004003C003E009000E60F5000DF
:10A8E0001B003200B40037003E009000E80F50001B
:10A8F000250032003E009000EF0F5000A80032000B
:10A90000AD00370092FF0700AEFF3700CA6A0200B1
:10A910000000000010C0B300E45A02000000000074
:10A92000A8FF37000A6B02000000000010C0B3004F
:10A93000E45A020000000000A2FF3700F06B0200A2
:10A9400000000000E45A0200000000009DFF3700F4
:10A950000040EB00606C02000000000010C0B3007B
:10A96000E45A02000000000096FF370010C0B30058
:10A97000606C02000000000010C0B300E45A020046
:10A98000000000008FFF370022C2BF00614060005E
:10A990000004E000FCFF3200301180001007980036
:10A9A0001E0090004800DD001007980022C2BF0082
:10A9B000614060000004E000FCFF320030118000C4
:10A9C0009E009000008070001007980022C2BF0017
:10A9D000614060000004E000FCFF320030118000A4
:10A9E000000F78001E0078004800DD00000F78009E
:10A9F00022C2BF00614060000004E000FCFF3200A2
:10AA0000301180001E0F70009E0090000000210099
:10AA1000808F500003003E00000021009E0F1000B8
:10AA2000040036000040EB00E45A02000000000081
:10AA300064FF37000000EB00200798000C0037008F
:10AA400022C2BF00614060000004E000FCFF320051
:10AA5000714080002E009000808040003011800006
:10AA6000804878002E0090000000E8002007980041
:10AA7000AE0090001E009000808F5000F0FF390063
:10AA8000CA6A0200000000000000EB0020079800E6
:10AA90000E003700714080002E00900000804000C2
:10AAA000104078000080FB009C6B0200000000005A
:10AAB0003E6C020000000000E14F5000D9FF320060
:10AAC0002E0090000000E80020079800AE009000E3
:10AAD0001E009000808F5000EEFF39001E00E9003C
:10AAE000100798000000EB002007980014003700C2
:10AAF000714080002E00900000844000F06B020046
:10AB000000000000004C7800AE0090001E00900095
:10AB1000808F5000040031000040EB00606C0200A8
:10AB2000000000000300370010C0B300606C02009A
:10AB3000000000002E0090000000E80020079800B0
:10AB40002E0090009E0F5000E9FF39000A6B0200B2
:10AB50000000000010C0B300E45A02000000000032
:10AB60000000EB00200798000900370071408000CA
:10AB70002E0090000080400010407800E45A02004F
:10AB8000000000002E0090000000E8002007980060
:10AB90002E0090009E0F5000F4FF390009FF37008F
:10ABA0000040EB0051FE070010C0B300E45A020061
:10ABB0000000000003FF37000040EB00E45A0200F1
:10ABC00000000000FFFE3700609D200090407800EC
:10ABD000F0C0B30080C06000609D20000148780094
:10ABE000609D2000104078008040E800609D2000BB
:10ABF0000148780010C0B300E45A020000000000D1
:10AC00008040EB00409D2000014878001000370094
:10AC100022C2BF00614060000004E000FCFF32007F
:10AC2000301180009C6B0200000000003E6C0200AE
:10AC300000000000E45A020000000000409D2000D7
:10AC4000104078008040E800409D200001487800D6
:10AC5000409D200090407800609D200010407800CA
:10AC600080CF5000EAFF3900D6FE3700609D2000FB
:10AC70009040780030C0B30080C06000609D20002C
:10AC800001487800609D20009040780020C0B3000B
:10AC90003C6A02000000000010C0B300E45A020049
:10ACA00000000000C7FE3700609D200010407800C3
:10ACB000908802000000000010C0B300E45A0200B7
:10ACC00000000000BFFE37000040EB00E45A020025
:10ACD00000000000BBFE37004F0478000080FA003F
:10ACE000000006000200FA00000F78001E00E000DD
:10ACF0000300320010C3B300330207000200370024
:10AD000000C3B300300207000080FA000000060014
:10AD10000600FA0010079800020037001E40780075
:10AD2000290207001E009000104F78001E40780096
:10AD3000404798004E4090000004E00002003200BE
:10AD400010C0B300404798004E4090009E00900015
:10AD50008100E800110798000004E000EFFF3A00CE
:10AD60000080FA00000006000600FA0010079800B4
:10AD7000020037001E407800130207001E009000FA
:10AD8000104F78001E407800404798004E409000D9
:10AD90000004E0000200320010C0B30040479800F9
:10ADA0004E4090009E0090008100E800110798003E
:10ADB0000004E000EFFF3A00D0C0B3000202070039
:10ADC000A0C0B300000207000080FA0000000600E7
:10ADD0000400FA002047980000C8B300004F780034
:10ADE00040892800CAFF07000040EB001047980088
:10ADF0000F0037002E4090001E4060000004E0006D
:10AE00000300320010C3B300EF0107000200370057
:10AE100000C3B300EC0107001E80FB000000D1005E
:10AE2000004F78001E4090000040E8001047980056
:10AE30001E409000E74F5000EEFF36000080FA0001
:10AE4000000006000E00FA00500798006107980005
:10AE50000040EB00004F780000102E00515F2000F2
:10AE600030079800410798000040EB001047980019
:10AE7000320037003E019000CE0190005E0090004D
:10AE8000EE009000A00502000000000010079800EE
:10AE9000210798001E04E00005003A001E00900003
:10AEA000AE009000E00F5000E08F58001800320014
:10AEB0001E0090000043B000C30107009E009000F8
:10AEC0003E009000000AB8009E0090004E009000E6
:10AED0000088B9000501780000014100BE00900023
:10AEE0002E0090000088B900000141008202780025
:10AEF0005E009000EE009000040050008580580035
:10AF0000500798006107980010C0B300004F780008
:10AF10003E009000CE009000A20020000300200020
:10AF2000A0050200000000003007980041079800CB
:10AF30001E4090000040E800104798001E4090001E
:10AF4000E74F5000CBFF36005E0090000043B0009A
:10AF50009D0107000080FA00000006000C00FA00C6
:10AF600040079800510798000000EB001007980078
:10AF70000000EB00000F78006000B8002007980088
:10AF8000310798004E019000DE019000F02324006C
:10AF9000F1002000800F5100818F59002100360000
:10AFA0004E009000DE00900002242400F3002000F8
:10AFB000A00502000000000020079800310798005B
:10AFC0002E0090006F000700C0C2B3007E01070092
:10AFD0004E009000DE00900002242400F3002000C8
:10AFE000C0050200000000004007980051079800CB
:10AFF0004E019000DE019000703E20000100200014
:10B00000800F5100818F590002003E007089280096
:10B010003FFF0700100020001007980010002000DC
:10B02000000F78004E019000DE019000703E20007D
:10B0300001002000800F5100818F5900320036003E
:10B040004E009000DE009000823E200003002000B1
:10B05000A0050200000000002007980031079800BA
:10B060002E019000BE01900040062000010020004B
:10B07000800F5100818F5900030036002E00900090
:10B0800040000700140037001E0090000000E000A0
:10B090000F0032002E019000BE019000A0002000A1
:10B0A00001002000800F5100818F590003003600FD
:10B0B00000C3B3004401070002003700C089280024
:10B0C00013FF07002E0090002E000700020037003B
:10B0D0002E0090002B000700C0C2B3003A01070009
:10B0E0004E009000DE009000823E20000300200011
:10B0F000C0050200000000004007980051079800BA
:10B1000010002000000F78004E019000DE0190003A
:10B110004006200001002000800F5100818F59005F
:10B12000030036004E0090001600070013003700A1
:10B130001E00E0000F0032004E019000DE01900082
:10B14000A000200001002000800F5100818F5900D5
:10B150000300360000C3B3001B01070002003700E4
:10B16000C0892800EAFE07004E0090000500070095
:10B17000020037004E009000020007000080FA0035
:10B18000000006000800FA00300798000040EB00BD
:10B19000004F780000712200200798000040EB006B
:10B1A000104798001E0037003E0090002E019000CE
:10B1B000110009000280D800100798001E04E0006A
:10B1C00003003A001E0090000000E0000C00320076
:10B1D0001E0090000043B000FB0007009E0090009E
:10B1E0002E0090000088B900800078003E0090009A
:10B1F000010050003007980010C0B300004F7800E5
:10B200002E009000A2002000110009000280D8004A
:10B21000200798001E4090000040E800104798006A
:10B220001E409000E34F5000DFFF36003E009000CC
:10B230000043B000E40007000080FA0000000600B0
:10B240000600FA00404798000040EB00004F7800ED
:10B2500040C6B300304798000040EB0020479800FC
:10B26000200037004E4090008080FB003E40900060
:10B270000081FB00110009008280D800104798006F
:10B280001E04E00003003A001E4090000004E000AD
:10B290000B0032001E4090000043B000CA000700BF
:10B2A0004E4190009E4090003E4090000088B900C2
:10B2B000004051004047980010C0B300004F780094
:10B2C0003E4090000080FB00A20020001100090019
:10B2D0000280D800304798002E4090000040E800DF
:10B2E000204798002E409000E14F5000DDFF3600CF
:10B2F0004E4090000043B000B30007000080FA0009
:10B30000000006000400FA0010079800F08A2800E8
:10B310007FFE07001E0090004400DE006F0F6000FB
:10B320009E007800F08928000080400010407800DE
:10B33000A50007001E0090006F0F60009E007800BF
:10B34000F089280000804000104078009E0007002F
:10B350000080FA00000006000400FA0010079800C0
:10B3600000C3B300F600070080C7B300F400070075
:10B370001E0090004400DE006F0F60009E00780009
:10B38000F08928000080400010407800EC000700A1
:10B390001E0090006F0F60009E007800F08928006A
:10B3A0000080400010407800E50007000080FA00AF
:10B3B000000006000400FA0010079800F08A280038
:10B3C00053FE07001E0090004C00DE006F0F60006F
:10B3D0009E007800F089280000804000104078002E
:10B3E000790007001E0090004800DE006F0F60002B
:10B3F0009E007800F089280000804000104078000E
:10B40000710007001E0090004400DE006F0F600016
:10B410009E007800F08928000080400010407800ED
:10B42000690007001E0090006F0F60009E0078000A
:10B43000F08928000080400010407800620007007A
:10B440000080FA00000006000800FA0030079800AB
:10B450003E009000CF80DE00640302000000000088
:10B46000926C2200B3312400C203020000000000ED
:10B4700010079800210798001E009000AE00900071
:10B48000C605020000000000004F78001E40780052
:10B490006BFF0700E0C2B3004B0007001E009000E6
:10B4A000AE009000C605020000000000CF80DE0064
:10B4B00064030200000000000001BE001E009000B6
:10B4C000AE00900046040200000000001007980043
:10B4D0002107980002002000031224001E009000A3
:10B4E000AE00900002050200000000001007980066
:10B4F000210798001E009000AE009000C6050200D3
:10B5000000000000004F78001E4078004CFF07004C
:10B510001E009000AE009000C60502000000000072
:10B52000CF80DE0064030200000000000001BE00C6
:10B530001E009000AE0090004604020000000000D3
:10B540001007980021079800020020000312240031
:10B550001E009000AE0090000205020000000000F6
:10B5600010079800210798001E009000AE00900080
:10B57000C605020000000000004F78001E40780061
:10B580002FFF07000080FA00000006000000FA000C
:10B5900022C2BF00614060000080FB000080FA0012
:10B5A000000006000000FA0022C2BF0061406000F7
:10B5B0000004E000FCFF3200301180000080FB003E
:10B5C0000080FA00000006000200FA00004F780038
:10B5D000D040800001102000010060000000E00069
:10B5E00006003A0023C2BF00624060000004E00091
:10B5F000FCFF3A001E00FB00201188000080FA00CA
:10B60000000006000200FA00004F78001E80FB00D8
:10B61000401188000080FA00000006000000FA00D7
:10B6200095C0BF00704060000004E00010003A00C8
:10B630005140800040408000808F50000C0032005C
:10B6400023C2BF00624060000004E000FCFF3A003B
:10B650008580A9009580A80031408000404080008E
:10B6600000804000104078000080FB00201188001E
:10B670000080FA0000000600809FBE000000FA0073
:10B680000140800020408000808040003011800018
:10B6900080487800204080000000E80020408800BA
:10B6A0002140800010408000808F500001003A004F
:10B6B0009560A9008560A9000080FA004F00BE00D7
:10B6C00000400600809FBE000000FA00404080005D
:10B6D0000000E80040408800414080005040800069
:10B6E000808F500002003A009580A90006003700C4
:10B6F00031408000404080000080400010407800D1
:10B700000080FB00201188008580A9000080FA00DD
:10B710004F00BE00004006000000FA000000EB00F1
:10B72000C05C880010002000B05C8800D040800021
:10B7300000A0A100D04088000080FA0000000600B0
:10B740000200FA00004F7800B15C8000C05C80000D
:10B75000808F500005003A00C222A900D04080002E
:10B7600000A0A000D04088000E003700714080008B
:10B77000B05C8000808040001E40780080487800E7
:10B78000B05C80000000E800B05C8800B15C800024
:10B7900000002100808F500002003A000000EB0002
:10B7A000B05C88000080FA00000006000200FA0089
:10B7B000C05C8000000FE800000021009E0F100018
:10B7C00002003A000000EB00000F7800B05C80003F
:10B7D0009E0F10000C00320023C2BF0062406000C8
:10B7E0000004E00008003A001E007800C05C8800F9
:10B7F00071408000C05C80000080400010407800F4
:10B800000080FB00201188000080FA000000060084
:10B810000200FA0000003700C05C8000000FE80062
:10B82000000021009E0F100002003A000000EB0013
:10B83000000F7800B05C80009E0F10000D003200F9
:10B8400023C2BF00624060000004E000F2FF3A0043
:10B850001E007800C05C880071408000C05C8000E1
:10B8600000804000104078000080FB00201188001C
:10B87000E9FF37000080FA00000006000800FA0027
:10B880002007980031079800900180001007980069
:10B890002E009000900188003E0090001080BA00B9
:10B8A000C800DD003E0090001000BA00008F70005C
:10B8B0001E009000900188001E0078000080FA00B1
:10B8C000000006000000FA00E08C28008856020004
:10B8D000000000000080FA00000006000200FA00EC
:10B8E000C222A80000010700F6FF07000000370091
:10B8F000F40007008040780060BA2000014878001A
:10B9000060BA2000104078000004E000E700350035
:10B9100060BA2000104078000004E00002003A0005
:10B92000E8FF0700F2FF370060BA200010407800FF
:10B93000E14F500004003A00EB000700EA00070066
:10B94000E0FF0700EAFF370060BA200010407800EF
:10B95000E24F500004003A00E3000700E200070055
:10B96000D8FF0700E2FF370060BA200010407800DF
:10B97000E34F500004003A00DB000700DA00070044
:10B98000D0FF0700DAFF370060BA200010407800CF
:10B99000E44F500004003A00D3000700D200070033
:10B9A000C8FF0700D2FF370060BA200010407800BF
:10B9B000E54F500006003A00CB0007009C4702000C
:10B9C00000000000C8000700BEFF0700C8FF3700E6
:10B9D00060BA200010407800E64F500004003A00A2
:10B9E000C1000700C0000700B6FF0700C0FF370016
:10B9F00060BA200010407800E74F500004003A0081
:10BA0000B9000700B8000700AEFF0700B8FF370015
:10BA100060BA200010407800EF4F50000A003A0052
:10BA200010C0B300E45A020000000000C222A900C6
:10BA300023C2BF00614060000004E000FCFF320050
:10BA40000000FE00AAFF370060BA20001040780016
:10BA5000F04F500003003A000040EB00DF01070008
:10BA6000A3FF370060BA200010407800F14F50006B
:10BA700003003A0010C0B300D80107009CFF370054
:10BA800060BA200010407800F24F500035003A00B4
:10BA90000000EB00800888000000EB00F008880040
:10BAA0000000EB00E00C8800A16C200091407800C1
:10BAB00000CEB30000C060006041B300CAE6B7002A
:10BAC000800007000080FB00000F78001E00780057
:10BAD0000000D100610060000004E00001003200BD
:10BAE00010A1A8009E007800618060000004E000C2
:10BAF000010032001081A800720007000080FB00E6
:10BB00004800DD00000F78006E0007000080FB0099
:10BB10001E0F70001E007800D00C88009E00780078
:10BB2000C10C880060002000E00C88006500070060
:10BB30000080FB004800DD00000F78006100070076
:10BB40000080FB001E0F70001E0078006008880057
:10BB500011E1A80010C0B300E45A02000000000088
:10BB600063FF370060BA200010407800F34F5000A8
:10BB70000D003A000000EB00800888000000EB0098
:10BB8000E00C8800A16C20009140780000CEB3004A
:10BB900000C06000CAE6B70010C0B300E45A02005B
:10BBA0000000000052FF370060BA2000104078000B
:10BBB000F44F50000E003A0021E3A800C0C0B300CB
:10BBC000F280020000000000000F780021E3A900CD
:10BBD0001E0078004800DE00E45A02000000000069
:10BBE0001E007800E45A02000000000040FF370009
:10BBF00060BA200010407800F54F500018003A005D
:10BC000021E3A800C0C0B300F280020000000000E1
:10BC1000000F780023C2BF00614060000004E00014
:10BC2000FCFF32001E0078004800DE00E45A0200EB
:10BC3000000000001E007800E45A0200000000002E
:10BC400022C2BF00614060000004E000EDFF32004E
:10BC500031118000010F780021E3A90024FF370093
:10BC600060BA2000104078000080FB004500DE0034
:10BC70000080FB000000D100610060000004E000D3
:10BC80000600320060BA2000104078001D00070056
:10BC9000E45A02000000000015FF37000040EB00EE
:10BCA000E45A02000000000011FF370060BA2000D3
:10BCB00010407800A3000700E45A020000000000D2
:10BCC0000BFF37000000FA0022C2BF006140600095
:10BCD0000004E000FCFF3200301180000080FB0017
:10BCE0000080FA00000006000000FA0000C0EB002F
:10BCF000040007000040EB00920007000080FA00FB
:10BD0000000006000400FA00204798000040EB0005
:10BD1000004F78002E4090000080FB004400DE00C1
:10BD2000610060000004E0000200320010C0B300B7
:10BD3000004F78009E40780061C060006140600064
:10BD40004201DD00912C200091407800B0CFB3007B
:10BD500000C0600002407000C9E2B7000040EB0084
:10BD6000004F78002E4090000080FB004300DE0072
:10BD7000610060000004E0000200320010C0B30067
:10BD8000004F78009E40780061C060006140600014
:10BD900000414000912C200091407800D0CFB300AA
:10BDA00000C0600002407000C9E2B7000040EB0034
:10BDB000004F78002E4090000080FB004200DE0023
:10BDC000610060000004E0000200320010C0B30017
:10BDD000004F78009E40780061C0600061416000C3
:10BDE000912C200091407800E0CFB30000C06000AB
:10BDF00002407000C9E2B7000040EB00004F78003D
:10BE00002E4090000080FB000000D1006100600027
:10BE10000004E0000200320010C0B300004F7800C0
:10BE20009E40780061C06000C700DD00C8C2BF004E
:10BE30000074A10001407000C8E2B7000040EB00B0
:10BE4000004F78002E4090000080FB0061006000F1
:10BE50000004E0000200320010C0B300004F780080
:10BE60009E40780061C06000614060004601DD00D6
:10BE7000812C200091407800F0CBB30000C060001E
:10BE800002407000C8E2B700500020007C8202002F
:10BE900000000000AE40900000CEB30000C0600083
:10BEA00020479800CBC2BF00644060000004E0005F
:10BEB000030032002E4090000044A000204798006C
:10BEC000CBC2BF00624060000004E000030032000B
:10BED0002E4090000034A00020479800CBC2BF0045
:10BEE000614060000004E000030032002E4090003A
:10BEF0000024A00020479800CAC2BF0001C8B300B8
:10BF0000014060000004E000030032002E40900079
:10BF10000014A00020479800CAC2BF000044B2002D
:10BF20000004E000030032002E4090000004A00056
:10BF3000204798002E4090000080FB000080FA000F
:10BF4000000006000400FA00204798002E409000F0
:10BF50000080FB004600DE00610060000004E0009D
:10BF600003003200C002A900C202A800020037008C
:10BF7000C002A900C202A9002E4090000080FB0070
:10BF80004500DE00610060000004E00003003200B4
:10BF9000C962A800CB62A90002003700CB62A900E9
:10BFA000C962A9000040EB00004F78002E409000CD
:10BFB0000080FB004400DE00610060000004E0003F
:10BFC0000200320010C0B300004F78009E4078009D
:10BFD00061C06000614060004201DD00B12C2000C2
:10BFE00091407800B0CFB30000C060000240700004
:10BFF000CBE2B7000040EB00004F78002E409000ED
:10C000000080FB004300DE00610060000004E000EF
:10C010000200320010C0B300004F78009E4078004C
:10C0200061C060006140600000414000B12C200010
:10C0300091407800D0CFB30000C060000240700093
:10C04000CBE2B7000040EB00004F78002E4090009C
:10C050000080FB004200DE00610060000004E000A0
:10C060000200320010C0B300004F78009E407800FC
:10C0700061C0600061416000B12C200091407800F7
:10C08000E0CFB30000C0600002407000CBE2B70018
:10C090000040EB00004F78002E4090000080FB0035
:10C0A0000000D100610060000004E00002003200E6
:10C0B00010C0B300004F78009E40780061C060005F
:10C0C000C700DD00CAC2BF000074A10001407000BB
:10C0D000CAE2B7000040EB00004F78002E4090000D
:10C0E0000080FB00610060000004E00002003200FC
:10C0F00010C0B300004F78009E40780061C060001F
:10C10000614060004601DD00A12C200091407800D4
:10C11000F0CBB30000C0600002407000CAE2B7007C
:10C12000500020007C82020000000000AE40900021
:10C1300000CEB30000C0600020479800CBC2BF0013
:10C14000644060000004E000030032002E409000D4
:10C150000044A00020479800CBC2BF0062406000AE
:10C160000004E000030032002E4090000034A000E4
:10C1700020479800CBC2BF00614060000004E0008F
:10C18000030032002E4090000024A00020479800B9
:10C19000CAC2BF0001C8B300014060000004E00053
:10C1A000030032002E4090000014A00020479800A9
:10C1B000CAC2BF000044B2000004E0000300320025
:10C1C0002E4090000004A000204798002E409000D0
:10C1D0000080FB000080FA00000006000400FA0066
:10C1E00020479800AE4090000040EB00C87D020060
:10C1F00000000000104798001E4090000004E0007E
:10C2000001003200C222A8001E409000E45A020041
:10C210000000000000003700C65A020000000000C5
:10C220000004E0000F003200D25A020000000000BB
:10C23000004F780000C0EB009E4F10000500320058
:10C240001E4090001E404000E45A02000000000022
:10C250000400370010C0B300E45A020000000000E0
:10C260001A0037001E4090000004E000EAFF3A0088
:10C27000405D80000000E00010003A000080EB000C
:10C28000405D8800C2C2BF000080FB000000D100FA
:10C29000614060000004A2006140600061406000F5
:10C2A00000414000212C200091407800D0CFB30005
:10C2B00000C0600002407000C2E2B700405D800034
:10C2C0000000E900405D8800D3FF37000080FA00DD
:10C2D000000006000600FA000000EB00800888005D
:10C2E0000000EB00F00888000000EB00E00C880084
:10C2F000504F80000000E00008003A00A16C2000D0
:10C300009140780000CEB30000C06000CAE6B700DC
:10C310000000EB00E04E88003D003700504F8000E9
:10C32000E30F500005003C00E0032000000F780000
:10C3300010A1A8001081A80015003700504F800000
:10C34000FE0F500005003C00A00F2000000F7800F9
:10C3500010A1A8001081A9000D003700514F8000E6
:10C36000400F2000808F500005003C00007D200021
:10C37000000F780010A1A9001081A8000400370068
:10C3800000E82300000F780010A1A9001081A90087
:10C39000504F8000000178001E0078001100090055
:10C3A0000280D8000000E900200798002E009000CD
:10C3B00060088800604F8000800078002E009000A8
:10C3C0000088B90042062000110009000280D80050
:10C3D00010079800A16C20009140780000CEB300B7
:10C3E00000C060006041B300CAE6B7001E009000C4
:10C3F000D00C88001E009000C00C88006000200057
:10C40000E00C880011E1A80020002000E04E880028
:10C410000080FA00000006001200FA000000EB00A5
:10C42000800888000000EB00F00888000000EB00A6
:10C43000E00C8800E04E8000E20F500014003A004B
:10C44000A16C20009140780000CEB30000C06000D5
:10C45000CAE6B700C1002000C02E200024850200DB
:10C46000000000000000EB00E04E880080578000D4
:10C470008000E800F00F200080806000E09E200037
:10C4800000804000104078000004E000AC00320062
:10C490000000EB0020079800805780008000E80033
:10C4A000F00F200000806000805788000820020004
:10C4B000000000003A1C0200000000004007980045
:10C4C00008200200000000003A1C020000000000EA
:10C4D000CF80DE006403020000000000008FBE0079
:10C4E0004E0090000000E00007003200CE009000F7
:10C4F000F0F92000808F500003003E002E009000D5
:10C500000000E800200798006011B8001E00BE007F
:10C51000BA030200000000000000E00001003C003F
:10C520000B00370002002000832C24001E00BE00F8
:10C53000BE030200000000000000E0000100350022
:10C54000030037002E0090000000E800200798004C
:10C550002E009000E20F5000110032000000EB00AE
:10C560009057880011012000802F200024850200B0
:10C570000000000011012000903020009A84020089
:10C58000000000008001EB0002FA200011002000F2
:10C590002003200034210200000000004007980022
:10C5A0004E009000E30F500005003E00E003200025
:10C5B0003007980010A1A8001081A80015003700CE
:10C5C0004E009000FE0F500005003E00A00F20001E
:10C5D0003007980010A1A8001081A9000D003700B5
:10C5E000CE009000400F2000808F500005003E00DC
:10C5F000007D20003007980010A1A9001081A8003C
:10C600000400370000E823003007980010A1A900BB
:10C610001081A9003E0090004E0190001100090019
:10C620000280D8000000E900600798002E0090000A
:10C63000E20F50000E003200010120007032200095
:10C640009A840200000000008001EB003206200006
:10C650008000EB00200320003421020000000000D5
:10C66000CF80DE006403020000000000008FBE00E7
:10C6700002002000832C24001E00BE00C203020022
:10C6800000000000008FBE006E009000CF80DE0032
:10C69000640302000000000070079800010F98007A
:10C6A0006E0090000000E00008003D000200200045
:10C6B000037824007E0090008E0890004804020059
:10C6C0000000000070079800010F98001E01BE00D6
:10C6D0007E0090008E08900002050200000000001D
:10C6E0006A0502000000000050079800A16C2000BD
:10C6F0009140780000CEB30000C060006041B300FC
:10C70000CAE6B7005E009000D00C88005E00900082
:10C71000C00C880060002000E00C88006E009000D3
:10C720006008880011E1A800A100200070332000FB
:10C73000248502000000000020002000E04E880058
:10C740000080FA00000006000000FA00E04E8000C1
:10C75000E20F500005003A00F101200010342000E3
:10C7600024850200000000003E003700F100200098
:10C77000003620009A840200000000000000EB0058
:10C78000F00888000000EB0080088800C942A8007B
:10C79000616820009140780000CEB30000C06000C6
:10C7A000A040B30086E6B700A00320008008880000
:10C7B0002E000700F04E8800014F8800F24E8000E6
:10C7C000034F8000F00F200001002000800F510077
:10C7D000818F590009003600F04E8000014F800023
:10C7E000C808DD000080FD00804078000040EB00BC
:10C7F000F04E8800014F880009003700B10020008A
:10C80000B01921009A84020000000000A00020005E
:10C810008008880015000700F04E8800014F88004E
:10C82000F04E8000014F8000AE5702000000000073
:10C83000808C28008856020000000000C08C280070
:10C84000B45602000000000086C6BF00F041B300ED
:10C8500086E6B7000000EB00F00888000000EB005F
:10C86000800888000080FA00000006000000FA003E
:10C870000080EB00700888000080EB0060088800F2
:10C880000000EB00400888000000EB003008880042
:10C890000000EB00B00888000000EB00A008880052
:10C8A00080002000F0088800400F2000E008880089
:10C8B00000402200D00888008780A9001FE1A8005E
:10C8C00011E1A80087C0BF00704060000004E000D4
:10C8D000FCFF320011E1A9001FE1A900300880002F
:10C8E000404F880040088000304F8800304F800063
:10C8F00001002000104F8800214F8800104F800059
:10C90000214F8000C000DD0000002000104F880093
:10C91000214F8800404F80006101B800104F800017
:10C92000214F80000200400083804800104F8800A3
:10C93000214F8800104F8000214F80000080FA00B6
:10C94000000006000000FA00A09C200010407800C3
:10C95000634060000004E00002003A00C942A80001
:10C9600001003700C8C2A800E1002000F036200016
:10C970009A840200000000000080FA000000060017
:10C980000000FA00A09C2000104078006340600086
:10C990000004E00003003A00C942A900CB42A8000D
:10C9A00002003700C8C2A900CAC2A8008100200046
:10C9B000D037200024850200000000000080FA002B
:10C9C000000006000000FA00A09C20001040780043
:10C9D000634060000004E00003003A00C942A9007F
:10C9E000CB42A90002003700C8C2A900CAC2A900F0
:10C9F0007100200050382000248502000000000053
:10CA00000080FA00000006000200FA00A09C20004E
:10CA100010407800634060000004E00009003A0024
:10CA2000C942A8000000000000000000CBC2BF0007
:10CA30000080FB004200DE0061406000004F780093
:10CA400008003700C8C2A800000000000000000075
:10CA5000CAC2BF000080FB004600DE0061406000EB
:10CA6000004F78001E80FB000080FA0000000600E6
:10CA70000C00FA000000EB00800888000000EB00CA
:10CA8000F00888000000EB00E00C8800E04E800019
:10CA9000E20F500014003A00A16C20009140780091
:10CAA00000CEB30000C06000CAE6B700C10020009D
:10CAB000C02E200024850200000000000000EB00D2
:10CAC000E04E8800805780008000E800F00F2000D2
:10CAD00080806000E09E20000080400010407800D0
:10CAE0000004E00064003200805780008000E8000D
:10CAF000F00F2000008060008057880008200200AE
:10CB0000000000003A1C020000000000CF80DE00A0
:10CB10006403020000000000008FBE0090578000F8
:10CB20000000E00008003A00020020004333240027
:10CB30001E00BE00BA030200000000000000E0007A
:10CB400001003C00100037000000EB009057880007
:10CB50003101200040242100248502000000000053
:10CB60008001EB00420B20008000EB00A0052000BC
:10CB70003421020000000000CF80DE0064030200C8
:10CB800000000000008FBE0010A1A8001081A800C6
:10CB9000204E20003007980002002C00A3552400EE
:10CBA0001E00BE00C203020000000000008FBE0095
:10CBB0003E009000CF80DE00640302000000000011
:10CBC00040079800510798003E0090000000E000E8
:10CBD00008003D0002002000037824004E00900071
:10CBE000DE009000480402000000000040079800AA
:10CBF000510798001E01BE004E009000DE0090001C
:10CC0000020502000000000002002000832724002B
:10CC100048040200000000006A0502000000000055
:10CC200020079800A16C20009140780000CEB3004E
:10CC300000C060006041B300CAE6B7002E0090005B
:10CC4000D00C88002E009000C00C880060002000EE
:10CC5000E00C88003E0090006008880011E1A80008
:10CC6000C100200070252100248502000000000082
:10CC700020002000E04E88000080FA00000006003E
:10CC80000000FA00A09C2000104078000040A000A6
:10CC9000A19C200080487800960007000080FA00E0
:10CCA000000006000000FA003C01070053000700E6
:10CCB00050032100104078000080FB000080FA0043
:10CCC000000006000400FA00100798001E00900003
:10CCD00071010700004F78001E04E00005003A00D3
:10CCE00031002000104420009A840200000000005F
:10CCF0000C00370010C0B3009E4F100005003A0032
:10CD000041002000404420009A84020000000000FE
:10CD10000400370081002000001221009A840200E4
:10CD200000000000001020000080FA000000060053
:10CD30000400FA00000F78001E0078001007980029
:10CD40001E0090000000E000040032001E00900071
:10CD5000E10F50000600320022003700610220007F
:10CD6000801221002485020000000000210037000D
:10CD7000D1002000E0142100248502000000000002
:10CD8000F1002000C01E21002485020000000000E8
:10CD9000020107000004E00008003A0050032100EF
:10CDA000104078000080FB00AA8102000000000013
:10CDB00000C2B300E45A02000000000022C2BF001B
:10CDC000614060000004E000F1FF3200301180009B
:10CDD000000F7800008F2800B45602000000000009
:10CDE0000400370041022000C020200024850200FA
:10CDF000000000000080FA00000006000400FA00B5
:10CE0000004F78001E80FB00100798009E009000E5
:10CE1000E28F50001A0032001E009000E20F500016
:10CE200007003C009E0090000100E0002F0032004F
:10CE30001E009000E10F50000C0032002700370068
:10CE40009E009000E48F5000170032001E009000FA
:10CE5000E40F50000F003500F00F20009E009000FE
:10CE6000808F5000180032001C00370001012000A4
:10CE7000B015210024850200000000001B003700CF
:10CE8000E1002000B016210024850200000000000F
:10CE900016003700F10020009017210024850200C1
:10CEA000000000001100370000C2B300E45A020085
:10CEB0000000000081002000001221009A8402007E
:10CEC00000000000090037005100200080182100F8
:10CED000248502000000000004003700E10020006B
:10CEE000D018210024850200000000000080FA0014
:10CEF000000006000000FA00C922A800C902A9002B
:10CF0000CB02A900CB22A9000080FA000000060095
:10CF10000400FA000040EB00410107000004E000BB
:10CF20000300320020002000100798000E00370098
:10CF3000CBC2BF000080FB000000D1006140600058
:10CF4000004F780010C0B300350107000004E00076
:10CF50000300320020002000100798000200370074
:10CF60001E80FB00100798001E0090000080FA0051
:10CF7000000006000600FA000040EB002047980081
:10CF80000040EB0010479800CBC2BF000080FB00C0
:10CF90000000D100E1406000400321001040780013
:10CFA00061C16000E1CFB300014060000240700049
:10CFB00041032100804878004003210010407800A0
:10CFC000614060000004E000030032001000200017
:10CFD000200798006E00370010C0B3001001070052
:10CFE0000004E00003003200410020002107980007
:10CFF000670037000040EB00304798001900370009
:10D000001E4090000080FB000000D10010479800F7
:10D01000BFFF0700004F780020C0B3009E4F1000F4
:10D0200003003A0041002000210798005800370013
:10D0300010C0B3009E4F100007003A009E409000C1
:10D0400000C8B30000C04000104798002E40900078
:10D050000004A200204798003E4090000040E800F5
:10D06000304798003E409000E74F5000E4FF360004
:10D07000500321009E40900001487800A4FF070063
:10D08000004F780020C0B3009E4F100003003A000C
:10D0900041002000210798003D0037001E40780025
:10D0A000E1406000600321001040780061C1600031
:10D0B000E1CFB30001406000024070006103210035
:10D0C00080487800600321001040780061406000D3
:10D0D0008080FB002E4090000080FB00808F50007D
:10D0E00008003A0060032100104078000020A000F2
:10D0F000610321008048780021002000210798006A
:10D100002300370060032100104078000020A100B8
:10D1100061032100804878007DFF0700004F780000
:10D1200020C0B3009E4F100003003A0041002000D1
:10D1300021079800160037001E407800614160000A
:10D140006003210090407800614061000041400090
:10D15000D0CFB30080C0600082C0700060032100A7
:10D1600001487800C902A90060032100104078003E
:10D17000624060000004E00003003A00310020003B
:10D1800021079800020037000000EB0020079800FC
:10D190002E0090000080FA00000006000200FA0055
:10D1A00000C0EB00004F7800C922A800C902A80007
:10D1B0000040EB001047980011003700CBC2BF00C1
:10D1C000614060000004E00007003A0069FF0700CA
:10D1D000004F78001E04E0000C00320040C0B30095
:10D1E0009E4F100009003200500020007C82020097
:10D1F000000000001E4090000040E800104798002A
:10D200001E409000E14F4000ECFF3A00C902A90027
:10D210001E80FB000080FA00000006000400FA00F7
:10D22000004F780010C0B3007D0007000004E0004C
:10D230000300320020002000100798001300370080
:10D240009E40780061C06000614060000041400085
:10D25000912C200091407800D0CFB30000C0600036
:10D2600002407000C9E2B7000040EB006C0007000C
:10D270000004E000030032002000200010079800A6
:10D28000020037008000EB00110798001E0090009C
:10D290000080FA00000006000800FA0040479800ED
:10D2A0000040EB0020479800C902A900CB02A9006A
:10D2B000C00320007C82020000000000CB22A900F5
:10D2C000C922A900C902A800100020007C82020027
:10D2D000000000000040EB00510007000004E000E7
:10D2E000030032004000200030079800490037005A
:10D2F0000000EB00000F78001C0037004E4090004B
:10D300000080FB00610060000004E0000B003200C0
:10D3100010C0B300C1FF07000004E00003003200AA
:10D3200040002000300798003A0037002E4090005F
:10D330000004A20020479800070037000040EB00DF
:10D34000B6FF07000004E0000300320040002000A8
:10D35000300798002F0037004E4090000080FB00FF
:10D360000000D100404798001E0FE8007000200028
:10D370009E0F1000E1FF36002E4090000004A20036
:10D38000204798002E409000A4FF07000004E00012
:10D390000300320040002000300798001D003700D5
:10D3A000C922A800CB22A90010C0B3001C000700AE
:10D3B0000004E00003003200400020003007980025
:10D3C00014003700D2FE0700E24F500003003A007D
:10D3D00040002000300798000E003700CCFE070008
:10D3E0000080FB00000F7800200020009E0F10003E
:10D3F00003003A0040002000300798000500370085
:10D40000C902A900CB02A9001E0078000080FB0021
:10D41000300798003E0090000080FA0000000600EF
:10D420000600FA00204798000080EB00000F78000B
:10D43000CBC2BF00614060008080FB002E409000A6
:10D440000080FB00808F500003003A000000EB00DA
:10D4500020079800050037001E0FE9001E00E000BD
:10D46000F3FF3A0010002000200798002E009000E3
:10D470000080FA00000006000400FA00004F780067
:10D4800011479800C0B920001E48780030C0B30092
:10D490009E4F100005003A0000202000F05C88003C
:10D4A00000082000005D88000400370000202000F4
:10D4B000F05C880000202000005D88001E40900085
:10D4C0000080FB00100798001E009000E10F500044
:10D4D000110032001E009000E20F500018003200D0
:10D4E0001E0090000000E000010032001E00370026
:10D4F00041C1B30020BA20000148780041C6B30002
:10D5000030BA20000148780021C3B30040BA20009F
:10D51000014878001D00370021C0B30020BA200068
:10D5200001487800A1C0B30030BA2000014878005B
:10D5300051C0B30040BA2000014878001300370002
:10D5400011C0B30020BA20000148780051C0B300D8
:10D5500030BA20000148780021C0B30040BA200052
:10D5600001487800090037008040EB0020BA200015
:10D57000014878008040EB0030BA20000148780074
:10D580008040EB0040BA2000014878000080FA009B
:10D59000000006000200FA000000EB00000F780017
:10D5A00030BA2000904078000030200009010700C8
:10D5B000CBC2BF00614060000004E0000400320004
:10D5C000CBC2BF00624060000004E00002003A00ED
:10D5D00010002000000F780030BA20009040780042
:10D5E000002020001701070030BA2000904078008A
:10D5F000001020001301070030BA2000904078008E
:10D6000000202000F30007001E0078000080FA00D0
:10D61000000006000000FA0030BA200090407800B8
:10D62000003020000701070030BA20009040780049
:10D6300000102000E700070030BA2000904078007A
:10D6400000202000E30007000000EB000080FA004B
:10D65000000006000C00FA00500798000000EB00E4
:10D66000000F7800909B2000104078000080FB00A5
:10D670008000E900100020000100DD003007980064
:10D680005E009000200798000000EB004007980023
:10D690002000370020BA200010417800AE00900032
:10D6A0003E0090000080600001202000FC00070088
:10D6B00030BA20009040780000102000C50007001C
:10D6C00000082000260107000080FB0010079800DA
:10D6D00030BA20009040780000102000D9000700E8
:10D6E0002E00900000004000200798001E007800E7
:10D6F00000004000000F78001E0090000000E000D5
:10D70000010032001E0FE8004E0090000000E8000B
:10D7100040079800909B2000104078008080FB001C
:10D720004E009000808F5000DAFF3E001E0078000F
:10D730000080FA00000006000800FA003007980098
:10D74000909B2000104078000080FB008000E900E2
:10D75000100020000100DD00100798003E0090003E
:10D76000000F78000000EB0020079800140037003D
:10D7700020BA2000104178001E0090001E006000BA
:10D7800001202000C600070030BA20009040780039
:10D79000001020008F00070030BA20009040780071
:10D7A00000102000A70007001E00780000004000C5
:10D7B000000F78002E0090000000E800200798007D
:10D7C000909B2000104078008080FB002E0090008D
:10D7D000808F5000E6FF3E000080FA000000060047
:10D7E0000600FA000000EB00000F78000020200087
:10D7F000DB0007000000EB00200798001600370050
:10D8000030BA20009040780000102000710007001E
:10D8100000202000D20007000080FB0010079800C5
:10D8200030BA2000904078000010200085000700EA
:10D830001E00780000004000000F78001E009000DD
:10D840000000E000010032001E0FE8002E009000F2
:10D850000000E80020079800909B2000104078000E
:10D860008080FB002E009000808F5000E4FF3E007F
:10D870001E0078000080FA00000006000200FA0096
:10D88000005D8000B600070030BA200090407800AC
:10D89000001020004F000700005D8000B00007006E
:10D8A000004F780030BA200090407800001020002F
:10D8B000640007001E80FB000080FA0000000600E4
:10D8C0000200FA00004F780020BA200010417800D2
:10D8D000F15C80001E80FB007100070030BA200060
:10D8E00090407800001020003A00070030BA200075
:10D8F0009040780000102000520007000080FA00DD
:10D90000000006000400FA00204798000040EB00E9
:10D91000004F78000900370030BA200090407800AE
:10D92000001020002B00070030BA20009040780043
:10D9300000102000430007001E4FE8002E4090001A
:10D940009E4F1000F4FF39000080FA00000006002E
:10D950000200FA00004F780020BA20001041780041
:10D96000F15C80001E80FB004D0007000080FA0083
:10D97000000006000200FA00004F780020BA2000E4
:10D98000104178001E80FB000110200044000700B9
:10D990000080FA00000006000200FA00004F780044
:10D9A00020BA2000104178001E80FB0001042000F6
:10D9B0003B0007000080FA00000006000000FA00AB
:10D9C000005D8000660007000080FB000080FA0018
:10D9D000000006000400FA00000F780021479800BC
:10D9E000A09C200010407800704060000004E0001F
:10D9F0000B003A00601680001E0070006016880060
:10DA00001E0078000080EA008180EA008000780033
:10DA10004016800000806000401688000300370038
:10DA2000401680001E007000401688002E409000B6
:10DA30000080FB007C820200000000000080FA00F1
:10DA4000000006000400FA00000F7800214798004B
:10DA50001E0078000080EA008180EA0080007800E3
:10DA60006016800000806000601688001E0078004C
:10DA70000080EA008180EA00800078004016800083
:10DA800000806000401688002E4090000080FB005F
:10DA90007C820200000000000080FA000000060006
:10DAA0000600FA00000F780011079800424798001E
:10DAB0001E00E0000F003A001E0090000080EA0007
:10DAC0008180EA008000780060168000008060009D
:10DAD000601688001E0090000080EA008180EA0045
:10DAE00080007800401680000080600040168800AA
:10DAF00015003700A09C20001040780070406000A6
:10DB00000004E0000C003A00611680001E00900046
:10DB100000807000601688001E0090000080EA00FF
:10DB20008180EA008000780040168000008060005C
:10DB30004016880004003700401680009E009000C8
:10DB400001007000401688004E4090000080FB00ED
:10DB50007C820200000000000080FA000000060045
:10DB60000400FA00000F7800401680001E007000CC
:10DB700040168800000000000000000000000000C7
:10DB8000501680001E0060000000E000030032001C
:10DB90001000200010079800020037000000EB0082
:10DBA000100798001E0090000080FA000000060098
:10DBB0000000FA00F06B0200000000000080FA0094
:10DBC000000006000200FA00000F78001E00780036
:10DBD0009C6B020000000000001020000080FA0092
:10DBE000000006000000FA00CA6A020000000000FF
:10DBF00081002000D09220009A84020000000000E2
:10DC0000D100200080442000248502000000000094
:10DC10000080FA00000006000000FA000A6B020013
:10DC20000000000061002000509320009A84020050
:10DC300000000000C10020005045200024850200A3
:10DC4000000000000080FA00000006000000FA005A
:10DC50003E6C0200000000000080FB000080FA0023
:10DC6000000006000000FA00DE6C02000000000068
:10DC70000080FB000080FA00000006000000FA00AF
:10DC80000040EB00BA6C0200000000000080FA00C7
:10DC9000000006000000FA0010C0B300BA6C0200D9
:10DCA000000000000080FA00000006000000FA00FA
:10DCB00010C0B300826C0200000000000080FA0077
:10DCC000000006000000FA000040EB00A86C020013
:10DCD000000000000080FA00000006000000FA00CA
:10DCE00010C0B300A86C0200000000000080FA0021
:10DCF000000006000000FA0001012000A0982000AA
:10DD00009A84020000000000809B200010407800F0
:10DD1000205902000000000000C2B300E45A0200D3
:10DD200000000000A09C2000104078000080FB0054
:10DD30004400DE0061406000205902000000000045
:10DD400000C2B300E45A02000000000031002000CD
:10DD5000F0AD20009A840200000000000080FA006C
:10DD6000000006000400FA00082002000000000085
:10DD70003A1C020000000000100798000820020072
:10DD8000000000003A1C020000000000000F7800B4
:10DD90001E0090000000E000090034001E0090000A
:10DDA000E40F500006003C001E0090000040E90017
:10DDB00080407800809B20000148780002003700F6
:10DDC0000000EB00100798001E00E0001000340077
:10DDD000200020009E0F10000D003C001E00780067
:10DDE0000040EA0061416000A09C20009040780063
:10DDF000614061004401DD00F0CEB30080C06000EE
:10DE000082C07000A09C200001487800020037000A
:10DE10000000EB00100798001E0090000000E000DA
:10DE200026003A000000EB0090578800B103200064
:10DE30006048200024850200000000008001EB0003
:10DE400042002000110020001000200034210200B8
:10DE5000000000000040E90080407800809B200026
:10DE600001487800F1042000B093200024850200CE
:10DE7000000000008001EB002200200011002000C3
:10DE80001000200034210200000000000040EA00E1
:10DE900061416000A09C20009040780061406100DA
:10DEA0004401DD00F0CEB30080C0600082C070008D
:10DEB000A09C200001487800010037008DFF07007A
:10DEC000CB02A900CB22A900C922A800C902A9003F
:10DED000809B20009040780020C0B3003C6A020084
:10DEE000000000000080FA00000006000400FA00B4
:10DEF000000F78001E007800100798001E009000A8
:10DF0000E10F50000C0032001E009000E10F5000A5
:10DF1000040039001E009000E20F5000070032009C
:10DF20000800370081032000A09920009A84020095
:10DF30000000000007003700100007002500070060
:10DF40000400370041022000C02020002485020088
:10DF5000000000000080FA00000006000200FA0045
:10DF6000000F7800B1002000C009210024850200C4
:10DF7000000000000080FA00000006000000FA0027
:10DF8000F1032000209D20002485020000000000F5
:10DF90000040EB00CC6C020000000000F00F2000FD
:10DFA0007C8202000000000010C0B300CC6C0200B4
:10DFB0000000000010C0B300826C020000000000EE
:10DFC0000040EB00CC6C0200000000000080FA0072
:10DFD000000006000A00FA00881F7800D102200025
:10DFE00010A120009A840200000000000000EB0055
:10DFF000000F7800100037001E047800F06B02005C
:10E000000000000080407800630047000174780041
:10E010009E00780063004700614078000080FB00AC
:10E02000825902000000000000C2B300E45A02005E
:10E03000000000001E0FE800300020009E0F1000BE
:10E04000EDFF3600808E2800B4560200000000006C
:10E05000A1002000E0A320009A840200000000003C
:10E0600063004700104078000080FB004400DE00A1
:10E070000080FB00400798004E009000E90F500020
:10E08000130032004E009000E90F500004003C00E5
:10E090004E009000E80F5000080032001B003700CF
:10E0A0004E009000EA0F50000E0032004E0090002B
:10E0B000EF0F500010003200140037006100200004
:10E0C00080A420009A8402000000000013003700A2
:10E0D00061002000E0A420009A84020000000000FB
:10E0E0000E0037006100200040A520009A84020045
:10E0F000000000000900370031002000A0A520002A
:10E100009A84020000000000040037007100200023
:10E11000D0A520009A84020000000000808E280014
:10E12000B456020000000000B100200040A620000C
:10E130009A84020000000000630047001040900035
:10E140000080FB004700DE000004E00005003A000C
:10E1500061002000F0A620009A8402000000000068
:10E1600004003700F100200050A720009A8402002C
:10E1700000000000808E2800B4560200000000005D
:10E18000C100200040A820009A8402000000000086
:10E1900063004700104090008080FB0080F72F0054
:10E1A000008060004380DE00204798002E409000F1
:10E1B0000004E00005003A00D100200000A9200082
:10E1C0009A840200000000001E0037002E409000DC
:10E1D000EF4F500005003A0031002000A0A52000BC
:10E1E0009A8402000000000016003700000420009E
:10E1F000000F7800E30047000040EB008048780003
:10E20000080037001E00780000004000000F780072
:10E2100063004700104078008040E800630047003A
:10E220000148780063004700904078002E4090003D
:10E2300080CF5000F3FF39001E007800C258020062
:10E2400000000000808E2800B4560200000000008C
:10E2500091012000D0A920009A8402000000000053
:10E26000630047009040900070C0B30000C06000A1
:10E270002047980010002000000F7800E3004700BE
:10E280000040EB0080487800080037001E0078004E
:10E2900000004000000F7800630047001040780045
:10E2A0008040E800630047000148780063004700B1
:10E2B000904078002E40900080CF5000F3FF39004E
:10E2C0001E0078002059020000000000808E280007
:10E2D000B4560200000000004F0478000080FA00ED
:10E2E000000006000200FA00000F78001E0078000F
:10E2F0008040780020032100104078000080FB005F
:10E300000000D100614060004401070000102000BF
:10E310000080FA00000006000000FA00200321003F
:10E32000104078000010A1002103210080487800EF
:10E3300041012000B0EC2000248502000000000014
:10E340000080FA00000006000000FA00200321000F
:10E35000104078000010A0002103210080487800C0
:10E3600021012000F0ED20002485020000000000C3
:10E370000080FA00000006000000FA00A09C2000C7
:10E38000104078000040A000A19C20008048780048
:10E3900020032100104078000010A000210321007C
:10E3A00080487800816A20009140780000CEB30058
:10E3B00000C060007040B300A8E6B700916C200078
:10E3C0009140780000CEB30000C060007040B30000
:10E3D000C9E6B700816C20009140780000CEB30000
:10E3E00000C060000034A000C8E6B700CAC2A9009F
:10E3F000C8C2A900C902A900C8E2A800C922A90090
:10E40000D0132000101288000000EB0020128800BA
:10E410000000EB000012880041E2A800D1012000BA
:10E4200040F0200024850200000000000080FA0077
:10E43000000006000800FA002007980080578000BE
:10E440008000E800F00F2000008060008057880006
:10E4500008200200000000003A1C0200000000003A
:10E46000100798000000EB00905788002E009000E5
:10E47000300798003E009000E30F50003C0032004F
:10E480003E009000E30F500004003E003E0090006C
:10E490000000E0000B0032000F0037003E0090004B
:10E4A000E60F5000480032003E009000E70F500099
:10E4B0006A0032003E009000E40F50003700320046
:10E4C0008B0037008109200060F6200024850200BF
:10E4D000000000008A003700510020003063200057
:10E4E0002485020000000000AC0007002E00900010
:10E4F000E10F5000820032001E0090000000E0009A
:10E50000030034001E009000E20F5000130034009E
:10E5100041022000E0FF20002485020000000000EE
:10E520008001EB00220020001100200020002000CC
:10E530003421020000000000100798001E00900027
:10E54000E10F500003003A000040EB0075000700A7
:10E550000200370080C0B3007200070041002000B5
:10E560002002210024850200000000006400370022
:10E5700011C0B3000040EB00A8000700F00020002D
:10E5800050820200000000005100200060022100C3
:10E590002485020000000000590037001E00900092
:10E5A0008040780000C8B30080C070000040EB00DD
:10E5B0009A000700A1002000B0022100248502007B
:10E5C000000000004E00370011C0B3000040EB0017
:10E5D00092000700F00020005082020000000000BE
:10E5E00000032000200798001E0090000000E000BB
:10E5F00002003A0000052000100798000000EB0020
:10E60000000F780011003700AE009000900320004A
:10E61000808F500002003600000320002007980081
:10E620002E0090008040780010C0B3007B000700EF
:10E630002E009000E45A0200000000002E0090001E
:10E640000000E800200798001E0FE8001E00900060
:10E650009E0F1000ECFF35002900370011C0B300F9
:10E660000040EB006D000700F00020005082020027
:10E670000000000010022000200798001E009000FB
:10E680000000E00002003A0000052000100798009A
:10E690000000EB00000F780011003700AE00900082
:10E6A000F0072000808F500002003600100220008A
:10E6B000200798002E0090008040780010C0B30022
:10E6C000560007002E009000E45A020000000000EF
:10E6D0002E0090000000E800200798001E0FE800C0
:10E6E0001E0090009E0F1000ECFF35000400370064
:10E6F00041022000C020200024850200000000000C
:10E700000080FA00000006000000FA00B1002000BE
:10E71000C009210024850200000000000080FA00EA
:10E72000000006000200FA00004F78001E4078004A
:10E730000042B000804078000040EB003700070046
:10E74000F0002000508202000000000081C0B300F1
:10E750000040EB0031000700F00020005082020072
:10E760000000000011C0B3000040EB002B000700C8
:10E77000F00020005082020000000000E1C0B30061
:10E780000040EB0025000700F0002000508202004E
:10E79000000000000080FA00000006000000FA00FF
:10E7A0000040EB006C000700F000200050820200E7
:10E7B0000000000031C0B3000040EB00260007005D
:10E7C00050002000508202000000000031C0B30061
:10E7D0000040EB0020000700000A20007C820200BD
:10E7E0000000000031C0B3000040EB001A00070039
:10E7F000000A20007C8202000000000021C0B3005B
:10E800000040EB0014000700000A20007C82020098
:10E81000000000000080FA00000006000200FA007C
:10E82000004F7800114798001E4090000080FB00C8
:10E830004400DE00804078001E407800060007009B
:10E840001E409000EF4060001E407800020007006C
:10E850000080FA00000006000200FA00004F780075
:10E86000114798001E4090004400DD0010479800BA
:10E870001E4090000004A0001047980010C0B30094
:10E880009E4F100003003A001E4090000014A000AC
:10E89000104798001E4090002F0007001E40900077
:10E8A0000034A000104798001E4090002A00070086
:10E8B0009E40900070CFB30000C0600010479800E9
:10E8C0001E409000240007000080FA0000000600AF
:10E8D0000200FA00004F78001E80FB004012880002
:10E8E00085C0BF00644060000004E000FCFF32000F
:10E8F00040128000004F78008540A9001E80FB0078
:10E900000080FA00000006000000FA0041E2A900C1
:10E91000A8C6BF00F041B300A8E6B700916C200084
:10E920009140780000CEB30000C06000C9E6B70097
:10E93000816C20009140780000CEB30000C06000E0
:10E94000C8E6B700CEE2A900CF02A900CEC2A90056
:10E950000080FA00000006000200FA00004F780074
:10E960001E407800DAFF0700CAC2A800CAC2A90088
:10E970000080FA00000006000000FA00008E280067
:10E9800088560200000000000080FA000000060027
:10E990000A00FA0070408000300798001000200044
:10E9A000C0818800F4FF070000003700D25A02003F
:10E9B00000000000104798001E4090000080FB00FF
:10E9C00040079800CE009000E38F500020003200F6
:10E9D0004E009000E30F50000A003C00CE00900073
:10E9E000E18F50005B0032004E009000E10F5000BC
:10E9F0005E003C00CE0090000100E000E700320025
:10EA0000DB0037004E009000E60F50000E00320091
:10EA1000CE009000E68F500004003C004E009000B5
:10EA2000E50F500095003200D1003700CE00900075
:10EA3000E78F5000640032004E009000E80F500055
:10EA400054003200CA003700CBFF0700D7FF370061
:10EA5000BE00900030C0B300804878003E009000B7
:10EA60008000E80080C0B3008048780021E3A8005F
:10EA7000C0C0B300F2800200000000002007980030
:10EA80003E0090008080E8002E0090004800DE00EC
:10EA9000804878003E009000E30040002E00900087
:10EAA00080487800B0C0B300F2800200000000008F
:10EAB000200798003E009000E40040002E009000E7
:10EAC0004800DE00804878003E009000E5004000ED
:10EAD0002E00900080487800A0C0B300F2800200B1
:10EAE00000000000200798003E009000E600400073
:10EAF0002E0090004800DE00804878003E00900024
:10EB0000E70040002E0090008048780090C0B300DD
:10EB1000F280020000000000200798003E009000F4
:10EB2000E80040002E0090004800DE008048780099
:10EB30003E009000E90040002E00900080487800E0
:10EB400021E3A900A10020003E009000BF000700C3
:10EB500096FF3700D25A02000000000010479800CC
:10EB60001E4090008F00070090FF3700D25A02002D
:10EB70000000000010479800D25A02000000000078
:10EB8000004F78009E4078001E409000C1000700B2
:10EB900086FF3700D25A020000000000104798009C
:10EBA000D25A020000000000004F78001E40900082
:10EBB0000080FB00C800DD001E80FB0000807000AC
:10EBC000C081880079FF3700D25A0200000000009F
:10EBD000104798001E4090000080FB00200798001E
:10EBE0001E409000E14F500004003A0030C0B300D6
:10EBF000025B0200000000000300370020C2B300E7
:10EC0000025B020000000000D25A02000000000077
:10EC100010479800D25A020000000000004F780010
:10EC20009E409000A0CAB30080CF500003003A007D
:10EC300050C5B3009E4F1000050032000000EB00ED
:10EC40002007980020C2B300025B02000000000011
:10EC5000BE00900070C0B300804878003E00900075
:10EC60008000E8002E0090008048780021002000FD
:10EC70003E009000750007004CFF3700D25A02009A
:10EC80000000000010479800D25A02000000000067
:10EC9000004F78008560A9001E4090000080FB00B6
:10ECA000C800DD001E80FB00008070001007980087
:10ECB0009E00900000002200808F5000020036006D
:10ECC00000002200100798001E009000670040001E
:10ECD0004300DE0020079800BE00900050C0B30043
:10ECE000804878003E0090000000E8009E409000C0
:10ECF000014878003E0090000080E8001E4878003F
:10ED0000310020003E00900050000700704080005D
:10ED1000004088002E009000000040001040880055
:10ED20000000EB00204088007140800040832000FC
:10ED300000804000304088000000EB004040880028
:10ED40000000EB00504088009560A800C081800062
:10ED50003140800004408000800178001E01900056
:10ED6000040078000C880200000000000FFF37004C
:10ED7000BE0090000040EB00804878003E0090000C
:10ED80008000E8000040EB0080487800110020007F
:10ED90003E0090002D00070004FF37000080FA00BD
:10EDA000000006000200FA00004F7800CAC2A90065
:10EDB000CB22A900CB02A900CB42A900CA02A9001C
:10EDC00020C0B3009E4F100006003A00CAC2A8003F
:10EDD000CB02A800CB22A800CB42A800CA02A80000
:10EDE00005003700CAC2A900CB02A900CB22A900A6
:10EDF000CB42A900CA02A90010C0B3009E4F100068
:10EE00000300320020C0B3009E4F100007003A00FC
:10EE1000C8C2A900C922A900C902A900C942A90003
:10EE2000C802A900C8E2A80006003700C8C2A800AE
:10EE3000C922A800C902A800C942A800C802A800A7
:10EE4000C8E2A8000080FA00000006000600FA00F0
:10EE500010079800210798000000EB00000F7800D1
:10EE6000070037009E0078001E00900000804000E0
:10EE700010407800E45A0200000000001E0FE80075
:10EE80002E0090009E0F1000F6FF39000080FA005F
:10EE9000000006000400FA00004F780011479800B7
:10EEA0001E80FB00100798001E009000E40F500029
:10EEB0002F0032001E009000E40F500007003C00BD
:10EEC0001E009000E10F50000B0032001E00900069
:10EED000E20F500014003200390037001E0090008D
:10EEE000E80F50002C0032001E009000F00F500080
:10EEF0001600320032003700C022A9001E409000E8
:10EF0000614060006140600000414000212C200011
:10EF100091407800D0CFB30000C060000240700084
:10EF2000C2E2B700260037001E4090000004E00057
:10EF300003003200C002A900C202A800200037006E
:10EF4000C002A900C202A9001D0037001E409000A7
:10EF50000004E00003003200C962A800CB62A900EF
:10EF600017003700CB62A900C962A900140037005E
:10EF70001E4090006140600061416000A12C2000B3
:10EF800091407800E0CFB30000C060000240700004
:10EF9000CAE2B7000A0037001E40900061406000DE
:10EFA000614060004201DD00B12C200091407800FA
:10EFB000B0CFB30000C0600002407000CBE2B700E9
:10EFC0000080FA00000006000000FA0040168000F1
:10EFD000017C20000100700040168800110007002D
:10EFE00020C0B3002D000700C65A02000000000038
:10EFF0000004E00005003200D25A020000000000C8
:10F00000260007000004E00004003A003601070073
:10F010000004E00001003A00F3FF37000080FA002E
:10F02000000006000000FA00C222A9000000EB0068
:10F03000400388000000EB00500388000000EB0054
:10F04000000388000000EB00100388000000EB00C4
:10F05000F0088800D10A200091407800F0C8B30081
:10F0600000C06000ADE0B7000000EB00E0088800E1
:10F0700000642000D008880000002100405E880065
:10F080008040EB0060BC2000014878000000EB00ED
:10F09000A05D88000080FA00000006000A00FA0067
:10F0A000004F7800F05D800040079800CE0090008F
:10F0B000E18F5000440032004E019000E10F5100FA
:10F0C000040039004E009000E20F50004F00320063
:10F0D000000137009E80FB00310798003E01900040
:10F0E000E20F5100150032003E009000E20F500088
:10F0F00007003C00BE0090000100E0000B00320061
:10F100003E019000E10F5100100032002300370053
:10F110003E009000F10F5000EE003200BE00900063
:10F12000F38F5000EB0032001C003700BDFF0700DA
:10F130001200200022079800E8003700A08D280068
:10F140008856020000000000E2003700C222A8003A
:10F150000000EB00F00888000000EB00B008880019
:10F160000000EB00A008880080002000F008880064
:10F170008660A9009660A900D10A2000914078001D
:10F18000F0C8B30000C060000044A000ADE0B700CC
:10F1900010002000A05D8800CE00370060BB20007A
:10F1A0001E48780041C0B300B0BB20000148780081
:10F1B0008040EB00C0BB2000014878001000200018
:10F1C000F05D8800C3003700C0BB2000104078000D
:10F1D0008040E800C0BB200001487800C0BB200090
:10F1E000104078008080FB0060BB20000080400061
:10F1F0001E487800C0BB200090407800B0BB2000C3
:10F200001040780080CF5000B200390060BB200071
:10F21000104078000080FB001007980010082000C4
:10F220009E009000808F50003E003200000C2000B5
:10F230001E019000800F51000500320000082000E0
:10F240009E009000808F50004E0032009F003700DB
:10F2500070BB2000104078000080FB004400DE00FE
:10F26000610060000004E000030032001003800031
:10F270000000A0001003880070BB20001040780040
:10F280000080FB004300DE00610060000004E0003D
:10F290000400320010038000010220000100700011
:10F2A0001003880070BB2000104078000080FB0035
:10F2B0004200DE00610060000004E0000400320053
:10F2C000100380000104200001007000100388007A
:10F2D00070BB2000104078000080FB000000D100CF
:10F2E000610060000004E0000400320010038000B0
:10F2F00001082000010070001003880070BB20008E
:10F30000104078000080FB00610060000004E00015
:10F310000400320010038000011020000100700082
:10F320001003880080BB2000104078000080FB00A4
:10F33000405E8800405E80004800DD00405E88003E
:10F3400070BB2000104078008080FB00405E800091
:10F3500000807000405E8800405E80004200DD005A
:10F3600064004000405E8800415E80000000210093
:10F37000808F50005500360000002100405E88005C
:10F380005200370090BB2000104078000080FB0046
:10F3900001002000005E8800115E8800005E800091
:10F3A000115E8000C808DD000080FD00804078000C
:10F3B0000040EB00005E8800115E880080BB2000EA
:10F3C000104078000081FB0003002000005E8000F8
:10F3D000115E80000000710081807100005E880075
:10F3E000115E8800005E8000115E8000C808DD00AC
:10F3F0000080FD00804078000040EB00005E880047
:10F40000115E880070BB2000104078000081FB0076
:10F4100003002000005E8000115E8000000071008B
:10F4200081807100005E8800115E8800005E8000AF
:10F43000115E80004209DD00CE00DE008100710017
:10F440004200DD0064004000E0804800920120009E
:10F4500003002000A005020000000000005E8800FC
:10F46000115E8800025E8000135E800000012000B3
:10F4700001002000800F5100818F590007003600E5
:10F48000005E8000115E800070005000E080580037
:10F49000005E8800115E8800040037001000200024
:10F4A00001002000005E8800115E8800005E800080
:10F4B000115E80004008DE0001002000E0088800A6
:10F4C000005E8000115E8000D00888000000EB0024
:10F4D000F05D88000000EB00200798002E009000EF
:10F4E0000080FA00000006000200FA00A05D800023
:10F4F000E10F5000010032003600370086C0BF0027
:10F50000684060000004E00003003A00100380003F
:10F510000000E0002F003A001FE1A8008780A9004A
:10F520000000EB00205E88000E0037007140800074
:10F53000205E800080804000501680004600DE0083
:10F540008048780087C0BF00704060000004E00081
:10F55000FCFF32008780A900205E80000000E800E8
:10F56000205E8800215E8000405E8000808F500019
:10F57000EEFF39000000EB00100388000000EB00F4
:10F58000F0088800405E8000205E88000A00370096
:10F5900071408000205E8000008040000000E90093
:10F5A00010407800E45A020000000000205E800055
:10F5B0000000E900205E8800205E80000000E0007E
:10F5C000F3FF3A0097FE070010002000000F7800BC
:10F5D000020037000000EB00000F78001E007800EA
:10F5E0000080FA00000006000000FA00F00F200082
:10F5F0002A6B0200000000000080FA0000000600F4
:10F600000400FA00000F78001E0078002A6B020048
:10F6100000000000000F7800A09C2000104078003F
:10F620000044B2000004E000030032001E00780035
:10F6300010079800020037000000EB001007980048
:10F640001E0090000080FA00000006000000FA0092
:10F65000A09C2000104078000060A000A19C200029
:10F6600080487800209D20001040780061406000B4
:10F670000004E000040032000040EB00CC6C02000B
:10F68000000000000300370010C0B300CC6C020083
:10F6900000000000209D20001040780061406000C4
:10F6A0000004E00003003200F0C2B300E45A02009C
:10F6B00000000000A100200060AB200024850200B3
:10F6C000000000000080FA00000006000000FA00C0
:10F6D000A09C2000104078000060A100A19C2000A8
:10F6E00080487800209D2000104078006140600034
:10F6F0000004E000040032000040EB00CC6C02008B
:10F70000000000000300370010C0B300CC6C020002
:10F7100000000000209D2000104078006140600043
:10F720000004E00003003200F0C2B300E45A02001B
:10F7300000000000A100200060AB20002485020032
:10F74000000000000080FA00000006000000FA003F
:10F75000A09C2000104078000060A100A19C200027
:10F7600080487800209D20001040780061406000B3
:10F770000004E0000400320010C0B300CC6C0200B2
:10F7800000000000030037000040EB00CC6C0200DA
:10F7900000000000209D20001040780061406000C3
:10F7A0000004E00003003200F0C2B300E45A02009B
:10F7B00000000000B100200000AC20002485020001
:10F7C000000000000080FA00000006000000FA00BF
:10F7D0003E6C0200000000000080FB000080FA0088
:10F7E000000006000000FA00DE6C020000000000CD
:10F7F0000080FB000080FA00000006000000FA0014
:10F8000010C0B300826C0200000000000080FA000B
:10F81000000006000000FA0010C0B300BA6C02003D
:10F82000000000000080FA00000006000000FA005E
:10F830000040EB00BA6C0200000000000080FA00FB
:10F84000000006000000FA0010C0B300A86C02001F
:10F85000000000000080FA00000006000000FA002E
:10F860000040EB00A86C0200000000000080FA00DD
:10F87000000006000000FA0041012000B0AC2000AA
:10F880009A84020000000000809B20001040780055
:10F89000205902000000000000C2B300E45A020038
:10F8A00000000000209D20001040780061406000B2
:10F8B000205902000000000000C2B300E45A020018
:10F8C00000000000A09C2000104078000080FB0099
:10F8D0004400DE006140600020590200000000008A
:10F8E00000C2B300E45A020000000000A08E28000D
:10F8F000B4560200000000000080FA00000006007C
:10F900000600FA0008200200000000003A1C020075
:10F9100000000000200798000820020000000000FE
:10F920003A1C020000000000000F780008200200CE
:10F93000000000003A1C02000000000010079800C0
:10F940002E0090000000E000090034002E0090001E
:10F95000E40F500006003C002E0090000040E9003B
:10F9600080407800809B200001487800020037002A
:10F970000000EB00200798001E00E0000F0034009C
:10F98000200020009E0F10000C003C001E0078009C
:10F990000040E900E1406000209D20001040780018
:10F9A00061C16000E1CFB30001406000024070001F
:10F9B000219D200080487800020037000000EB0005
:10F9C000200798001E0090000000E00010003400A6
:10F9D0001E009000E20F50000D003C001E00900041
:10F9E0000040EA0061416000A09C20009040780047
:10F9F000614061004401DD00F0CEB30080C06000D2
:10FA000082C07000A09C20000148780002003700EE
:10FA10000000EB00200798002E0090000000E0009E
:10FA20003A003A00B103200060482000248502001B
:10FA3000000000008001EB004200200011002000C7
:10FA40001000200034210200000000000040E90006
:10FA500080407800809B200001487800D101200080
:10FA60007022210024850200000000008001EB00CC
:10FA7000220020001100200020002000342102007C
:10FA8000000000000040E900E1406000209D2000EF
:10FA90001040780061C16000E1CFB3000140600018
:10FAA00002407000219D200080487800F104200071
:10FAB000B093200024850200000000008001EB00CC
:10FAC000220020001100200010002000342102003C
:10FAD000000000000040EA0061416000A09C20009E
:10FAE00090407800614061004401DD00F0CEB30039
:10FAF00080C0600082C07000A09C20000148780097
:10FB00000000EB00905788000100370059FF070004
:10FB1000A09C2000104078000060A100A19C200063
:10FB200080487800A09C2000104078000050A10080
:10FB3000A19C200080487800809B200090407800A5
:10FB400030C0B3003C6A020000000000C922A900D6
:10FB5000C902A900C8E2A800209D2000104078003A
:10FB600061406000CC6C0200000000000080FA00E0
:10FB7000000006000000FA0001012000A00421009E
:10FB800024850200000000000080FA00000006004A
:10FB90000200FA00004F7800114798008040EB0007
:10FBA000A0B92000014878001E04E00003003A00DC
:10FBB000D04080000080A000D04088001E04E000FB
:10FBC000110032001E4090000004E0000E003200E0
:10FBD000F103200020AE2000248502000000000078
:10FBE00011012000B01F2100248502000000000048
:10FBF000C65A0200000000000004E000FCFF3200D2
:10FC0000D25A0200000000004100200010B2200083
:10FC10002485020000000000CB42A800C942A900D0
:10FC20003100200050B220009A8402000000000041
:10FC3000CBC2BF000080FB004200DE0061406000DC
:10FC400011C0B30011010700CB42A900C942A800AE
:10FC5000C222A800C022A9008100200080B220009A
:10FC60009A84020000000000C2C2BF000080FB00B6
:10FC70000000D1006140600011C0B3000301070023
:10FC8000C222A900C962A800CB62A900810020009D
:10FC900000B320009A84020000000000CBC2BF0025
:10FCA0000080FB004300DE006140600011C0B30033
:10FCB000F6000700CB62A900C962A90081002000FC
:10FCC00080B320009A84020000000000CBC2BF0075
:10FCD0000080FB004300DE00614060008040EB00DC
:10FCE000EA000700C002A900C202A800200020000C
:10FCF00050820200000000004100200000B42000FB
:10FD00009A84020000000000C2C2BF00614060008F
:10FD100011C0B300DD000700E100200040B4200066
:10FD2000248502000000000021E3A800210020003B
:10FD300020B520009A8402000000000072352000E7
:10FD4000712B200090C0B300860007001E40900079
:10FD50000004E000080032003100200040B520001F
:10FD60009A8402000000000072352000712B2000F0
:10FD7000B0C0B3007B0007004100200070B5200038
:10FD80009A8402000000000002252000011B2000D0
:10FD9000A0C0B300730007001E4090000004E00004
:10FDA0000800320031002000B0B520009A84020023
:10FDB0000000000002252000011B2000C0C0B3008D
:10FDC0006800070021E3A90081002000E0B52000C1
:10FDD000248502000000000041168000F0C32F00BF
:10FDE000008060004016880061168000003C200002
:10FDF00000807000601688004006200050820200DB
:10FE00000000000010C0B30077000700A100200030
:10FE100060B620002485020000000000611680000A
:10FE2000F0C32F0000806000601688001E40900024
:10FE30000004E00002003200C962A800CB62A90001
:10FE40004006200050820200000000000040EB004D
:10FE5000650007001E4090000004E0000D00320025
:10FE6000A100200000B7200024850200000000004F
:10FE700040168000013C2000010070004016880000
:10FE800040062000508202000000000010C0B300B5
:10FE9000550007001E04E0001C0032001E409000C8
:10FEA0000004E00019003200C002A900C202A8004C
:10FEB000201680000010A0002016880001022000FB
:10FEC000A0B720002485020000000000F1002000FF
:10FED000C01E21002485020000000000C65A020056
:10FEE000000000000004E000FCFF3200D25A0200D3
:10FEF0000000000020168000D1FF2F0001006000EC
:10FF000020168800C002A900C202A900A880020031
:10FF10000000000061002000A0B920009A840200C7
:10FF200000000000A0B92000104078002059020015
:10FF3000000000008100200000BA2000248502009B
:10FF400000000000D04080000080A100D040880068
:10FF5000A0B92000104078000080FB000080FA006B
:10FF6000000006000A00FA002047980021079800C8
:10FF70003207980080C2B300E45A0200000000007B
:10FF80002E409000F280020000000000000F780078
:10FF90001E007800245A02000000000090C2B30046
:10FFA000E45A0200000000002E0090009E0F100096
:10FFB000060036003E0090009E0F10000300310046
:10FFC0001000200040079800020037000000EB00FE
:10FFD000400798000E48900011C0B3002B000700A6
:10FFE0000080FA00000006000200FA00004F7800CE
:10FFF0004100200080BA20009A8402000000000026
:020000040001F9
:10000000CBC2BF000080FB000000D1006140600057
:100010009E4078001D00070031002000C0BA20007B
:100020009A84020000000000CBC2BF006140600063
:100030009E4078001500070041002000F0BA200023
:100040009A84020000000000CAC2BF000080FB00CA
:100050004700DE009E4078000C00070021002000D1
:1000600030BB20009A84020000000000CAC2BF001A
:100070000080FB004600DE00614060009E4078008A
:10008000020007000080FA00000006000200FA00EB
:10009000004F7800114798001E4090009E4F1000BE
:1000A00005003A003100200050BB200024850200EA
:1000B00000000000090037005100200080BB200034
:1000C0002485020000000000A0B920001040780044
:1000D0008040E800A0B92000014878000080FA00C4
:1000E000000006000000FA00A09C200010407800EC
:1000F0000040A100A19C2000804878008040EB00D7
:10010000809B200001487800A09C200010407800CF
:100110000020A100A19C200080487800A09C200025
:10012000104078000000A1000010A100A19C200058
:1001300080487800A09C2000104078000030A1008A
:10014000A19C2000804878000080FA000000060092
:100150000000FA00C922A800C902A800C8E2A8004D
:10016000C8C2A800C942A800C222A900C022A90092
:10017000A16C20009140780000CEB30000C0600068
:10018000CAE6B7000000EB00A0408800D5FF0700DA
:10019000CB62A900C962A900C002A900C202A900DD
:1001A0002D83A9002D43A9002D23A9002D63A900AB
:1001B000013220009140780000CEB30000C07000F2
:1001C00020E3B7000000EB008019880020F0210038
:1001D000201988000000EB00101988000080FA0048
:1001E000000006000200FA00004F78001E80FB00AD
:1001F000401988002023A8002003A90020C3BF00C5
:10020000614060000004E000FCFF32000018800044
:100210000080FA00000006000000FA0021E3A800B8
:10022000C0C0B300EFFF0700245A02000000000026
:1002300021E3A9000080FA00000006000200FA0095
:10024000E1002000C03820002485020000000000EA
:10025000F1002000C01E21002485020000000000E3
:10026000F1002000A03920009A8402000000000064
:100270000000EB00245A02000000000011002000E2
:10028000903A20009A840200000000000F0037001E
:1002900021E3A800C0C0B300D2FF0700000F780020
:1002A00021E3A900008C280088560200000000000D
:1002B0001E007800245A02000000000011002000F7
:1002C000903A20009A84020000000000C65A020002
:1002D000000000000004E000EDFF3200D25A0200EE
:1002E00000000000608C2800B456020000000000EE
:1002F0000080FA00000006000000FA0000812000E3
:1003000010407800E94F50000800320000812000C2
:10031000104078000080FB0080004000E081200059
:100320000080400010007800401188000000EB00C1
:10033000001188002062A8000000EB001011880066
:1003400021E2A8002342A8008560A9000080FA00ED
:10035000000006000400FA00000F7800909B2000C7
:1003600010407800EF4F500007003E00909B2000A7
:10037000104078000080FB00EF001000F0FF270025
:100380000180DE001E0F6000904080001007980082
:100390001E009000E10F5000170032001E00900078
:1003A000E10F5000070039001E009000E20F5000DE
:1003B0001E0032001E009000E30F50002A003200A1
:1003C00035003700A09C2000104078000042B200A9
:1003D0000004E000040032001E007800DA59020038
:1003E000000000002C0037001E0078008259020037
:1003F0000000000028003700A09C2000104078007A
:100400000042B2000004E000040032001E00780048
:10041000C2580200000000001F0037001E007800D4
:1004200020590200000000001B003700A09C2000A3
:10043000104078000042B2000004E00006003200E4
:100440001E007800E85602000000000000C2B30061
:10045000E45A0200000000001E007800E856020086
:10046000000000000C003700A09C20001040780025
:100470000042B2000004E000040032001E007800D8
:100480004800DE00E45A0200000000001E00780070
:10049000E45A0200000000000080FA00000006009C
:1004A0000600FA00200798000000EB00000F78001B
:1004B0000C0037000000EB00100798000500370023
:1004C000A00F20000C0007001E0090000000E800B4
:1004D000100798001E009000E30F5000F8FF340052
:1004E0001E0FE8002E0090009E0F1000F1FF350057
:1004F0000080FA00000006000400FA0010079800CF
:100500000000EB00000F7800110037000000000031
:1005100000000000000000000000000000000000DB
:1005200000000000000000000000000000000000CB
:1005300000000000000000000000000000000000BB
:100540000000000000000000000000001E0FE80096
:100550001E0090009E0F1000ECFF35000080FA0096
:10056000000006000600FA00200798000000EB00DB
:100570001007980010002000000F78000D003700D1
:100580001E00900000004000100798002E00900010
:100590001E0060000000E000030032001E0090001A
:1005A0000000A000100798001E0078000000400026
:1005B000000F78001E00E000F1FF3A00909B200041
:1005C00010407800F04F500007003200909B200050
:1005D000104078000080FB00F00010001E0090002A
:1005E0000100DE00100798001E0090000080FA0055
:1005F000000006000C0800001200000002000000CD
:1006000000003A00100000000000000000000000A0
:100610000000000000000000B80900001A000000FF
:10062000000000003A100000001000000000000070
:10063000D209000002000000000000001E080000B7
:100640001200000002000000143404000D820600B5
:100650004003A00001CF000067004400002200001A
:10066000D40900000800000000000000DC090000C0
:1006700012000000000000003008000042010000ED
:1006800002000000E486E40086E48600E486F600CA
:10069000860C8700E486E40086E48600E4860C008D
:1006A00087E486000C870C008720870034874A0087
:1006B000876087006E874800695A000000000000CC
:1006C00000F26D00F26D0C006E0C6E00E26DD80051
:1006D0006D4A6E003E6E6E006E626E00326E5600A7
:1006E0006E266E000C8776006FB26E004A87AE00F1
:1006F0006F7A6E00325749005245000000006600D4
:100700007B267B00A67BA6007B007B00F47A0A0098
:100710007C167C00227C2E007CF27B00FE7BE600B7
:100720007B0C8700208780007C4A8700BA7D3A00D6
:100730007C3357004952450000000000E486E40085
:1007400086E48600E486620066526600E486E40081
:1007500086E48600E4860C0087E486000C870C00A3
:100760008798660040664A00876087006E874B0066
:100770004559420000000000008C71008C71A400FB
:1007800071A4710072710C0087E48600E486E400B5
:1007900086E486000C87E400860C87000C871A002C
:1007A00072BC710084748400736E87004C434400F3
:1007B000000000000000E40086E48600E486E40017
:1007C000862089001889E40086E48600E486E40037
:1007D000860C8700E4860C00870C870020871200B7
:1007E000894A870060876E00874449004F000000F7
:1007F00000000000000000000000000000000000F9
:1008000000000000000000000000000000000000E8
:1008100000000000000000000000000000000000D8
:1008200000000000000000000000000000000000C8
:1008300000000000EE090000A80100000000000018
:10084000960B0000040000000000000000080000FB
:100850000C000000000000009A0B000002000000E5
:10086000000000009C0B00000A00000000000000D7
:10087000A60B00000400000000000000AA0B00000E
:100880000A00000000000000B40B00001600000089
:100890000000000072090000460000000200000095
:1008A000C887CC0087CF8700D487D90087DE870030
:1008B000E487EB0087EF8700F587FB0087FF870061
:1008C00002880700880C880011881800881E88009C
:1008D00024882900882E880036883A00883E8800BF
:1008E00046884A008851880055885C0088628800E4
:1008F00066886B0088708800768800000000000021
:10090000CA0B000068040000000000003210000064
:10091000020000000000000034100000040000008D
:10092000000000003810000002000000000000007D
:10093000000000000600FA00100798002107980048
:100940001E009000000F7800380037001E0078006D
:1009500032002000110009000200D8008000FD00D4
:100960000000E0000B003A001E007800320020007A
:10097000110009000200D80000004000800078004B
:10098000608F2300008040001000BA00E45A02008B
:10099000000000001E007800320020001100090055
:1009A0000200D8008000FD00E10F50000C003A006A
:1009B0001E00780032002000110009000200D8005B
:1009C0000000400080007800608F2300008040001D
:1009D0001000BA004800DE00E45A020000000000E7
:1009E0001E00780032002000110009000200D8002B
:1009F0008000FD00E20F50000B003A001E0078005E
:100A000032002000110009000200D8000000400060
:100A100080007800608F2300008040001080BA00C2
:100A2000E45A0200000000001E0FE8001E009000C3
:100A3000AE009000010040009E0F5000C3FF3C003C
:100A40000080FA00000006000400FA00000F7800A1
:100A5000110798009E0090001E007800B5FF070067
:100A6000E08E2800B4560200000000000080FA006A
:100A7000000006000000FA000102200030262100DC
:100A8000F1FF0700B104200030282100EEFF07002D
:100A900051022000E02C2100EBFF07007102200032
:100AA000302F2100E8FF070041012000A031210084
:100AB000E5FF070011012000E0322100E2FF0700FE
:100AC00071022000F0332100DFFF0700A1012000A8
:100AD00060362100DCFF0700D10220000038210031
:100AE000D9FF070041012000D03A2100D6FF0700BE
:100AF00021022000103C2100D3FF0700D10220007A
:100B0000303E2100D0FF0700B1012000004121004C
:100B1000CDFF070001022000B0422100CAFF0700FC
:100B2000B1012000B0442100C7FF070041022000AE
:100B300060462100C4FF070001022000A0482100F8
:100B4000C1FF070081012000A04A2100BEFF07006D
:100B5000E1012000204C2100BBFF070081022000A2
:100B6000004E2100B8FF0700410220008050210004
:100B7000B5FF070051032000C0522100B2FF07005B
:100B8000D103200010562100AFFF07000080FA00BB
:100B9000000006000400FA00E1002000409120005F
:100BA00064FF0700C65A0200000000000004E000D5
:100BB000FCFF3200D25A020000000000004F780013
:100BC0001E407800E45A020000000000E08E280079
:100BD000B45602000000000090C7B3009E4F100002
:100BE0000300320090C5B3009E4F100003003A008E
:100BF0001000200010079800020037000000EB00F2
:100C0000100798001E0090000080FA000000060007
:100C10000600FA00000F780021479800324798003C
:100C200043479800544798002E4090006140600070
:100C30006140600000414000F12C200091407800AC
:100C4000D0CFB30000C0600002407000CFE2B70018
:100C5000616A20009140780000CEB30000C06000BF
:100C60007040B300A6E6B700916C20009140780078
:100C700000CEB30000C060005040B300C9E6B7002A
:100C80001E007800C01188000000EB008011880071
:100C90003062A8003E40900061406000614060000A
:100CA0004401DD000123200091407800F0CEB30024
:100CB00000C060000240700030E2B7004E4090007B
:100CC0006340600063406000004140000123200059
:100CD0009140780090CFB30000C0600002407000E7
:100CE00030E2B7005E40900061406000614160000A
:100CF0000123200091407800E0CFB30000C06000E5
:100D00000240700030E2B7000000EB009011880054
:100D10000080FA00000006000000FA0031E2A8009E
:100D20003342A80087C0A9000080FA000000060036
:100D30000000FA0031E2A9003342A900A6C6BF00B4
:100D4000F041B300A6E6B700616C20009140780046
:100D500000CEB30000C06000C6E6B700CF22A900F5
:100D60000080FA00000006000200FA00000F780080
:100D700033C2BF00624060000004E000FCFF3A00A4
:100D80001E007800A01188000080FA000000060014
:100D90000000FA0032C2BF00614060000004E000C1
:100DA000FCFF3200B01180000080FA000000060055
:100DB0000000FA0032C2BF00614060000080FB000A
:100DC0000080FA00000006000000FA001102200076
:100DD00000422000248502000000000010002000D6
:100DE000905788000080FA00000006000200FA0018
:100DF000000F78001102200000422000248502002C
:100E00000000000010002000905788000010200013
:100E10000080FA00000006000000FA001102200025
:100E20000042200024850200000000001000200085
:100E3000905788000000EB000080FA0000000600D8
:100E40000200FA00000F780011022000004220008A
:100E50002485020000000000100020009057880048
:100E60000080FA00000006000000FA0081C0B30014
:100E7000909B200001487800A09C20001040780042
:100E80000050A100A19C2000804878000080FA005A
:100E9000000006000000FA0081C0B300909B200013
:100EA00001487800A09C2000104078000050A1006C
:100EB000A19C2000804878000080FA000000060015
:100EC0000000FA0001012000A00421002485020096
:100ED000000000000080FA00000006000000FA0098
:100EE000C08E2800B4560200000000000080FA0006
:100EF000000006000000FA0005000700F2080200EA
:100F0000000000000000EB000080FA000000060076
:100F10000000FA004507A9000080EB006019880076
:100F20004227A900416A20009140780000CEB3001A
:100F300000C060005040B300A4E6B700416C200040
:100F40009140780000CEB30000C060003040B30094
:100F5000C4E6B70081C0B3000081200001487800DA
:100F60000000EB0090408800A88002000000000014
:100F70007C8102000000000068C0A8008000EB0037
:100F8000F00F20003E5C020000000000B04088002E
:100F900021002000F00F20003E5C02000000000055
:100FA000C0408800CAC2BF00644060000004E00086
:100FB0000400320011C6B300A0812000014878006F
:100FC0000300370021C6B300A0812000014878004B
:100FD00068C0A900D04080000080A100D0408800F7
:100FE00081C0B300909B200001487800C038020007
:100FF000000000000000EB0090018800608E2800D7
:10100000B456020000000000B222020000000000FE
:101010000080FA0000000600889FBE008A9FBE0084
:101020008C1F78008002EB000203E9008003780047
:101030000104780003067800A92C20009A00200003
:101040006B00200010408000E48242000028E6008F
:10105000050078000408E300FEFF35003701780042
:10106000B70178000280FD0003026900F40FB200AE
:1010700004016900848169000280FD00F000200005
:101080000030E60006007800800078000C8009003F
:10109000000000001980A1000281D3001950AD00AA
:1010A0008381D3001958AD000C80090000000000B6
:1010B0001980A0001970A3000482D3008100E90008
:1010C000F2FF3100EF0010000122DE00041C780066
:1010D0004300DE000000E8000A28B4009580AB0061
:1010E00008003200404080000A08E300050032009A
:1010F0008580A9009580A8000608B400100078003B
:101100002011880070035300CEFF31004F06780095
:101110004F05BE004F04BE000E5B0400000000003F
:101120000200FA00004F78001E80FB004300DE0042
:10113000610060000004E00003003200C002A9006A
:10114000C202A80002003700C002A900C202A90022
:101150001E80FB004200DE00610060000004E00031
:1011600003003200C962A800CB62A9000200370068
:10117000CB62A900C962A9001E80FB000000D1005B
:10118000610060000004E00003003200C942A900D1
:10119000CB42A80002003700C942A900CB42A900F7
:1011A0001E80FB00610060000004E00013003200BC
:1011B000A09C200010407800704060000004E00017
:1011C000050032004016800001042000010070007C
:1011D00040168800110037006116800000042000CE
:1011E000008070006016880041168000F0FB2F0020
:1011F00000806000401688000800370061168000FB
:10120000F0FB2F000080600060168800411680000F
:10121000F0FB2F0000806000401688000080FA007C
:10122000000006000000FA000080FA00000006003E
:101230000000FA00501680000080FA00000006004E
:101240000400FA00000F78001E0078004700DE005E
:101250000000A200610060000004E000060032000F
:101260001E007800825E0200000000000080FB008B
:1012700010079800050037001E007800A25F0200EA
:10128000000000000080FB00100798001E00900086
:101290000080FA00000006000000FE00FFFFFF00D3
:1012A000FFFFFF00FFFFFF00FFFFFF00FFFFFF004A
:1012B000FFFFFF00FFFFFF00FFFFFF00FFFFFF003A
:1012C000FFFFFF00FFFFFF00FFFFFF00FFFFFF002A
:1012D000FFFFFF00FFFFFF00FFFFFF00FFFFFF001A
:00000001FF
